:100000000C94822A0C9452930C9427930C94FC9297
:100010000C94D1920C94A6920C947B920C945092D6
:100020000C9425920C94B32A0C94B32A0C94B32A02
:100030000C94B32A0C94D4930C94B32A0C94B32A42
:100040000C94B32A0C9434620C94B32A0C94B32A03
:100050000C94B32A0C94B32A0C947A880C947D9552
:100060000C94B32A0D9495280D9439290C94B32A35
:100070000C94B32A0C94B32A0C94B32A0C94B32A8C
:100080000C94B32A0C94B32A0C94B32A0C94B32A7C
:100090000C94B32A0C94B32A0C94B32A0C94B32A6C
:1000A0000C94B32A0C94B32A0C94B32A0C94B32A5C
:1000B0000C94B32A0C94B32A0C94B32A0C94B32A4C
:1000C0000C94B32A0C94B32A0C94B32A0C94B32A3C
:1000D0000C94B32A0C94B32A0C94B32A0C94B32A2C
:1000E0000C94B32A8C8E8F8E7E8E828E888EC68ED6
:1000F000938E978E9D8EA18EA58EAB8EAF8EB38E76
:10010000C68EB98EBD8EC18E99949E94A394AD94E3
:10011000B7943095C194C994D194DB94E594EF944D
:10012000FE940895309512951C95269544F42AF472
:100130002DF430F433F43FF436F44DF439F43CF458
:10014000F600F2000201E800E600FE00F000FE000A
:10015000E400E200FE00EA00E000E000F400F40049
:10016000F400000100010001FA00DE00DE00DE0004
:10017000084AD73B3BCE016E84BCBFFDC12F3D6C0E
:1001800074319ABD56833DDA3D00C77F11BED9E474
:10019000BB4C3E916BAAAABE000000803F05A84C54
:1001A000CDB2D44EB93836A9020C50B99186880820
:1001B0003CA6AAAA2ABE000000803F000D94ED2BA9
:1001C0000D94D82B0D94FA280D94F6280D94EE2852
:1001D0000D94E6280D9400290D9468150D94C61C05
:1001E0000D94F2280D94CA280D94DF2B0D94C42889
:1001F0000D9490250D94F32B0D94961D0D940329C9
:100200000D94E62B0D94DB280D949C1E4E414E4917
:100210004E495459494E46CDCCCC3D0AD7233C17C4
:10022000B7D13877CC2B329595E6241FB14F0A0011
:100230000020410000C84200401C4620BCBE4CCA01
:100240001B0E5AAEC59D74434F4D4D554E4943410B
:1002500054494F4E0044525952554E004552524F48
:10026000525300494E464F004543484F0020746F9B
:100270006F206C6F6E6720657874727573696F6E2E
:100280002070726576656E7465640A0020636F6C19
:100290006420657874727573696F6E20707265760C
:1002A000656E7465640A0047322F473320626164CB
:1002B00020706172616D65746572730A00536C65BC
:1002C00065702E2E2E0050726F62696E6720666117
:1002D000696C6564004D31313720426564206C657E
:1002E00076656C696E67206661696C65642E0A4785
:1002F00030205A31300A47302045300A4D333030F3
:100300002050323520533838300A4D3330302050A9
:1003100035302053300A4D333030205032352053A1
:100320003838300A4D333030205035302053300AC1
:100330004D3330302050323520533838300A47346E
:10034000205331004D3131372050726F6265207378
:1003500075636365737366756C0A0050524F42454E
:10036000204641494C20434C45414E204E4F5A5A5D
:100370004C450A004D31303920523137300A4D3169
:100380003137205265776970696E67206E6F7A7AAF
:100390006C650A4730205A31300A4D3130392052CD
:1003A0003137300A4D313137205265776970696EC7
:1003B00067206E6F7A7A6C650A47313220503020A0
:1003C0005331322054300A4D3130342053313630DD
:1003D0000A4D3131372050726F62696E6720626555
:1003E0006400205A3A200020593A200042656420D7
:1003F000583A2000456E642066696C65206C69730C
:10040000740A00426567696E2066696C65206C69D4
:1004100073740A004D313235005072696E74207465
:10042000696D653A2000000125301D0C182829FF50
:1004300024311C0B174527FF232F1B0A1E4443FFA3
:10044000FF16040308060202222B1A4142FF03385A
:1004500009FF3646696C616D656E7420757365645D
:100460003A200053746174733A20002C204C6F6E54
:1004700067657374206A6F623A2000546F74616C10
:100480002074696D653A200053746174733A2000DA
:100490002C204661696C65643A20002C2046696E08
:1004A00069736865643A20005072696E74733A200B
:1004B0000053746174733A2000680263025C025551
:1004C0000247026F66660044454255473A004D3187
:1004D00031332053006F6B0020573A004578747217
:1004E0007564657220436F6F6C696E672E2E2E00E7
:1004F00045787472756465722048656174696E67C9
:100500002E2E2E0020573A0042656420636F6F6CD8
:10051000696E672E2E2E00426564206865617469DD
:100520006E672E2E2E004C756C7A426F74205441EB
:100530005A2036204F66662E00544845524D414C95
:100540005F50524F54454354494F4E004155544F0C
:100550005245504F52545F53445F53544154555386
:1005600000454D455247454E43595F504152534512
:100570005200434153455F4C494748545F425249FA
:100580004748544E45535300544F47474C455F4CE2
:10059000494748545300534F4654574152455F50C2
:1005A0004F574552004255494C445F5045524345D0
:1005B0004E54004C4556454C494E475F44415441CA
:1005C000005A5F50524F4245004155544F4C4556DA
:1005D000454C005052494E545F4A4F420050524FD2
:1005E0004752455353004155544F5245504F525472
:1005F0005F54454D5000564F4C554D45545249435C
:1006000000454550524F4D0053455249414C5F58AB
:100610004F4E5F584F4646004649524D574152454E
:100620005F4E414D453A4D61726C696E20204649DE
:10063000524D574152455F56455253494F4E3A31FC
:100640002E312E392E3334204558545255444552BC
:100650005F545950453A48617264656E65645374DD
:1006600065656C20534F555243455F434F44455F8A
:1006700055524C3A68747470733A2F2F636F6465E7
:100680002E616C6570686F626A656374732E636F48
:100690006D2F646966667573696F6E2F4D41524C9C
:1006A000494E2050524F544F434F4C5F5645525382
:1006B000494F4E3A312E30204D414348494E455F17
:1006C000545950453A4C756C7A426F742054415AD3
:1006D00020362045585452554445525F434F554E9D
:1006E000543A3120555549443A3834356630303320
:1006F000632D616562642D346535332D6136623951
:100700002D3764303938346664653630390A002F45
:100710002F20007A5F70726F62653A20007A5F6DF9
:1007200061783A20007A5F6D696E3A2000795F6DDA
:1007300061783A2000795F6D696E3A2000785F6DCC
:1007400061783A2000785F6D696E3A2000526570DA
:100750006F7274696E6720656E6473746F70207356
:1007600074617475730A004D31343520533C696EE1
:100770006465783E206F7574206F662072616E67C5
:10078000652028302D31290A0050726F6265205A89
:10079000204F66667365743A200020643A00206931
:1007A0003A0020703A00496E76616C696420657881
:1007B0007472756465720A00426564204C657665E2
:1007C0006C696E6720004661696C656420746F20F7
:1007D000656E61626C6520426564204C6576656C6F
:1007E000696E670A00426564204C6576656C20433B
:1007F0006F7272656374696F6E204D61747269788F
:100800003A0020202020202846312E30203D20662E
:10081000756C6C20636F7272656374696F6E2C20E7
:1008200046302E30203D206E6F20636F72726563FC
:1008300074696F6E290A002020466164653A2020A1
:100840002020202020202020202020202020204682
:10085000002020536D6F6F7468696E6720286D6D7E
:10086000293A202020202020205300202044697392
:1008700074616E636520286D6D293A202020202048
:100880002020205A004261636B6C61736820636FA3
:100890007272656374696F6E206973206163746935
:1008A00076653A0A004261636B6C61736820636F1E
:1008B0007272656374696F6E20697320696E61631B
:1008C000746976653A0A004261636B6C61736820F3
:1008D0006D6561737572656D656E7420286D6D2927
:1008E0003A2020003F4B2076616C7565206F75744F
:1008F000206F662072616E67652028302D313029A7
:100900002E0A00416476616E6365204B3D004163B1
:10091000746976652045787472756465723A200052
:10092000496E76616C69642065787472756465726D
:100930000A0025753A2530327500253032753A2582
:100940003032750025756420253032753A253032F5
:10095000750000060900FE00000000000109000803
:10096000FE000005080806000040F0C88888987856
:1009700010050808060000C0F88888888888F805EF
:1009800005050600012030F83020050808060000A3
:100990002070F820202020E00509090600FF2070C3
:1009A000A8A8B8888870200509090600FFE080C063
:1009B000B0A8283028280509090600FFF8A888886B
:1009C000888888A8F8050A0A0600FE205050505072
:1009D00088A8A8887003030306000340A04000060F
:1009E0000900FE0701920321207FFF07FF07FF0098
:1009F000000006000001070706020080808080805A
:100A00000080030202060105A0A0050707060000FA
:100A10005050F850F850500507070600002078A005
:100A20007028F020050707060000C0C81020409875
:100A3000180507070600006090A040A89068020310
:100A400003060104C0408003070706010020408020
:100A500080804020030707060100804020202040BE
:100A60008005050506000120A870A82005050506DB
:100A700000012020F820200203030602FFC040806E
:100A8000050101060003F8020202060200C0C005CB
:100A90000505060001081020408005070706000034
:100AA0007088888888887003070706010040C04066
:100AB000404040E00507070600007088087080800D
:100AC000F8050707060000F81020100808F00507D1
:100AD0000706000010305090F810100507070600B8
:100AE00000F880F00808887005070706000070808D
:100AF00080F0888870050707060000F8081020209D
:100B00002020050707060000708888708888700517
:100B10000707060000708888780808700205050637
:100B20000200C0C000C0C00206060602FFC0C0002E
:100B3000C0408004070706000010204080402010BD
:100B4000050303060002F800F80407070601008009
:100B5000402010204080050707060000708808101C
:100B600020002005070706000070880868A8A87004
:100B7000050707060000708888F888888805070739
:100B8000060000F08888F08888F005070706000056
:100B900070888080808870050707060000F08888CC
:100BA000888888F0050707060000F88080F08080BC
:100BB000F8050707060000F88080F08080800507B0
:100BC00007060000708880B888887005070706004F
:100BD00000888888F88888880107070602008080D6
:100BE00080808080800507070600003810101010F4
:100BF00090600507070600008890A0C0A0908805B7
:100C00000707060000808080808080F805070706BF
:100C1000000088D8A888888888050707060000880B
:100C200088C8A89888880507070600007088888803
:100C3000888870050707060000F08888F0808080AB
:100C400005070706000070888888A89068050707D0
:100C5000060000F08888F0A09088050707060000CD
:100C6000788080700808F0050707060000F820204B
:100C700020202020050707060000888888888888AB
:100C800070050707060000888888888850200507B7
:100C9000070600008888888888A85005070706008E
:100CA000008888502050888805070706000088883B
:100CB0008850202020050707060000F80810204073
:100CC00080F8030707060100E08080808080E0054F
:100CD00005050600018040201008030707060100F3
:100CE000E02020202020E005030306000420508897
:100CF000050101060000F802020206020580400517
:100D000005050600007008788878050707060000CA
:100D10008080B0C88888F0050505060000708080D6
:100D20008870050707060000080868988888780515
:100D300005050600007088F88070050707060000AA
:100D40003048E0404040400506060600FF708888B5
:100D50007808700507070600008080B0C88888887A
:100D60000107070602008000808080808003080859
:100D70000601FF200020202020A0400407070600D5
:100D800000808090A0C0A090030707060100C0402B
:100D900040404040E0050505060000D0A8A8A8A8EE
:100DA000050505060000B0C8888888050505060009
:100DB0000070888888700506060600FFF08888F0B5
:100DC00080800506060600FF7888887808080505F3
:100DD00005060000B0C8808080050505060000708B
:100DE000807008F00407070600004040E0404040E3
:100DF0003005050506000088888898680505050601
:100E0000000088888850200505050600008888A80D
:100E1000A8500505050600008850205088050606E4
:100E20000600FF888888780870050505060000F828
:100E3000102040F803070706010020404080404092
:100E400020010707060200808080808080800307E1
:100E50000706010080404020404080050202060055
:100E600002689000000006000020202020202000C2
:100E70005A005900202020200058000920000000BE
:100E8000000000000000000000003FFFF000000034
:100E900000000000000000000038007000000000AA
:100EA000000000000000000030FC300000000000E6
:100EB0000000000000000020FC1000000000000006
:100EC000000000000000207810000000000000007A
:100ED00000000000002030100000000000000000B2
:100EE000000000002C00D03FC00000000000000007
:100EF0002082002E31D07FE00000000000000010B2
:100F000041002F7BD07FE000000000000000104176
:100F1000002F7BD07FE00000000000000020820056
:100F20002E31D03FC0000000000000004104002C22
:100F300000D03FC000000000000000820800203008
:100F4000107FE00000000000000082080020781000
:100F50007FE00000000000000041040020FC107F42
:100F6000E00000000000000020820030FC301F8004
:100F7000000000000000000000003800700F0000BA
:100F8000000000000000FFFFC03FFFF0060000006F
:100F90000000000000FFFFC0000000000000000093
:100FA000000000000000003FFFF000000000000013
:100FB0000000000000003800700000000000000089
:100FC000000000000031863000000000000000003A
:100FD0000000000023871000000000000000000057
:100FE00000000027879000000000000000000000C3
:100FF00000002F87D000000000000000000000006B
:10100000002F03D03FC0000000000000002082003D
:101010002030107FE00000000000000010410020A0
:1010200078107FE0000000000000001041002078F0
:10103000107FE0000000000000002082002030103F
:101040003FC0000000000000004104002F03D03F1B
:10105000C0000000000000008208002F87D07FE061
:10106000000000000000008208002787907FE00059
:101070000000000000004104002387107FE0000012
:1010800000000000002082003186301F8000000038
:10109000000000000000003800700F000000000099
:1010A000000000FFFFC03FFFF0060000000000004E
:1010B0000000FFFFC000000020746F6F206C6F6E97
:1010C0006720657874727573696F6E2070726576CB
:1010D000656E7465640A0020636F6C6420657874C3
:1010E000727573696F6E2070726576656E74656473
:1010F0000A0024F4D43050C38E20C2A24017828B41
:101100007011127A910D816CD90AA861E108C75853
:101110006607615143061E4B5D05C145A7041A4190
:101120001104093D9803713931034036DB02653300
:101130009102D4305402802E1D02632CEE01752AD8
:10114000C501B028A001102781018F2564012B243F
:101150004B01E0223401AC211F018D200D01801FC5
:10116000FC00841EED00971DDF00B81CD200E61BBA
:10117000C600201BBC00641AB200B219A8000A19EC
:10118000A0006A189900D117910040178B00B5167E
:10119000840031167E00B31579003A157300C71428
:1011A0006F0058146A00EE1366008813630025135D
:1011B0005E00C7125B006C12570015125400C1117B
:1011C000510070114F0021114B00D61049008D10B5
:1011D00047004610440002104200C00F4000800F3C
:1011E0003E00420F3C00060F3B00CB0E3800930E32
:1011F00037005C0E3500270E3400F30D3200C10DB0
:101200003100900D3000600D2E00320D2D00050DC7
:101210002C00D90C2B00AE0C2900850C29005C0C8D
:101220002700350C27000E0C2600E80B2400C40B09
:101230002400A00B23007D0B23005A0B2100390B47
:101240002100180B2000F80A1F00D90A1E00BB0A53
:101250001E009D0A1D00800A1D00630A1C00470A2B
:101260001B002C0A1B00110A1A00F7091A00DD09DD
:101270001900C4091900AB091900920917007B096C
:101280001800630917004C091600360916002009DA
:1012900016000A091500F5081500E0081400CC082E
:1012A0001400B8081400A4081400900813007D0866
:1012B00012006B0813005808120046081200340888
:1012C0001100230811001208110001081100F00795
:1012D0001000E0071000D0071000C0071000B00792
:1012E0000F00A107100091070E0083070F0074077D
:1012F0000F0065070E0057070E0049070E003B0759
:101300000D002E070E0020070D0013070D00060725
:101310000D00F9060C00ED060D00E0060C00D406E9
:101320000C00C8060C00BC060C00B0060C00A4069D
:101330000B0099060C008D060B0082060B00770649
:101340000B006C060B0061060A0057060B004C06EA
:101350000A0042060A0038060A002E060A00240681
:101360000A001A060A001006090007060A00FD0511
:101370000900F4050900EB050900E2050900D9059B
:101380000900D0050900C7050900BE050900B5051B
:101390000800AD050800A50509009C050800940596
:1013A00008008C050800840508007C050800740509
:1013B00008006C050700650508005D050700560577
:1013C00008004E05070047050700400508003805DE
:1013D0000700310507002A050700230507001C0543
:1013E0000600160507000F050700080506000205A0
:1013F0000700FB040600F5040700EE040600E804FD
:101400000600E2040700DB040600D5040600CF0452
:101410000600C9040600C3040600BD040600B704A4
:101420000600B1040500AC040600A6040600A004F2
:1014300005009B04060095040500900406008A043C
:10144000050085040500800406007A040500750483
:101450000500700405006B040500660405006104C6
:1014600005005C04050057040500520405004D0406
:10147000050048040500430405003E0404003A0446
:10148000050035040500300404002C040500270481
:101490000400230405001E0404001A0404001604BA
:1014A0000500110404000D040400090405000404EF
:1014B000040000040400FC030400F8030400F40327
:1014C0000400F0030400EC030400E8030400E40358
:1014D0000400E0030400DC030400D8030400D40388
:1014E0000400D0030400CC030400C8030300C503B8
:1014F000030024F404D9201BC40C5C0E9804C40916
:101500005F0265077101F405F900FB04B3004804AC
:101510008700C10369005803550003034500BE025C
:101520003A008402310053022A00290225000402F5
:101530002000E4011C00C8011900AF011700980148
:1015400014008401130071011000610110005101A9
:101550000E0043010D0036010B002B010B00200192
:101560000B00150109000C01090003010800FB0034
:101570000800F3000800EB000700E4000600DE00AE
:101580000600D8000600D2000600CC000500C70007
:101590000500C2000500BD000400B9000400B5004C
:1015A0000400B1000400AD000400A9000400A5007F
:1015B0000300A20003009F0004009B0003009800AA
:1015C00003009500020093000300900003008D00CB
:1015D00002008B00030088000200860002008400E5
:1015E0000300810002007F0002007D0002007B00FA
:1015F000020079000200770001007600020074000A
:10160000020072000100710002006F0002006D0014
:1016100001006C0002006A0001006900020067001E
:101620000100660001006500010064000200620024
:10163000010061000100600001005F0002005D0028
:1016400001005C0001005B0001005A00010059002C
:10165000010058000100570001005600010055002C
:10166000010054000100530000005300010052002B
:10167000010051000100500001004F0001004E0028
:1016800000004E0001004D0001004C0001004B0025
:1016900000004B0001004A00010049000100480021
:1016A000000048000100470001004600000046001D
:1016B0000100450000004500010044000100430016
:1016C0000000430001004200000042000100410010
:1016D000000041000100400001003F0000003F0009
:1016E00001003E0000003E0001003D0000003D0002
:1016F00001003C0000003C0000003C0001003B00F9
:1017000000003B0001003A0000003A0001003900EF
:1017100000003900010038000000380000003800E7
:1017200001003700000037000100360000003600DD
:1017300000003600010035000000350000003500D3
:1017400001003400000034000000340001003300C8
:1017500000003300000033000100320000003200BE
:1017600000003200010031000000310000003100B3
:1017700001003000000030000000300001002F00A8
:1017800000002F0000002F0000002F0001002E009D
:1017900000002E0000002E0001002D0000002D0092
:1017A00000002D0000002D0001002C0000002C0086
:1017B00000002C0000002C0001002B0000002B007A
:1017C00000002B0000002B0001002A0000002A006E
:1017D00000002A0000002A00010029000000290062
:1017E0000000290000002900000029000100280055
:1017F0000000280000002800000028000000280049
:10180000010027000000270000002700000027003B
:10181000000027000100260000002600000026002E
:101820000000260000002600010025000000250021
:101830000000250000002500000025000000250014
:101840000100240000002400000024000000240007
:1018500000002400010023000000230000002300FA
:1018600000002300000023000000230000002300EC
:1018700001002200000022000000220000002200DF
:1018800000002200000022000100210000002100D1
:1018900000002100000021000000210000002100C4
:1018A00000002100010020000000200000002000B6
:1018B00000002000000020000000200000002000A8
:1018C0000000200001001F0000001F0000001F009A
:1018D00000001F0000001F0000001F0000001F008C
:1018E00001001E0000001E0000001E0000001E007F
:1018F0000000C23100001C260000F4190000D80FBF
:101900000000EB080000C004000075020000400168
:101910000000436172642072656D6F7665640043F8
:1019200061726420696E73657274656400000609F3
:1019300000FE06018902FE20FFFE07FE06FE0000F3
:1019400000060007010606060200808080800080F5
:10195000030303060103A0A0A00507070600FF502C
:1019600050F850F850500509090600FE2070A8A054
:101970007028A870200608080600FF40A84810201C
:101980004854080507070600FF609090609890682B
:101990000103030602038080800207070602FF405E
:1019A0008080808080400207070602FF8040404020
:1019B0004040800505050600008850F85088050560
:1019C000050600002020F820200204040602FEC0C4
:1019D000404080050101060002F8020202060200F2
:1019E000C0C00406060601001010204080800406D6
:1019F00006060100609090909060030606060100C4
:101A000040C0404040E004060606010060901020FF
:101A100040F0040606060100F020601010E0050604
:101A20000606000010305090F8100406060601006B
:101A3000F080E01010E00406060601006080E090EF
:101A40009060040606060100F010102040400406D5
:101A50000606010060906090906004060606010092
:101A6000609090701060020505060200C0C000C0C2
:101A7000C00207070602FEC0C000C0404080050546
:101A8000050600001860806018050303060001F8D1
:101A900000F8050505060000C0300830C00407073F
:101AA0000601006090106040004005060606000038
:101AB0007090A8B08070050606060000205088F8D7
:101AC0008888050606060000F088F08888F004067D
:101AD0000606010060908080906004060606010002
:101AE000E090909090E0040606060100F080E0800F
:101AF00080F0040606060100F080E0808080040685
:101B000006060100609080B09060040606060100A1
:101B10009090F0909090030606060100E04040404F
:101B200040E005060606000038101010906004061C
:101B30000606010090A0C0A09090040606060100D1
:101B40008080808080F005060606000088D8A8A85E
:101B5000888804060606010090D0B0909090050693
:101B60000606000070888888887004060606010052
:101B7000E09090E080800407070601FF609090D01D
:101B8000B06010040606060100E09090E09090041A
:101B900006060601006090402090600506060600DB
:101BA00000F82020202020040606060100909090D6
:101BB000909060040606060100909090F060600529
:101BC00006060600008888A8A8D88805060606002C
:101BD000008850202050880506060600008888509E
:101BE000202020040606060100F010204080F003AB
:101BF0000606060100E080808080E00406060601FB
:101C000000808040201010030606060100E020201E
:101C10002020E0050303060003205088050101068B
:101C200000FEF802020206020480400404040601D9
:101C300000709090700406060601008080E090908D
:101C4000E0040404060100708080700406060601AA
:101C50000010107090907004040406010060B0C081
:101C600070040606060100205040E04040040606CD
:101C70000601FE6090907010600406060601008068
:101C800080E09090900306060601004000C04040AE
:101C9000E00308080601FE200060202020A0400488
:101CA00006060601008080A0C0A09003060606017B
:101CB00000C040404040E0050404060000D0A8A851
:101CC00088040404060100E09090900404040601D6
:101CD00000609090600406060601FEE09090E080AF
:101CE000800406060601FE70909070101004040433
:101CF000060100A0D0808004040406010070C030FA
:101D0000E00406060601004040E0405020040404C0
:101D10000601009090907004040406010090906009
:101D20006005040406000088A8A850040404060105
:101D300000906060900406060601FE9090907090FE
:101D400060040404060100F02040F00307070601C8
:101D500000204040804040200107070602FF8080AD
:101D6000808080808003070706010080404020407B
:101D7000408004020206010350A0FFFFFFFFFFFFA7
:101D8000FFFFFFFFFFFFFFFFFFFFFFFFFFFFFFFF63
:101D9000FFFFFFFFFFFFFFFFFFFFFF000000060048
:101DA0000701060606020080008080808004060687
:101DB0000601FF2070A0A070200507070600FF3075
:101DC0004840F04040F8050505060000A85088503E
:101DD000A80506060600008850F820F8200107072D
:101DE0000602FF808080008080800407070601FFD4
:101DF000708060906010E0030101060105A00607F5
:101E000007060000788494A49484780305050601ED
:101E10000160A06000E00505050600002850A05004
:101E200028040303060100F010100401010601025A
:101E3000F00607070600007884B4A4A4847804019F
:101E400001060105F0040303060102609060050726
:101E5000070600FF2020F8202000F80305050601F2
:101E60000140A02040E0030505060101C0204020FC
:101E7000C002020206020440800405050601FF902C
:101E800090B0D08005060606000078E8E8682828AB
:101E9000010101060202800202020602FE408003E6
:101EA000050506010140C04040E0030505060101AB
:101EB00040A04000E0050505060000A0502850A005
:101EC0000508080600FF40C0405070307810050833
:101ED000080600FF40C04050680810380508080692
:101EE00000FFC0204030F0307810040707060100E2
:101EF0002000206080906005070706000040202039
:101F00005070888805070706000010202050708850
:101F100088050707060000205020507088880507B4
:101F20000706000028502050708888050707060023
:101F300000500020507088880507070600002050D8
:101F4000205070888805060606000078A0F0A0A042
:101F5000B80408080601FE6090808090602040046C
:101F600007070601004020F080E080F00407070624
:101F700001002040F080E080F00407070601002007
:101F800050F080E080F00407070601005000F08068
:101F9000E080F00307070601008040E0404040E099
:101FA0000307070601002040E0404040E003070728
:101FB00006010040A0E0404040E0030707060100A2
:101FC000A000E0404040E00506060600007048E83A
:101FD00048487004070706010050A090D0B09090C8
:101FE00004070706010040206090909060040707F6
:101FF00006010020406090909060040707060100F1
:102000002050609090906004070706010050A06087
:102010009090906004070706010050006090909037
:102020006005050506000088502050880408080651
:1020300001FF1070B0B0D0D0E080040707060100A7
:102040004020909090906004070706010020409087
:1020500090909060040707060100205090909090A7
:1020600060040707060100500090909090600507FB
:1020700007060000102088502020200406060601D4
:102080000080E09090E0800406060601006090A0C9
:10209000A090A004070706010040200070909070F7
:1020A00004070706010020400070909070040707A5
:1020B0000601002050007090907004070706010090
:1020C00050A0007090907004060606010050007049
:1020D00090907004070706010020502070909070C7
:1020E00005040406000070A8B0780406060601FE88
:1020F00070808070204004070706010040200060C7
:10210000B0C07004070706010020400060B0C07036
:1021100004070706010020500060B0C070040606E6
:10212000060100500060B0C0700307070601008080
:102130004000C04040E0030707060100204000C007
:102140004040E003070706010040A000C04040E017
:10215000030606060100A000C04040E00407070691
:102160000100306010709090600407070601005075
:10217000A000E09090900407070601004020006056
:102180009090600407070601002040006090906076
:1021900004070706010020500060909060040707C4
:1021A00006010050A0006090906004060606010041
:1021B0005000609090600505050600002000F800C2
:1021C0002004040406010070B0D0E00407070601F3
:1021D0000040200090909070040707060100204006
:1021E0000090909070040707060100205000909026
:1021F000907004060606010050009090907004094B
:10220000090601FE2040009090907090600408083C
:102210000601FE8080E09090E080800408080601BE
:10222000FE50009090907090604E6F204368656300
:102230006B73756D2077697468206C696E65206EAC
:10224000756D6265722C204C617374204C696E65EB
:102250003A200053544F505045442E20005072698C
:102260006E7465722073746F707065642064756538
:1022700020746F206572726F72732E204669782009
:10228000746865206572726F7220616E6420757368
:1022900065204D39393920746F207265737461720D
:1022A000742E202854656D70657261747572652096
:1022B00069732072657365742E2053657420697488
:1022C0002061667465722072657374617274696EE0
:1022D00067290A004E6F20436865636B73756D2034
:1022E00077697468206C696E65206E756D626572C1
:1022F0002C204C617374204C696E653A2000636831
:1023000065636B73756D206D69736D617463682CA3
:10231000204C617374204C696E653A20004C696EE4
:1023200065204E756D626572206973206E6F742032
:102330004C617374204C696E65204E756D626572D8
:102340002B312C204C617374204C696E653A20004F
:102350004D313130004D333100534420726561649A
:10236000206572726F720A00446F6E652070726928
:102370006E74696E672066696C650A0020466C6F32
:10238000773A200020643A0020693A0020703A0031
:1023900043290A0061626C656420286D696E2074AF
:1023A000656D702000436F6C64206578747275648D
:1023B00065732061726520004B64200023646566AC
:1023C000696E652044454641554C545F004B692079
:1023D0000023646566696E652044454641554C544A
:1023E0005F004B70200023646566696E652044457C
:1023F0004641554C545F00504944204175746F74F8
:10240000756E652066696E69736865642120507514
:102410007420746865206C617374204B702C204BA1
:102420006920616E64204B6420636F6E7374616E0B
:1024300074732066726F6D2062656C6F7720696EB1
:10244000746F20436F6E66696775726174696F6E31
:102450002E680A00504944204175746F74756E658A
:10246000206661696C6564212074696D656F75749F
:102470000A00453120544845524D414C2052554E9A
:10248000415741590042454420544845524D414C22
:102490002052554E4157415900546865726D616C28
:1024A0002052756E6177617900453120486561740D
:1024B000696E67206661696C6564004265642068C6
:1024C000656174696E67206661696C656400486562
:1024D0006174696E67206661696C65640050494487
:1024E000204175746F74756E65206661696C6564F2
:1024F000212054656D706572617475726520746F0A
:102500006F20686967680A00204B643A2000204BFE
:10251000693A2000204B703A20000A20436C617316
:1025200073696320504944200A002054753A200002
:10253000204B753A2000206D61783A2000206D69AB
:102540006E3A200020643A200020626961733A20CC
:1025500000504944204175746F74756E6520666142
:10256000696C6564212042616420657874727564C9
:102570006572206E756D6265720A00504944204193
:1025800075746F74756E652073746172740A004F90
:10259000666673657473206170706C69656400456C
:1025A00072723A20546F6F206661722100546F6F0F
:1025B000206661722066726F6D2072656665726555
:1025C0006E636520706F696E740A00454550524F06
:1025D0004D204F4B0A003A200050726F6265205A1E
:1025E000204F6666736574003F5A206F7574206FC4
:1025F000662072616E676520282D3220746F203549
:10260000290A00496E736572742066696C616D6594
:102610006E7420616E6420707265737320627574CD
:10262000746F6E20286F72204D313038290A0050A7
:102630007265737320627574746F6E20286F7220D8
:102640004D3130382920746F2068656174206E6FB9
:102650007A7A6C650A00496E736572742066696CDB
:10266000616D656E7420616E642070726573732095
:10267000627574746F6E20286F72204D3130382966
:102680000A004E6F2063617365206C696768740A85
:10269000001000C90210012C014001220170011834
:1026A00001B0010E01F00104015002FA00B002F085
:1026B000003003E600D003DC009004D2007005C8AF
:1026C00000A006BE000008B400B009AA00D00BA00C
:1026D00000600E960060118C0000158200201978B1
:1026E00000C01D6E00A0226400B0275A00902C503C
:1026F0000000314600E0343C0010383200903A28A7
:1027000000603C1E00A03D1400803E0A00203F00F7
:10271000006265640A002C2073797374656D207300
:10272000746F7070656421204865617465725F49DB
:10273000443A20004265642068656174696E6720D0
:102740006661696C65640048656174696E672066DE
:1027500061696C65640045312048656174696E6724
:10276000206661696C65640048656174696E672004
:102770006661696C6564004B494C4C45442E2000F1
:102780001000AD0330016A0150022B0170030A01F1
:102790009004F500B005E500D006D800F007CE00A3
:1027A0001009C500300ABE00500BB700700CB10014
:1027B000900DAB00B00EA600D00FA200F0109D004F
:1027C00010129900301395005014920070158E006D
:1027D00090168B00B0178700D0188400F019810084
:1027E000101B7E00301C7B00501D7900701E76008F
:1027F000901F7300B0207000D0216E00F0226B009B
:10280000102469003025660050266300702761009F
:1028100090285E00B0295C00D02A5900F02B5600A9
:10282000102D5400302E5100502F4E0070304B00B0
:1028300090314800B0324500D0334200F0343E00C1
:1028400010363B00303737005038330070392E00D7
:10285000903A2900B03B2300D03C1B00F03D110012
:10286000103F0100F03F00004531204572723A20D0
:102870004D415854454D50004572723A204D4158D3
:1028800054454D5020424544004D415854454D500B
:10289000207472696767657265640045312045720E
:1028A000723A204D494E54454D50004572723A20BF
:1028B0004D494E54454D5020424544004D494E54DB
:1028C000454D5020747269676765726564004D38C4
:1028D0003420582059205A204500202F0020424003
:1028E0003A0020403A000000200023002600290082
:1028F0002C002F0032000001000003010601090135
:10290000024D6963726F737465707320756E6176C2
:1029100061696C61626C650A0045313A200045309E
:102920003A20005A3A2000593A2000583A20004DE7
:1029300053312C4D53322050696E730A0045727228
:102940006F722077726974696E6720746F204545D5
:1029500050524F4D210A001FFFFFFFFFFFFF600095
:1029600000000001FF400000000000FF80000000A8
:1029700000007F83CF00000C303F87FF80000C30C9
:102980001F867980000C000F8C30C7838C30E78C59
:1029900030CFC7CC31F38C30DCECEC33B98C30D891
:1029A0006C6C33198C30D06C0C33198C30D86C0CA7
:1029B00033198C30DC6C0E3B198C30CF7C079F199F
:1029C0008C30C77C038F19400000000000026000BB
:1029D00000000000061FFFFFFFFFFFF82020506CE3
:1029E000616E6E6572427566666572427974657372
:1029F0003A20002046726565204D656D6F72793A08
:102A00002000436F6D70696C65643A204A616E20E6
:102A1000313020323031390A00207C204175746811
:102A20006F723A2028416C657068204F626A656356
:102A3000747320496E632E2C204C756C7A426F742F
:102A400020476974205265706F7369746F727929B9
:102A50000A004A616E203130203230313931333A48
:102A600035303A313500204C617374205570646103
:102A70007465643A2000312E312E390A004D61729E
:102A80006C696E0020536F667477617265205265C1
:102A90007365740A00205761746368646F6720521D
:102AA000657365740A002042726F776E206F7574CB
:102AB0002052657365740A002045787465726E61F2
:102AC0006C2052657365740A00506F77657255709B
:102AD0000A0073746172740A006175746F25692E3F
:102AE00067006572726F722077726974696E672011
:102AF000746F2066696C650A00456E6473746F704C
:102B00007320256320256320256320256300205042
:102B10003A00205A3A0020593A0020583A00656E8F
:102B20006473746F7073206869743A2000446F6E28
:102B30006520736176696E672066696C652E0A0090
:102B40004D3239004739310A4730205A3135204655
:102B50003630300A4739300A473020583137302074
:102B6000593239302046333030300A4D3131372038
:102B70005072696E742061626F727465642E0050C9
:102B800072696E7465722053746174730046697261
:102B90006D776172652056657273696F6E004D6165
:102BA000696E000A003B20454550524F4D20496E4A
:102BB0006465783A20005570646174696E67207AA4
:102BC0006F666673657420696E20454550524F4D9F
:102BD0003A20000E000E000E000E000E000E000E39
:102BE000000E007FC03F801F000E00040004000E96
:102BF000001F003F807FC00E000E000E000E000E72
:102C0000000E000E000E0003F8000FFE001E0F0065
:102C1000380700380380700380700FE07007C070C1
:102C200003807001007000003800003807001E0F9C
:102C3000000FFE0003F80000FE0003FF800783C0C2
:102C40000E01C00E00E01C00E07F00E03E00E01C32
:102C500000E00800E00000E00001C00E01C00F0726
:102C60008007FF0001FC00FFFFFF7F80FFC0FFC067
:102C7000FFC07F807F80FFC0FFC0FFC03F001E00FD
:102C80000C0050726F6265205A204F66667365743F
:102C90000050726F6265205A204F6666736574003B
:102CA000466C6F7700466C6F770046616E207370DC
:102CB00065656420310046616E207370656564202F
:102CC000310042656400426564004E6F7A7A6C653B
:102CD000004E6F7A7A6C65005370656564005370BE
:102CE000656564004D61696E004D6F766520580022
:102CF0004D6F76652059004D6F7665205A004578F6
:102D000074727564657220004D6F766520302E31C7
:102D10006D6D004D6F766520316D6D004D6F766580
:102D20002031306D6D004D6F7665206178697300DC
:102D3000457874727564657220004D6F7665205A0F
:102D4000004D6F76652059004D6F7665205800451F
:102D50007874727564657220004175746F20686FB5
:102D60006D6500473238004D6F7665205A004D6F13
:102D700076652059004D6F76652058004D6F766559
:102D80006D656E74002569730025696D2025697372
:102D9000002569682025696D20256973002569640F
:102DA000202569682025696D2025697300256979CA
:102DB00020256964202569682025696D20256973AF
:102DC00000486F6D696E67206661696C656400011B
:102DD000050800FF060121023520FFFF07FF06FF5F
:102DE000090050221656808080800080153353A041
:102DF000A0A00257575050F850F850500257572093
:102E000070A07028702013355580A040A020024784
:102E10005740A0A040A0A0502513538080801226C8
:102E2000564080808080401226568040404040803E
:102E30000245559060F060900255552020F8202002
:102E4000113353604080044151F011335340E0404E
:102E500002465610102040808012365640A0A0A096
:102E6000A04012365640C0404040E00246566090B6
:102E7000106080F0024656F02060109060024656C6
:102E80002060A0F02020024656F080E01090600202
:102E900046566080E0909060024656F01020204038
:102EA0004002465660906090906002465660909056
:102EB000701060122555C0C000C0C0113656606049
:102EC00000604080123656204080804020034353EB
:102ED000F000F012365680402020408012365640D6
:102EE000A020400040015858304898A8A890403091
:102EF000024656609090F09090024656E090E09026
:102F000090E0024656609080809060024656E090C5
:102F1000909090E0024656F080E08080F0024656A5
:102F2000F080E0808080024656609080B090600221
:102F300046569090F0909090123656E040404040B7
:102F4000E002465670202020A04002465690A0C0C5
:102F5000A0A0900246568080808080F00246569065
:102F6000F0F090909002465690D0F0B0B0900246AB
:102F700056609090909060024656E09090E080807D
:102F8000014757609090D0B06010024656E0909094
:102F9000E09090024656609040209060123656E0D5
:102FA00040404040400246569090909090600246CB
:102FB00056909090906060024656909090F0F090FD
:102FC0000246569090606090900256568888502035
:102FD0002020024656F010204080F0123656E08045
:102FE000808080E0024656808040201010123656C5
:102FF000E020202020E016325240A0014151F0167E
:103000002252804002445470909070024656808054
:10301000E09090E0123454608080600246561010B8
:103020007090907002445460B0C0600246562050C8
:1030300040E0404001455560907010600246568067
:1030400080E09090901236564000C04040E011372A
:10305000572000202020A040024656808090E0901B
:1030600090123656C040404040E0025454D0A8A8C8
:10307000A8024454E0909090024454609090600103
:103080004555E090E0808001455570907010100229
:103090004454A0D0808012345460C020C0024656F0
:1030A0004040E040502002445490909070123454BC
:1030B000A0A0A04002545488A8A850024454906094
:1030C00060900145559090709060024454F020400B
:1030D000F0024757304020C02040302216568080F2
:1030E00080808080024757C02040304020C0064288
:1030F0005250A0FFFFFFFFFFFFFFFFFFFFFFFFFF9B
:10310000FFFFFFFFFFFFFFFFFFFFFFFFFFFFFFFFCF
:10311000FFFFFFFF0900502216568000808080804C
:103120000146562070A0A070200246562050E04074
:1031300050A002555588705070880256568850F835
:1031400020F8202217578080800080808002475717
:103150007080E0907010E0173151A002565670A8B0
:10316000C8C8A87014355560A06000E003435350F0
:10317000A050123353E02020143151E00256567013
:10318000E8D8E8D870173151E015335340A0401209
:10319000355540E04000E014355540A02040E01493
:1031A0003555C020C020C0162252408001455590A0
:1031B0009090E08002565678E8E86828282411515B
:1031C00080112252408014355540C04040E01435F3
:1031D0005540A04000E0034353A050A00247578051
:1031E0008080A060F0200247578080A0D01020701F
:1031F00002475780408060A0F020123656400040C1
:1032000080A04002475740206090F09090024757BE
:1032100020406090F0909002475760906090F0904E
:103220009002475750A06090F0909002475790004E
:103230006090F0909002475760906090F0909002FC
:10324000465670A0A0F0A0B00147576090808090D3
:1032500060400247574020F080E080F0024757204E
:1032600040F080E080F00247576090F080E080F00E
:103270000247579000F080E080F01237578040E01E
:10328000404040E01237572040E0404040E01237D5
:103290005740A0E0404040E0123757A000E04040D7
:1032A00040E00256567048E848487002475750A020
:1032B00090D0B0909002475740206090909060026C
:1032C0004757204060909090600247576090609010
:1032D00090906002475750A06090909060024757CE
:1032E00090006090909060123353A040A002465628
:1032F00070B0B0D0D0E002475740209090909060DE
:1033000002475720409090909060024757609090FD
:103310009090906002475790009090909060025774
:10332000571020885020202002465680E09090E0E0
:10333000800246566090A0A090A00247574020000F
:103340007090907002475720400070909070024734
:10335000572050007090907002475750A000709016
:1033600090700246565000709090700247576090DF
:103370006070909070025454F068B07811355560C8
:103380008080604002475740200060B0C060024724
:103390005720400060B0C06002475760900060B0A6
:1033A000C060024656500060B0C06012375780407F
:1033B00000C04040E0123757204000C04040E012BB
:1033C000375740A000C04040E0123656A000C04031
:1033D00040E0024757A040A010709060024757504D
:1033E000A000E090909002475740200060909060CD
:1033F000024757204000609090600247576090005D
:103400006090906002475750A00060909060024624
:10341000569000609090601235554000E0004002E8
:10342000445470B0D0E00247574020009090907014
:1034300002475720400090909070024757609000DC
:10344000909090700246569000909090700148586D
:1034500020400090907090600147578080E090E09D
:1034600080800147579000909070906001050700A0
:10347000FE0500FB01F220FFFE05FE05FE020040F6
:103480000215258080800080053242A0A00255658B
:1034900050F850F8500146562070C030E0200255D8
:1034A000659010204048025565608068906805125C
:1034B0002280800225354080808040022535804072
:1034C000404080043343A040A003334340E0400128
:1034D00022324080043141E002112180025565080A
:1034E000102040800245556090909060022535C0C4
:1034F00040404040024555E0106080F0024555E0F4
:10350000106010E00245552060A0F020024555F003
:1035100080E010E00245556080E09060024555F083
:103520001020404002455560906090600245556013
:1035300090701060031323800080021424800080A8
:10354000800235452040804020033343E000E00204
:1035500035458040204080024555E0106000400223
:1035600055657088B8A870024555609090F090023B
:103570004555E090E090E002354560808080600233
:103580004555E0909090E0023545E080E080E00213
:103590003545E080E080800245557080B090700233
:1035A00045559090F09090023545E0404040E00253
:1035B0004555301010906002455590A0C0A0900273
:1035C000354580808080E002556588D8A8888802CB
:1035D000455590D0B0909002455560909090600213
:1035E0004555E09090E080014656609090906010C4
:1035F000024555E09090E09002455570806010E0E3
:10360000023545E040404040024555909090906022
:103610000245559090A0A04002556588A8A8A850E2
:1036200002455590906090900245559090701060C2
:10363000023545E0204080E0022535C0808080C012
:103640000255658040201008022535C0404040C02A
:1036500005324240A0024151F0052232804002442E
:10366000547090907002455580E09090E002344490
:1036700060808060024555107090907002445460E4
:10368000B0C0600235452040E04040004656709092
:103690009070106002455580E09090900215258052
:1036A0000080808000273740004040404080024535
:1036B000558090A0E0900215258080808080025483
:1036C00064F0A8A8A8024454E0909090024454608A
:1036D000909060004656E09090E0808000465670E2
:1036E0009090701010023444A0C080800244547046
:1036F000C030E002354540E0404020024454909004
:1037000090700244549090A040025464A8A8505075
:10371000023444A04040A000465690909070106043
:10372000024454F02040F002354560408040600281
:1037300015258080808080023545C0402040C0052E
:10374000425250A0FFFFFFFFFFFFFFFFFFFFFFFF01
:10375000FFFFFFFFFFFFFFFFFFFFFFFFFFFFFFFF79
:10376000FFFFFFFFFF020040FFFFFFFFFFFFFFFF24
:10377000FFFFFFFFFFFFFFFFFFFFFFFFFFFFFFFF59
:10378000FFFFFFFFFFFFFFFFFFFFFFFFFFFFFFFF49
:10379000FFFFFFFFFFFFFFFFFFFFFFFFFFFFFFFF39
:1037A000FFFFFFFFFFFFFFFFFFFFFFFFFFFFFFFF29
:1037B000FFFFFFFFFFFFFFFFFFFFFFFFFFFFFFFF19
:1037C000FFFFFFFFFFFFFF01060D00FE090166027C
:1037D000D620FFFE0BFE0AFE0D00602219698080D4
:1037E00080808080800080183363A0A0A00357678A
:1037F0005050F850F850500259692078A0A0702815
:1038000028F02002596948A85010204050A8900282
:10381000586840A0A040A0989068281363808080DA
:10382000113B6B2040408080808080404020113BD5
:103830006B8040402020202020404080065565209D
:10384000A870A8200455652020F82020113363605B
:103850004080065161F811336340E0400259690825
:1038600008101020404080800259692050888888C4
:10387000888850200259692060A02020202020F84C
:103880000259697088880810204080F8025969F848
:1038900008102070080888700259691010305050C4
:1038A00090F81010025969F88080B0C80808887034
:1038B00002596970888080F088888870025969F898
:1038C0000810102020404040025969708888887094
:1038D0008888887002596970888888780808887094
:1038E00011386840E040000040E04011386840E096
:1038F000400000604080025969081020408040204C
:103900001008045464F80000F8025969804020103F
:103910000810204080025969708888081020200013
:103920002002596970888898A8A8B08078025969DF
:103930002050888888F8888888025969F048484863
:1039400070484848F002596970888080808080887B
:1039500070025969F048484848484848F002596997
:10396000F8808080F0808080F8025969F88080803B
:10397000F080808080025969708880808098888873
:103980007002596988888888F88888888812396917
:10399000E040404040404040E0025969381010107B
:1039A0001010109060025969888890A0C0A090887B
:1039B000880259698080808080808080F8025969FF
:1039C0008888D8A8A88888888802596988C8C8A81B
:1039D000A898988888025969708888888888888813
:1039E00070025969F0888888F080808080015A6A66
:1039F00070888888888888A87008025969F0888843
:103A000088F0A090888802596970888080700808C2
:103A10008870025969F82020202020202020025997
:103A20006988888888888888887002596988888821
:103A300088505050202002596988888888A8A8A8F2
:103A4000A8500259698888505020505088880259DF
:103A500069888850502020202020025969F80810D9
:103A60001020404080F8113B6BE080808080808097
:103A7000808080E002596980804040201010080852
:103A8000113B6BE0202020202020202020E0085344
:103A900063205088015161F82A22628040025666F4
:103AA000700878889868025969808080F0888888D2
:103AB00088F002566670888080887002596908080C
:103AC000087888888888780256667088F8808870B8
:103AD00002596930484040F040404040005868700A
:103AE00088888878088870025969808080B0C88882
:103AF0008888881238684000C040404040E0004A52
:103B00006A10003010101010909060025969808087
:103B10008090A0C0A09088123969C04040404040C9
:103B20004040E0025666D0A8A8A8A888025666B011
:103B3000C888888888025666708888888870005887
:103B400068F0888888F08080800058687888888845
:103B500078080808025666B0C880808080025666E1
:103B60007088601088700258684040F040404048BB
:103B700030025666888888889868025666888888E1
:103B80005050200256668888A8A8A8500256668819
:103B90005020205088005868888888986808887065
:103BA000025666F810204080F8015B6B1820202038
:103BB00020C02020202018221969808080808080E9
:103BC000808080015B6BC0202020201820202020D6
:103BD000C008536348A890FFFFFFFFFFFFFFFFFFF0
:103BE000FFFFFFFFFFFFFFFFFFFFFFFFFFFFFFFFE5
:103BF000FFFFFFFFFFFFFFFF0D006022196980003C
:103C0000808080808080800358682070A8A0A0A851
:103C1000702002596930484040E0404048B00356A7
:103C20006688705050708802596988885050F82012
:103C3000F820202219698080808000808080801296
:103C40004A6A609080609090601090601A3262A022
:103C5000A00359697088A8D8C8D8A8887004576785
:103C6000700878887800F80356662850A0A050287D
:103C7000045363F80808163161E00359697088E855
:103C8000D8D8E8D888700A5161F8174464609090D9
:103C9000600357672020F8202000F807356540A012
:103CA0002040E007356540A04020C02A22624080C5
:103CB0000058688888888898E8808002596978E880
:103CC000E8E8E868282828262161C0202262408090
:103CD00007356540C04040E00457677088888870A9
:103CE00000F8035666A050282850A0025A6A40C027
:103CF0004040E00818283808025A6A40C04040E0B6
:103D00001028081038025A6A40A04020A0481828FD
:103D10003808025969200020204080888870025AA3
:103D20006A40200020508888F88888025A6A10204B
:103D30000020508888F88888025A6A30480020504D
:103D40008888F88888025A6A28500020508888F8A5
:103D50008888025A6A50500020508888F888880263
:103D60005A6A20502020508888F88888025969585B
:103D7000A0A0A0B0E0A0A0B8005B6B70888080809D
:103D8000808088702040025A6A402000F88080F0CD
:103D90008080F8025A6A102000F88080F08080F855
:103DA000025A6A304800F88080F08080F8025A6A2F
:103DB000505000F88080F08080F8123A6A8040000D
:103DC000E04040404040E0123A6A204000E040407D
:103DD000404040E0124A6A609000E040404040406D
:103DE000E0123A6AA0A000E04040404040E00259A2
:103DF00069F0484848E8484848F0025A6A285000A4
:103E00008888C8A8988888025A6A402000708888E4
:103E100088888870025A6A1020007088888888888C
:103E200070025A6A30480070888888888870025A00
:103E30006A28500070888888888870025A6A5050B2
:103E4000007088888888887003556588502050885D
:103E5000015B6B08709898A8A8A8C8C87080025A1F
:103E60006A40200088888888888870025A6A1020F2
:103E70000088888888888870025A6A304800888854
:103E80008888888870025A6A505000888888888894
:103E90008870025A6A102000888850202020200252
:103EA000596980F0888888F0808080025969609024
:103EB00090A0A0908888B0025969402000700878CE
:103EC00088986802596910200070087888986802FC
:103ED00059693048007008788898680259692850F4
:103EE0000070087888986802596950500070087806
:103EF000889868025A6A3048300070087888986854
:103F0000025666702870A0A850005868708880809B
:103F1000887020400259694020007088F8808870BD
:103F20000259691020007088F88088700259693041
:103F300048007088F8808870025969505000708875
:103F4000F8808870123969804000C040404040E0ED
:103F5000123969204000C040404040E01249696089
:103F60009000C040404040E0123969A0A000C0402D
:103F7000404040E0025A6A5020601070888888886B
:103F800070025969285000B0C88888888802596929
:103F9000402000708888888870025969102000705D
:103FA00088888888700259693048007088888888B5
:103FB0007002596928500070888888887002596991
:103FC000505000708888888870035767202000F858
:103FD000002020015868087098A8A8C8708002596D
:103FE00069402000888888889868025969102000F4
:103FF0008888888898680259693048008888888845
:104000009868025969505000888888889868005BD1
:104010006B1020008888889868088870005A6A8029
:1040200080B0C88888C8B08080005B6B5050008822
:104030008888986808887000000000000000000070
:104040000000000000000000000000000000000070
:10405000000000000000000000000C000000000054
:1040600000000C0000000000000012000000000032
:1040700000002300000000000000210000000000FC
:1040800000004C800000000000005E800000000086
:1040900000009240000000000000A140000000006D
:1040A000000121200000000000027F9000000000BD
:1040B00000020010000000000007FFF800000000F0
:1040C00000040008000000000008000400000000D8
:1040D00000080006000000000010000200000000C0
:1040E00000301E010000000000207F810000000061
:1040F0000041FFE0800000000043FCF08000000071
:1041000000873B7840000000018EDBFC600000006F
:10411000010FEBCC20000000021FEDB610000000E4
:10412000021FDEB6100000000439CD7F0800000039
:104130000436E0FF08000000087EC0BB84000000D9
:10414000187F005D86000000107FC0ED8200000037
:10415000203CC07301000000203B337F01000000C1
:10416000701BE77E03800000C81DEEDE04C0000067
:10417000880FDEDC04400001240FDF3C0920000131
:104180002607DBF8192000027203E7F01390000203
:104190005101FFE02290000489007F80244800093B
:1041A00004801E004824000BFE400000DFF40010D5
:1041B000004000008002001FFFFFFFFFFFFE000025
:1041C00000000000000000000000000000000000EF
:1041D000000000000000001022103C3C0E1F0010E8
:1041E00022100422110400102210082211040010D1
:1041F0002210083C1104001022101022110400109B
:10420000221020221104001E1C1E3C3C0E04000043
:10421000000000000000000000000000000000009E
:10422000000000000000000000000000000000008E
:10423000000000000000000000000000000000007E
:10424000000000000000000000000000000000006E
:10425000000000000000000000000000000000005E
:10426000000000000000000000000000000000004E
:1042700000000000006F70656E206661696C656407
:104280002C2046696C653A200043616E6E6F742085
:104290006F70656E20737562646972200065636873
:1042A0006F3A00453120544845524D414C205255FB
:1042B0004E415741590042454420544845524D41D2
:1042C0004C2052554E4157415900546865726D61FA
:1042D0006C2052756E617761790000002200250024
:1042E00028002B002E0031003400020100000501DF
:1042F00008010B0100002100240027002A002D00E6
:104300003000330001010000040107010A01050526
:104310000505070508080808020202020A0A08083B
:104320000404040401010101010101010303030369
:1043300003030303040707070C0C0C0C0C0C0C0CF8
:104340000202020206060606060606060B0B0B0B09
:104350000B0B0B0B0102102020080810204010202E
:104360004080020102010804020101020408102039
:104370004080804020100804020180040201804037
:1043800020100804020108040201010204081020A0
:1043900040800102040810204080436F6F6C646FFE
:1043A000776E0046616E207370656564203100464B
:1043B000616E20737065656420310042656400425F
:1043C0006564004E6F7A7A6C65004E6F7A7A6C6520
:1043D000004D61696E005654726176206D696E0001
:1043E0005654726176206D696E0056547261762063
:1043F0006D696E00566D696E00566D696E00566D82
:10440000696E00566D6178204500566D61782045D3
:1044100000566D6178204500566D6178205A00562F
:104420006D6178205A00566D6178205A00566D6192
:1044300078205900566D6178205900566D617820BA
:104440005900566D6178205800566D6178205800EB
:10445000566D61782058004D6F74696F6E00416D24
:104460006178204500416D6178204500416D61789B
:10447000205A00416D6178205A00416D61782059C1
:1044800000416D6178205900416D617820580041EC
:104490006D6178205800412D74726176656C004121
:1044A0002D74726176656C00412D72657472616362
:1044B0007400412D726574726163740041636365B9
:1044C0006C00416363656C004D6F74696F6E0056DC
:1044D000652D6A65726B0056652D6A65726B0056B4
:1044E000652D6A65726B00567A2D6A65726B00568F
:1044F0007A2D6A65726B0056792D6A65726B00566B
:10450000792D6A65726B0056792D6A65726B00565B
:10451000782D6A65726B0056782D6A65726B00564D
:10452000782D6A65726B004D6F74696F6E0045453A
:1045300050524F4D206461746173697A65206572D1
:10454000726F722E0A00290A002062797465733B2B
:1045500020637263200053657474696E677320531F
:10456000746F726564202800290A002062797465DE
:10457000733B2063726320002073746F7265642044
:1045800073657474696E6773207265747269657699
:104590006564202800202863616C63756C61746514
:1045A0006429210A0020213D2000454550524F4DED
:1045B00020435243206D69736D61746368202D2020
:1045C0002873746F7265642920002053697A653AF4
:1045D0002000496E6465783A2000204D61726C6954
:1045E0006E3D563535290A0028454550524F4D3D00
:1045F00000454550524F4D2076657273696F6E20AD
:104600006D69736D61746368200050757267652011
:104610006D6F726500456E642066696C616D656ED4
:1046200074206368616E6765000020204E6F7A7A9F
:104630006C653A20006368616E6765006F66207480
:1046400068652066696C616D656E74005761697498
:1046500020666F722073746172740020204E6F7A2E
:104660007A6C653A2000200066696C616D656E7435
:1046700020756E6C6F6164005761697420666F729B
:104680000020204E6F7A7A6C653A20002000506C32
:104690006561736520776169742E2E2E004865610F
:1046A00074696E67206E6F7A7A6C650020204E6F99
:1046B0007A7A6C653A2000200068656174206E6F1C
:1046C0007A7A6C652E00507265737320627574740B
:1046D0006F6E20746F0020204E6F7A7A6C653A20DE
:1046E00000746F20636F6E74696E75652E2E2E00D8
:1046F000616E6420707265737320627574746F6E7E
:1047000000496E736572742066696C616D656E74C4
:104710000020204E6F7A7A6C653A2000200066698E
:104720006C616D656E74206C6F61640057616974B3
:1047300020666F720020204E6F7A7A6C653A2000F6
:10474000200066696C616D656E74207075726765B6
:10475000005761697420666F7200506C6561736503
:1047600020776169742E000020496E76616C69645F
:1047700020657874727564657220000000A0C10025
:1047800000A0C10000000000009643008096430096
:10479000008743486F6D6520257325732573206658
:1047A00069727374002066697273740A005A005942
:1047B000005800486F6D652000486F6D652058599E
:1047C0002066697273740A00486F6D65205859201D
:1047D0006669727374007C3C3E5E2B3D3F2F5B5DCF
:1047E0003B2C2A225C004573746570732F6D6D003D
:1047F0004573746570732F6D6D005A7374657073B3
:104800002F6D6D005A73746570732F6D6D00597341
:10481000746570732F6D6D005973746570732F6DAF
:104820006D005873746570732F6D6D0058737465E7
:1048300070732F6D6D004D6F74696F6E004F6666FB
:10484000004F6E2000456E6473746F702061626F5C
:1048500072740053746570732F6D6D004A65726BCE
:1048600000416363656C65726174696F6E005665C3
:104870006C6F636974790050726F6265205A204FC3
:10488000666673657400416476616E636564205387
:10489000657474696E67730043616E6E6F74206532
:1048A0006E746572207375626469723A2000022E1C
:1048B0002E004D61696E0000457874727564656400
:1048C00020746F74616C3A2000256C642E25696D2C
:1048D00000004C6F6E67657374206A6F62207469A4
:1048E0006D653A200000546F74616C207072696EBF
:1048F000742074696D653A2000436F6D706C657447
:1049000065643A20005072696E7420436F756E744E
:104910003A20004D36303020423020542564004D7E
:1049200037303120542564004D373032203B256428
:10493000004D37303220542564004368616E67654E
:104940002066696C616D656E7400507265686561A2
:104950007420437573746F6D00507265686561747F
:1049600020437573746F6D005072656865617420C3
:10497000414253005072656865617420504C41009B
:104980004D61696E005052494E5420504155534577
:104990004400554E4C4F41442046494C414D454EF4
:1049A00054004C4F41442046494C414D454E540023
:1049B0004D3234004D32332025730053442063615F
:1049C0007264206F6B0A006F70656E526F6F742097
:1049D0006661696C65640A00766F6C756D652E6939
:1049E0006E6974206661696C65640A0053442069CD
:1049F0006E6974206661696C0A0057726974696E29
:104A00006720746F2066696C653A20006F70656E70
:104A1000206661696C65642C2046696C653A2000EB
:104A20006F70656E206661696C65642C2046696CE8
:104A3000653A200046696C652073656C6563746532
:104A4000640A002053697A653A200046696C652043
:104A50006F70656E65643A20002066696C653A2067
:104A600000646F696E67006672657368004E6F77E9
:104A70002000454E4420535542524F5554494E450F
:104A80000A002220706F73002220706172656E74BC
:104A90003A2200535542524F5554494E4520434106
:104AA0004C4C207461726765743A22004B494C4C3F
:104AB00045442E2000747279696E6720746F2063FC
:104AC000616C6C207375622D67636F646520666925
:104AD0006C6573207769746820746F6F206D616EE8
:104AE00079206C6576656C732E204D4158206C657D
:104AF00076656C2069733A004572726F723A0043B2
:104B00006C69636B20746F20726573756D652E2EF2
:104B10002E004E6F206D6F76652E00286E6F20661A
:104B2000696C6529005344207072696E74696E6700
:104B3000206279746520004E6F7420534420707297
:104B4000696E74696E670A0043757272656E7420CF
:104B500066696C653A200046696C652064656C6521
:104B60007465643A0044656C6574696F6E206661B3
:104B7000696C65642C2046696C653A200050726F40
:104B80007465637465642050696E0A00205A3A00A7
:104B900020593A0020436F756E7420583A00204522
:104BA0003A00205A3A0020593A00583A003A004355
:104BB00061703A00205400205200416363656C65C7
:104BC000726174696F6E3A205000205A00205900BB
:104BD000580020204D61783A2000205A00205900CA
:104BE000580020204D696E3A20004F6E20004F661D
:104BF0006600536F667420656E6473746F70733AE9
:104C000020000A0A426564204C6576656C20436F7B
:104C10007272656374696F6E204D61747269783A5F
:104C200000202B000A436F72726563746564204232
:104C30006564204865696768742076732E20426534
:104C40006420546F706F6C6F67793A0A00202B00F4
:104C50000A4265642048656967687420546F706F04
:104C60006772617068793A0A2020202B2D2D2D2043
:104C70004241434B202D2D2B0A2020207C20202038
:104C800020202020202020207C0A204C207C202056
:104C90002020282B29202020207C20520A2045205B
:104CA0007C20202020202020202020207C20490A39
:104CB0002046207C20282D29204E20282B29207CAE
:104CC00020470A2054207C20202020202020202043
:104CD00020207C20480A2020207C20202020282DF5
:104CE00029202020207C20540A2020207C202020E5
:104CF00020202020202020207C0A2020204F2D2D25
:104D00002046524F4E54202D2D2B0A2028302C3077
:104D1000290A004D65616E206F662073616D706CAD
:104D2000656420706F696E74733A200020643A20C5
:104D30000020623A200045716E20636F65666669E7
:104D40006369656E74733A20613A20003474682098
:104D500070726F626520706F696E742C2064697365
:104D600074616E63652066726F6D20706C616E6534
:104D70003A2000202844525952554E2900473239D2
:104D8000204175746F20426564204C6576656C69BE
:104D90006E67003F20284C2C522C462C4229206F55
:104DA0007574206F6620626F756E64732E0A003F03
:104DB00050726F626520706F696E74732028592974
:104DC00020697320696D706C61757369626C652010
:104DD00028322D32292E0A003F50726F62652070F2
:104DE0006F696E74732028582920697320696D706B
:104DF0006C61757369626C652028322D32292E0A28
:104E0000003F2856296572626F7365206C65766570
:104E10006C20697320696D706C61757369626C6573
:104E20002028302D34292E0A00506C6561736520CE
:104E30007265736574005052494E54455220484182
:104E40004C544544005072696E7465722068616C00
:104E50007465642E206B696C6C28292063616C6C0E
:104E60006564210A00656E7175657565696E6720F8
:104E700022000000A0C10080964300000000000056
:104E800048420000484200004040000000005761D6
:104E9000726E696E673A20486F6D696E6720427561
:104EA0006D702044697669736F72203C20310A006E
:104EB0000202040000A0400000A0400000004000EA
:104EC00000A0430080A04300008743FF01FF496E1C
:104ED000736572742066696C616D656E7420616EB5
:104EE0006420707265737320627574746F6E20280D
:104EF0006F72204D313038290A002F2F6163746999
:104F00006F6E3A726573756D650A004D3630303AD2
:104F100020546F6F20636F6C6400486F74656E641B
:104F200020746F6F20636F6C640A002F2F616374AD
:104F3000696F6E3A70617573650A004861726463E7
:104F40006F6465642044656661756C742053657494
:104F500074696E6773204C6F616465640A0028236E
:104F6000000028230000640000001027000000005B
:104F7000964300009643000040400000C8410000F6
:104F8000C9420000C9420000C8440000D2433A0AA6
:104F90000020286D6D290020204D36303320002060
:104FA00055004C0046696C616D656E74206C6F61D4
:104FB000642F756E6C6F6164206C656E67746873C6
:104FC0003A0A0020204D393030204B004C696E6584
:104FD000617220416476616E63653A0A0020204D5B
:104FE000383531205A005A2D50726F6265204F6655
:104FF000667365740020440020490020204D333042
:105000003420500020440020490020204D3330310E
:105010002050005049442073657474696E67733A78
:105020000A0020460020420020480020204D313454
:10503000352053004D6174657269616C206865614B
:1050400074757020706172616D65746572733A0A6F
:105050000020204D3432302053004175746F2042BF
:105060006564204C6576656C696E673A0A00205A63
:105070000020590020204D323036205800486F6DF6
:1050800065206F66667365743A0A00204500205AF1
:105090000020590020580020540020530020204DAB
:1050A00032303520420020453C6D61785F655F6A93
:1050B00065726B3E0020583C6D61785F785F6A6571
:1050C000726B3E20593C6D61785F795F6A65726BE7
:1050D0003E205A3C6D61785F7A5F6A65726B3E0074
:1050E000416476616E6365643A20423C6D696E5F2F
:1050F0007365676D656E745F74696D655F75733E2A
:1051000020533C6D696E5F66656564726174653ECF
:1051100020543C6D696E5F74726176656C5F666584
:105120006564726174653E002054002052002020A6
:105130004D323034205000416363656C6572617498
:10514000696F6E2028756E6974732F7332293A2047
:10515000503C7072696E745F616363656C3E20528F
:105160003C726574726163745F616363656C3E2059
:10517000543C74726176656C5F616363656C3E0A72
:1051800000204500205A0020590020204D323031A7
:105190002058004D6178696D756D20416363656CC1
:1051A00065726174696F6E2028756E6974732F73F0
:1051B00032293A0A00204500205A002059002020B8
:1051C0004D3230332058004D6178696D756D206621
:1051D00065656472617465732028756E6974732FD8
:1051E00073293A0A00204500205A00205900202047
:1051F0004D393220580053746570732070657220E9
:10520000756E69743A0A0020204D323030204430E7
:105210000A0020204D323030204400204469736160
:10522000626C65640A0046696C616D656E7420731A
:10523000657474696E67733A0020204D31343920EB
:1052400043203B20556E69747320696E2043656C62
:10525000736975730A002020473231202020203BDB
:10526000004C756C7A426F742054415A203620727B
:10527000656164792E005072696E74696E672E2EB6
:105280002E005072696E7420706175736564004DF4
:10529000313235004D3234005072696E74206162D3
:1052A0006F72746564005072696E742066726F6DFF
:1052B0002053440053746F70207072696E740052F2
:1052C0006573756D65207072696E740050617573D9
:1052D00065207072696E74004E6F205344206361C4
:1052E00072640041626F7574205072696E746572E9
:1052F000004368616E67652066696C616D656E74F8
:10530000004368616E67652066696C616D656E74E7
:10531000004D36303020423000436F6E666967754D
:10532000726174696F6E0054656D70657261747539
:105330007265004D6F76656D656E740054756E65AF
:1053400000496E666F2073637265656E004D6F76FF
:105350006520617869730044697361626C652073CC
:1053600074657070657273004D3834004175746FE8
:1053700020686F6D6500473238004D61696E004DE1
:105380003530320A4D353030004C6F616420736522
:105390007474696E677300526573746F726520660A
:1053A00061696C736166650053746F726520736523
:1053B0007474696E677300416476616E636564201E
:1053C00053657474696E6773004D61696E00526550
:1053D00073656E643A20002042002050006F6B001D
:1053E000627573793A2070617573656420666F72B7
:1053F00020696E7075740A00627573793A20706165
:105400007573656420666F7220757365720A006239
:105410007573793A2070726F63657373696E670A8A
:10542000004B494C4C45442E20004B494C4C2063CA
:10543000617573656420627920746F6F206D756388
:105440006820696E6163746976652074696D652092
:105450002D2063757272656E7420636F6D6D616E61
:10546000643A2000556E6B6E6F776E20636F6D6DC2
:10547000616E643A202200486F74656E6420746F18
:105480006F20636F6C640A0000000A0B02090C0DA8
:105490000E080703040100000000000000000000E7
:1054A00000000000000000000000000000000000FC
:1054B00000000000121110000000000000000000B9
:1054C000000000000000000000000000000050721A
:1054D0006F62696E67206661696C65640A0050726C
:1054E0006F62696E67206661696C656400205A3A74
:1054F000200020593A200042656420583A200000DC
:1055000012B3EC0011241FBECFEFD1E2DEBFCDBF3E
:1055100000E00CBF13E0A0E0B2E0E4EFF1E702E04E
:105520000BBF02C007900D92AC39B107D9F726E145
:10553000ACE9B3E001C01D92AA38B207E1F71AE264
:10554000C1E8DAE200E006C021970109802FFE01E0
:105550000F946B38C038D10780E00807A9F70E9484
:10556000109E0D94E9380C9400002F923F924F92B8
:105570005F926F927F928F929F92AF92BF92CF92E3
:10558000DF92EF92FF920F931F93CF93DF93CDB7EC
:10559000DEB7C657D1090FB6F894DEBF0FBECDBF38
:1055A000E5968FAFE59781E08093E31490914A0BE5
:1055B0009D3411F40C944B33943511F40C94E63F64
:1055C000973411F00C942A40E090480BF090490B6E
:1055D0002AE1E216F10409F499C6E4F444E0E41681
:1055E000F1044CF452E0E516F1040CF059C0F7FE5A
:1055F00033C00C94473384E0E816F10409F447C63D
:105600009CE0E916F10411F00C9447330E9444DA4F
:105610000C942C40AEE1EA16F10409F4F9C644F406
:10562000ECE1EE16F10409F4AAC60CF475C6ACC69A
:105630002BE5E216F10409F4BEC73CE5E316F104DC
:1056400009F4BDC74AE5E416F10411F00C944733A0
:105650001092A3030C942C4080911802882311F41B
:105660000C942C408AE50E94446E482F89E5E79609
:105670004FAFE7970E94446E682F88E5E6966FAFBC
:10568000E6970E94446EE7964FADE797E6966FADBA
:10569000E6970E9439D981110C942C400C94374024
:1056A00041E061E081E00E9439D981110C942C40E5
:1056B00080911802882311F40C942C4011E092E0A0
:1056C000E916F10409F010E00E9437D782E50E9444
:1056D0008B6E882309F45CC10E940D6E6B017C0106
:1056E00020916612309167124091681250916912B0
:1056F0002CAF3DAF4EAF5FAF80916A1290916B12AD
:10570000A0916C12B0916D1224968CAF9DAFAEAF8C
:10571000BFAF24972091E4143091E5144091E61432
:105720005091E7142C962CAF3DAF4EAF5FAF2C9746
:105730008091E8149091E914A091EA14B091EB14CF
:1057400028968CAF9DAFAEAFBFAF289720E030E07A
:10575000A901C701B6010F941231882309F47DC550
:105760002CAD3DAD4EAD5FAD2C966CAD7DAD8EAD2F
:105770009FAD2C970F941231811111C024962CAD3E
:105780003DAD4EAD5FAD249728966CAD7DAD8EAD31
:105790009FAD28970F941231882309F45EC520E04D
:1057A00030E0A901C701B6010F941231881F882784
:1057B000881F181307C0412C512C80E8682E8FE3F6
:1057C000782E06C0412C512C00E8602E0FEB702E75
:1057D0002CAD3DAD4EAD5FAD2C966CAD7DAD8EADBF
:1057E0009FAD2C970F947B3564966CAF7DAF8EAFD9
:1057F0009FAF649724962CAD3DAD4EAD5FAD249721
:1058000028966CAD7DAD8EAD9FAD28970F947B35FE
:1058100068966CAF7DAF8EAF9FAF689764962CADE6
:105820003DAD4EAD5FAD6497CA01B9010F947731BC
:105830004B015C0168962CAD3DAD4EAD5FAD6897F8
:10584000CA01B9010F9477319B01AC01C501B401C4
:105850000F947C350F94E73760966CAF7DAF8EAFB9
:105860009FAF609720E030E040E05FE30F94773136
:105870004B015C01A7019601C701B6010F94773176
:105880006B017C01A5019401C501B4010F9477312E
:105890009B01AC01C701B6010F947B350F94E7372C
:1058A0009B01AC01C301B2010F9477312B013C0184
:1058B0002C962CAD3DAD4EAD5FAD2C976CAD7DAD56
:1058C0008EAD9FAD0F947C3520E030E040E05FE38B
:1058D0000F9477316B017C0168966CAD7DAD8EAD18
:1058E0009FAD6897905860962CAD3DAD4EAD5FADC5
:1058F00060970F9458369B01AC01C301B2010F941D
:1059000077319B01AC01C701B6010F947C352CADFA
:105910003DAD4EAD5FAD0F947B356B017C0128969C
:105920002CAD3DAD4EAD5FAD289724966CAD7DADF1
:105930008EAD9FAD24970F947C3520E030E040E0A1
:105940005FE30F9477314B015C0160962CAD3DAD68
:105950004EAD5FAD609764966CAD7DAD8EAD9FAD85
:1059600064970F9458369B01AC01C301B2010F94A8
:1059700077319B01AC01C501B4010F947C352496AD
:105980002CAD3DAD4EAD5FAD24970F947B3514C06B
:1059900089E40E948B6E882329F00E940D6E6B01B2
:1059A0007C0103C0C12CD12C76018AE40E948B6E4D
:1059B0008823F9F00E940D6E2C966CAF7DAF8EAFF0
:1059C0009FAF2C9720E030E0A901C701B6010F94EA
:1059D000123181111EC020E030E0A9012C966CAD7F
:1059E0007DAD8EAD9FAD2C970F941231811111C0FA
:1059F00034C420E030E0A901C701B6010F94123190
:105A0000882309F42AC42C961CAE1DAE1EAE1FAE10
:105A10002C97A701960150582CAF3DAF4EAF5FAF0A
:105A20002C968CAD9DADAEADBFAD2C97B0582496E5
:105A30008CAF9DAFAEAFBFAF2497CA01B9010F9431
:105A400077314B015C0124962CAD3DAD4EAD5FAD81
:105A50002497CA01B9010F9477319B01AC01C501AC
:105A6000B4010F947C350F94E737A4966CAF7DAFEB
:105A70008EAF9FAFA497209166123091671240912C
:105A800068125091691228962CAF3DAF4EAF5FAFB0
:105A90002897A701960128966CAD7DAD8EAD9FAD80
:105AA00028970F947C3568966CAF7DAF8EAF9FAF13
:105AB000689780916A1290916B12A0916C12B091CC
:105AC0006D1260968CAF9DAFAEAFBFAF60972C9656
:105AD0002CAD3DAD4EAD5FAD2C97BC01CD010F940B
:105AE0007C35A8966CAF7DAF8EAF9FAFA897209105
:105AF000E4143091E5144091E6145091E714649653
:105B00002CAF3DAF4EAF5FAF649768962CAD3DAD07
:105B10004EAD5FAD689764966CAD7DAD8EAD9FADBB
:105B200064970F947B356B017C018091E814909110
:105B3000E914A091EA14B091EB146C968CAF9DAF70
:105B4000AEAFBFAF6C97A8962CAD3DAD4EAD5FAD7F
:105B5000A897BC01CD010F947B354B015C012091CE
:105B60006E1230916F124091701250917112A09686
:105B70002CAF3DAF4EAF5FAFA0976091EC1470912A
:105B8000ED148091EE149091EF140F947B352B015E
:105B90003C018091F0149091F114A091F214B09115
:105BA000F314E0968CAF9DAFAEAFBFAFE0972091FE
:105BB0007212309173124091741250917512AC961A
:105BC0002CAF3DAF4EAF5FAFAC97A70196016CAD68
:105BD0007DAD8EAD9FAD0F947731E4966CAF7DAF08
:105BE0008EAF9FAFE497A501940124966CAD7DAD77
:105BF0008EAD9FAD24970F9477319B01AC01E49655
:105C00006CAD7DAD8EAD9FADE4970F947C35E49681
:105C10006CAF7DAF8EAF9FAFE497A50194016CADE3
:105C20007DAD8EAD9FAD0F9477314B015C01A70127
:105C3000960124966CAD7DAD8EAD9FAD24970F94EB
:105C400077319B01AC01C501B4010F947B35E4961B
:105C50002CAD3DAD4EAD5FADE4970F94EF356B01CC
:105C60007C0120E030E0A9010F94123187FF0AC0C7
:105C70002BED3FE049EC50E4C701B6010F947C35B1
:105C80006B017C01112351F02BED3FE049EC50E416
:105C9000C701B6010F947B356B017C0120E030E039
:105CA000A901C701B6010F941231811128C0649671
:105CB0002CAD3DAD4EAD5FAD649728966CAD7DAD1E
:105CC0008EAD9FAD28970F941231811118C06C963C
:105CD0002CAD3DAD4EAD5FAD6C9760966CAD7DADBE
:105CE0008EAD9FAD60970F941231811108C0BBED4E
:105CF000CB2EBFE0DB2EB9ECEB2EB0E4FB2EA701E0
:105D00009601A4966CAD7DAD8EAD9FADA4970F941A
:105D100077314B015C0120E030E0A901C301B20101
:105D20000F9412318823C9F0A5019401C501B40173
:105D30000F9477314B015C01A3019201C301B201C1
:105D40000F9477319B01AC01C501B4010F947C35F0
:105D50000F94E7374B015C010DC020E030E0A90152
:105D6000C501B4010F94A23787FF04C0B7FAB094FD
:105D7000B7F8B0942FE632E143E85AE3C501B40125
:105D80000F94123187FF02C00C942C40C501B4015E
:105D90000F94F1360F94C5361B01672B19F422249A
:105DA0002394312CB10180E090E00F9416314B0127
:105DB0005C019B01AC01C701B6010F9458362896CF
:105DC0006CAF7DAF8EAF9FAF2897A5019401C30143
:105DD000B2010F945836A4966CAF7DAF8EAF9FAFD3
:105DE000A497AC962CAD3DAD4EAD5FADAC97E096B3
:105DF0006CAD7DAD8EAD9FADE0970F947B35A50169
:105E000094010F945836E0966CAF7DAF8EAF9FAF84
:105E1000E09728962CAD3DAD4EAD5FAD2897CA01F9
:105E2000B9010F94773120E030E040E05FE30F9458
:105E300077319B01AC0160E070E080E89FE30F9454
:105E40007B356C966CAF7DAF8EAF9FAF6C97A09695
:105E50008CAD9DADAEADBFADA09789879A87AB875E
:105E6000BC87AC962CAD3DAD4EAD5FADAC972D87EC
:105E70003E874F87588B6091000270910102072E78
:105E8000000C880B990B0F9418312091640230910B
:105E9000650240916602509167020F9477312AE0C3
:105EA00037ED43E25CE30F9477316CAB7DAB8EABA7
:105EB0009FAB0E9471959B01AC0128533F4F4F4F00
:105EC0005F4FA0962CAF3DAF4EAF5FAFA0974CACED
:105ED0005DAC6EAC7FAC41E050E062965FAF4EAF20
:105EE000629759E12D965FAF2D9762962EAD3FAD2B
:105EF00062972215330509F455C10E94338C0E9424
:105F00007195DC01CB01A0962CAD3DAD4EAD5FADE2
:105F1000A097821B930BA40BB50BB7FD11C00E9479
:105F200071959B01AC0128533F4F4F4F5F4FA09697
:105F30002CAF3DAF4EAF5FAFA09780E00F94FA203B
:105F40002D963FAD2D9731502D963FAF2D97332392
:105F500009F44BC06C962CAD3DAD4EAD5FAD6C976A
:105F600024966CAD7DAD8EAD9FAD24970F947731A7
:105F70006B017C0128962CAD3DAD4EAD5FAD2897F1
:105F8000B201C3010F947731A70196010F947C35BC
:105F90007B018C016C962CAD3DAD4EAD5FAD6C9729
:105FA000B201C3010F9477314B015C0128962CADEF
:105FB0003DAD4EAD5FAD289724966CAD7DAD8EADF9
:105FC0009FAD24970F9477319B01AC01C501B401BB
:105FD0000F947B352B013C01C701D80124968CAF6F
:105FE0009DAFAEAFBFAF24975DC062964EAD5FADC3
:105FF0006297BA0180E090E00F94163128962CAD9C
:106000003DAD4EAD5FAD28970F9477314B015C01EC
:106010000F9455366B017C01C501B4010F94DD3737
:106020004B015C01A70196016CAD7DAD8EAD9FADBE
:106030000F9477312B013C01A50194012C966CAD96
:106040007DAD8EAD9FAD2C970F9477319B01AC0148
:10605000C301B2010F947C352B013C01A5019401D1
:106060006CAD7DAD8EAD9FAD0F9477314B015C0172
:10607000A70196012C966CAD7DAD8EAD9FAD2C9792
:106080000F9477319B01AC01C501B4010F947B35AE
:1060900024966CAF7DAF8EAF9FAF249759E12D96BC
:1060A0005FAF2D979201A30168966CAD7DAD8EAD6B
:1060B0009FAD68970F947C3569837A838B839C832B
:1060C00024962CAD3DAD4EAD5FAD2497A8966CAD3A
:1060D0007DAD8EAD9FADA8970F947C356D837E838B
:1060E0008F839887A4962CAD3DAD4EAD5FADA49740
:1060F00069857A858B859C850F947C3569877A873D
:106100008B879C87E0962CAD3DAD4EAD5FADE097A3
:106110006D857E858F8598890F947C356D877E8708
:106120008F87988BCE0101960F948324E0906F1691
:106130001CA61DA61EA61FA689819A81AB81BC81C3
:1061400088A399A3AAA3BBA38D819E81AF81B885A3
:106150008CA39DA3AEA3BFA389859A85AB85BC857F
:1061600088A799A7AAA7BBA7AE01485D5F4FBE014C
:106170006C5D7F4FCE0180960E948184CE018C960B
:106180006C018E010C5C1F4F9E01235F3F4FAE01DF
:10619000485D5F4FBE016C5D7F4F0C970E94C54DFF
:1061A000811151C0E0906F1618AA19AA1AAA1BAA49
:1061B0008091E4149091E514A091E614B091E71455
:1061C00088A399A3AAA3BBA38091E8149091E91492
:1061D000A091EA14B091EB148CA39DA3AEA3BFA32E
:1061E0008091EC149091ED14A091EE14B091EF1405
:1061F00088A799A7AAA7BBA7AE01485D5F4FBE01BC
:106200006C5D7F4FCE0180960E948184DE01D09626
:106210006D018E010C5C1F4F20EF34E1AE01485D33
:106220005F4FBE016C5D7F4FCE0180960E94C54DD1
:1062300080E1E4EEF4E1A6E6B2E101900D928A95E8
:10624000E1F70C942C406296EEADFFAD629731966B
:106250006296FFAFEEAF629748CEE8EFFAE4849122
:106260008F010F5F1F4F882321F00F943D27F80106
:10627000F6CFE7EAF2E084918F010F5F1F4F88238A
:1062800011F40C942C400F943D27F801F4CF80E5D5
:106290000E948B6E882329F00E94CD6D6B017C01DA
:1062A00003C0C12CD12C760183E50E948B6E88231C
:1062B00061F00E940D6E20E030E04AE754E40F9454
:1062C00077310F94C5366B017C010E94755F809118
:1062D000A00E811105C060E08DEB92E00E945F6F1F
:1062E0000E947195C60ED71EE81EF91E0E94719578
:1062F000DC01CB018C199D09AE09BF09B7FD02C0B5
:106300000C942C4080E00F94FA20F0CF8093180278
:106310001092B3120C942C4041E061E081E00E94A5
:1063200039D981110C942C4080E090E0A8ECB2E4C3
:1063300089839A83AB83BC8380E090E0A6E9B3E4D1
:106340008D839E83AF83B88780E090E0A0EAB1E4BC
:1063500089879A87AB87BC8780E50E948B6E8823EC
:1063600019F00E94DD6D01C060E068A3BE016F5F9F
:106370007F4FCE0180960F94A7260C942C4080E08E
:106380000E94ACDB0C942C4080E00E94AED813E05D
:1063900001E01092741610927516109276161092F3
:1063A000771600937C0B24982C9A0898109A0E94D8
:1063B0000CFF10927C0B249A2C98089A10988091CC
:1063C0003515882351F080913515882369F084E4D0
:1063D00093E00F948D150C942C4084E793E00F9478
:1063E0008D151150B1F6EFCFEBE5F3E084918F01FD
:1063F0000F5F1F4F882321F00F943D27F801F6CF40
:1064000085ED92E00F948D1586EC92E00F94F215D5
:10641000C0906612D0906712E0906812F0906912F6
:1064200088E50E948B6E811108C020E030E0A90150
:10643000C701B6010F947C3502C00E940D6E68A39F
:1064400079A38AA39BA3C0906A12D0906B12E090AC
:106450006C12F0906D1289E50E948B6E811108C05C
:1064600020E030E0A901C701B6010F947C3502C0DD
:106470000E940D6E9B01AC0169837A838B839C83A0
:1064800068A179A18AA19BA10F94FF14882311F41C
:106490000C942C4080E00E94AED80E9404DA85E47F
:1064A0000E948B6E882321F00E94FE6D182F04C07D
:1064B00085E40E94446E11E086E50E948B6E88237D
:1064C00021F00E94DD6D262F01C021E0412FBE0189
:1064D0006F5F7F4FCE0180960F946E296B017C0118
:1064E0009B01AC010F94283881115FC088A099A04E
:1064F000AAA0BBA020E030E0A901C501B4010F941F
:10650000123187FD05C027E137EB41E558E304C0B0
:1065100027E137EB41E558EBC501B4010F947C3519
:10652000AB01BC018CEE93E00F94E40E89809A805D
:10653000AB80BC8020E030E0A901C501B4010F941C
:10654000123187FD05C027E137EB41E558E304C070
:1065500027E137EB41E558EBC501B4010F947C35D9
:10656000AB01BC0187EE93E00F94E40E20E030E035
:10657000A901C701B6010F94123187FD05C027E1BB
:1065800037EB41E558E304C027E137EB41E558EB31
:10659000C701B6010F947C35AB01BC0182EE93E0DC
:1065A0000F94E40E8AE00F943D270E94EBD90E94DD
:1065B00063FA0C942C408093A3030C942C4040E08D
:1065C00053E05DAF4CAFE6E6EE2EE2E1FE2EF8E7DB
:1065D000CF2EF6E1DF2E312C00E010E0ACADBDADEA
:1065E0008D91BDAFACAF0E948B6E8823B9F10E9434
:1065F0000D6E2B013C01133049F0F60120813181F1
:10660000428153810F947B352B013C01D7012D91A1
:106610003D914D915C91C301B2010F947B354B01CB
:106620005C012DEB37E346E855EB0F94A23787FD6D
:106630000AC02DEB37E346E855E3C501B4010F94DA
:10664000123118165CF4133011F001E002C033244B
:106650003394F70140825182628273821F5FF4E0BB
:10666000EF0EF11C24E0C20ED11C143009F0B6CF9D
:10667000002319F00E94876D06C0332021F082E7C5
:1066800092E10E94E4F60E9463FA0C942C400F946D
:10669000712C0C942C408091480B9091490B8937B8
:1066A000910511F40C94343C0CF0FEC08D3491052E
:1066B00009F42DC30CF079C08A31910509F494C214
:1066C0000CF040C08431910509F42DC294F481315D
:1066D000910509F424C244F4029710F00C94E33FAE
:1066E0000E9480FE0C942C40429709F449C60C94F9
:1066F000E33F8731910509F45DC274F4853191055A
:1067000009F454C2469711F00C94E33F1092640FC1
:106710001092650F0C942C408831910509F460C2E9
:10672000499711F00C94E33F1092640F0E9451B10D
:1067300084E194E090939B1280939A120E94286DBA
:106740000C942C408F31910509F468C29CF48C3173
:10675000910509F451C20CF44BC28D31910511F42D
:106760000C942C404E9711F00C94E33F0E94DFFBF9
:106770000C942C408934910509F4B8C24CF4803251
:10678000910509F443C28A9709F472C20C94E33F5D
:106790008B34910509F4B7C28C34910511F00C9437
:1067A000E33F0E9451B10C942C408B36910509F4C3
:1067B0002CC50CF040C08435910509F4E1C5CCF43A
:1067C0008135910509F4C1C534F48E34910509F47D
:1067D000A2C20C94E33F8235910509F4CEC58335FE
:1067E000910511F00C94E33F81E08093A2030C9497
:1067F0002C408836910509F490C39CF485359105A9
:1068000009F4F1C58C35910511F00C94E33F10E0CB
:10681000C12E13E0D12E0AE8E02E02E1F02E10E0A6
:10682000FBC58936910509F445C48A36910509F4FA
:10683000C7C40C94E33F8237910509F46CC6ACF4ED
:106840008E36910509F48AC334F48D36910509F426
:1068500071C40C94E33F8F36910509F492C38137DC
:10686000910509F4FEC30C94E33F8637910509F4C2
:10687000C3C654F48337910509F452C68537910590
:1068800009F4ABC60C94E33F8737910509F400C7C0
:106890008837910511F00C94E33F81E080937A0BE7
:1068A0008093780B0C942C408E3531E0930711F4D3
:1068B0000C94FA3D0CF08FC08E3C910511F40C94B1
:1068C000D13C0CF043C08E3B910509F465C4ACF497
:1068D0008C38910509F446C434F48D37910509F4D8
:1068E000AAC40C94E33F8139910509F4C2C78B39DE
:1068F000910509F4FAC30C94E33F8B3C910511F424
:106900000C94CB3CACF4883C910511F40C94B03C55
:10691000893C910511F00C94E33F3EE5E32E35E10F
:10692000F32E00E013E044E0D42ED00E0C94B33CE0
:106930008C3C910511F40C94CE3C8D3C910511F0EA
:106940000C94E33F0E94D3F80C942C40823251E027
:10695000950711F40C941F3DDCF48C3D910511F466
:106960000C94D73C4CF4833D910511F00C94E33F1B
:106970000E94F5F70C942C408D3D910511F40C9478
:10698000DA3C823E910511F40C94DD3C0C94E33F1B
:106990008E32B1E09B0711F40C94F43D6CF48C3210
:1069A000F1E09F0711F40C942A3D8D32914011F4CF
:1069B0000C94533D0C94E33F8F3231E0930711F474
:1069C0000C94F73D8033914011F00C94E33F0E940A
:1069D000B0800C942C40863F51E0950711F40C9444
:1069E000133F0CF04BC08239B1E09B0711F40C94BB
:1069F000033E14F58336F1E09F0711F40C94FD3D3E
:106A00004CF48F35914011F00C94E33F0E94D37504
:106A10000C942C40803941E0940711F40C94003E12
:106A20008139914011F00C94E33F81E00E94F3D84A
:106A30000E9463FA0C942C408C3AA1E09A0709F466
:106A4000B3C76CF4843AE1E09E0711F40C94093E5C
:106A5000893A914011F40C94923E0C94E33F843FA8
:106A600021E0920711F40C94103F853F914011F002
:106A70000C94E33F0F94B91C0C942C40833543E0F5
:106A8000940711F40C94303F2CF58C31A2E09A0756
:106A900011F40C94223F7CF4873FE1E09E0711F44F
:106AA0000C94163F883F914011F00C94E33F0E94F4
:106AB0004E790C942C40883522E0920711F40C9406
:106AC0002D3F8B35924011F00C94E33F0E94587695
:106AD0000C942C408C3843E0940711F40C94B43F90
:106AE00094F48438A3E09A0711F40C94333F8B3864
:106AF000934011F00C94E33F80E0E82E83E0F82E01
:106B000010E00C948D3F803AE3E09E0709F482C0C8
:106B1000873E934011F40C94CE3F0C94E33F0E94C7
:106B200076FE0C942C40E3E0F4E084918F010F5F3B
:106B30001F4F882321F00F943D27F801F6CF1092C4
:106B4000081240E050E0BA018BEB9FE00E9411E197
:106B50008BE1EBEBFFE0DE01159601900D928A953B
:106B6000E1F78091B90F9091BA0F9C838B838AE8EB
:106B700093E09A83898340E050E0BE016F5F7F4FCE
:106B800080E090E00E9491B7CE0101960F948515A8
:106B9000E4EFF3E084918F010F5F1F4F882311F41E
:106BA0000C942C400F943D27F801F4CF0E948DF2F5
:106BB0000C942C40E091460BF091470B8081882388
:106BC00029F0803209F410823196F8CF40E061E07C
:106BD0008091460B9091470B0E949CF00C942C40A6
:106BE0000E9431FD0C942C400E9417FD0C942C4007
:106BF0000E948FFC0C942C4040E060E08091460B9A
:106C00009091470B0E949CF00C942C400E949EFB9C
:106C10000C942C400E9493FB0C942C400E941DB1BC
:106C200068A379A38AA39BA3BE016F5F7F4FCE01A8
:106C300080960E9440B260E0CE0101960E940C72E4
:106C4000EDE9F2E484918F010F5F1F4F882321F05B
:106C50000F943D27F801F6CFBE016F5F7F4F89E1AA
:106C600094E00F941A0F8AE00F943D270C942C4067
:106C700083E50E948B6E882311F40C942C400E94B3
:106C8000ED6DE82E80E50E948B6E811114C081E0CD
:106C9000E11001C080E080937C0B882331F02498C0
:106CA0002C9A0898109A0C942C40249A2C98089AA4
:106CB00010980C942C4080E50E948B6E882339F04C
:106CC0000E94ED6D182F87FF03C00C942C401DE02F
:106CD000E6E2F4E08DE28E0F9491191711F40C9412
:106CE0004C4131968E13F8CF0C944F418091640F34
:106CF00081110C942C4080E50E94446E81110C940B
:106D00006A410C942C400E9466B10C942C400E9465
:106D1000C3B10C942C4083E50E948B6E811103C09B
:106D2000E1EBF4E009C00E94DD6D6E347105C1F73E
:106D30000E9430B20C942C4084918F010F5F1F4F42
:106D4000882321F00F943D27F801F6CFE8EAF4E01C
:106D500084918F010F5F1F4F882321F00F943D27EF
:106D6000F801F6CF6091680B7091690B80E090E0BC
:106D70004AE00F949027EBE9F4E084918F010F5FD4
:106D80001F4F882321F00F943D27F801F6CF609123
:106D90006A0B70916B0B80E090E04AE00F949027B3
:106DA000E0E9F4E084918F010F5F1F4F882321F009
:106DB0000F943D27F801F6CF6091680B7091690B35
:106DC00080916A0B90916B0B681B790B8091660B1D
:106DD000815021E030E0823010F020E030E0621B92
:106DE000730B80E090E04AE00F9490278AE00F94C4
:106DF0003D27E8E8F4E084918F010F5F1F4F88235F
:106E000021F00F943D27F801F6CF80916C0B909103
:106E10006D0BA0916E0BB0916F0B88A399A3AAA3E1
:106E2000BBA3BE016F5F7F4FCE0180960E9440B230
:106E3000EBE7F4E084918F010F5F1F4F811106C0D3
:106E40009E012F5F3F4F7901890104C00F943D27B8
:106E5000F801F0CFD8018D918D01882319F00F949E
:106E60003D27F8CF8091700B9091710BA091720B20
:106E7000B091730B88A399A3AAA3BBA3BE016F5FB4
:106E80007F4FCE0180960E9440B2EBE6F4E0849101
:106E90008F010F5F1F4F882321F00F943D27F801CA
:106EA000F6CFF70181917F01882319F00F943D27D8
:106EB000F8CF8AE00F943D27E3E6F4E084918F0158
:106EC0000F5F1F4F882321F00F943D27F801F6CF65
:106ED000E3E5F4E084918F010F5F1F4F882321F0D9
:106EE0000F943D27F801F6CF20E030E04AE754E464
:106EF0006091740B7091750B8091760B9091770B6C
:106F00000F94583642E00F9410288DE60F943D27D9
:106F10008AE00F943D270C942C4088E690E00E9474
:106F20009FDE81110C942C408091731683FF02C068
:106F30000C942C4083E50E948B6E882311F40C94F2
:106F40002C400E940D6E0F94C036709372166093A1
:106F5000711680E00E94FC880C942C408EE40E9404
:106F60008B6E882311F40C942C400E94DD6D60938D
:106F7000C1147093C2148093C3149093C4140C94DE
:106F80002C4083E50E94446E882359F083E50E94DB
:106F90008B6E882319F00E94ED6D01C080E0809314
:106FA0007316EDE9F2E484918F010F5F1F4F882380
:106FB00021F00F943D27F801F6CFE7ECF4E084913F
:106FC0008F010F5F1F4F882321F00F943D27F80199
:106FD000F6CF809173168823A1F179EBC72E74E068
:106FE000D72EE12CF12C20E08091731690E00E2C2E
:106FF00002C0959587950A94E2F780FF17C0BB24DD
:10700000B394B20E222319F08CE20F943D27F601BF
:1070100025913491F901849189010F5F1F4F8823D5
:1070200021F00F943D279801F5CF2B2DFFEFEF1A9C
:10703000FF0A32E0C30ED11C45E0E416F104A1F6CC
:107040000CC0E3ECF4E084918F010F5F1F4F8823A5
:1070500021F00F943D27F801F6CF8AE00F943D27E9
:10706000FBC783E50E948B6E882359F00E94ED6D6B
:107070008D3318F480935802EFC78CE38093580245
:10708000EBC7EDE9F2E484918F010F5F1F4F882376
:1070900021F00F943D27F801F6CF4091580250E0BF
:1070A00060E070E08EEC94E00F94C70E8AE00F94DD
:1070B0003D27D2C789E690E00E949FDE811111C072
:1070C000E5EDF4E084918F010F5F1F4F882321F0DD
:1070D0000F943D27F801F6CF0E94F7878AE00F94BE
:1070E0003D271092E3140C94EB4583E50E948B6ED0
:1070F000882309F4B1C70E94ED6D182F8D3308F075
:107100001CE31093C1150E9471956B017C01212F26
:1071100030E0A8EEB3E00F946C35C60ED71EE81E23
:10712000F91EC092BD15D092BE15E092BF15F09227
:10713000C01592C78DE690E00E949FDE81118CC73A
:107140008091731683FD88C783E50E948B6E8CAF98
:1071500081110C94754182E50E948B6E81110C9413
:1071600075417AC78091731683FD76C783E50E94C7
:107170008B6E882309F470C70E940D6E0F94C03681
:107180006639710514F066E970E07093130B609333
:10719000120B0E94B18860C78091731683FD5CC793
:1071A00083E50E948B6E65968FAF659781110C9475
:1071B000164382E50E948B6E81110C9416434CC7D6
:1071C00080E50E948B6E882339F00E94ED6D182FA8
:1071D000823008F041C701C010E083E50E948B6E49
:1071E000882319F00E94DD6D02C06FEF70E0E12F7F
:1071F000F0E06F3F710510F06FEF70E0EE0FFF1FD2
:10720000ED58F24F7183608327C780E50E948B6E33
:10721000882339F00E94DD6D6230710508F01CC7CB
:1072200002C060E070E0660F771FFB01ED58F24F7F
:107230001182108211C78CE40E94446E882381F071
:107240000E940D6E6B017C0120E030E0A9010F94DB
:10725000A23787FF0AC0F7FAF094F7F8F09405C058
:10726000C12CD12CE12C80E4F82EF7FAF094F7F839
:10727000F094CCA6DDA6EEA6FFA680E090E0A8ECF8
:10728000B2E489839A83AB83BC8380E090E0A6E973
:10729000B3E48D839E83AF83B88780E090E0A0EA5B
:1072A000B1E489879A87AB87BC8788E50E948B6E9B
:1072B000882379F088E50E948B6E882319F00E945C
:1072C0000D6E03C060E070E0CB0169837A838B832D
:1072D0009C8389E50E948B6E882379F089E50E9462
:1072E0008B6E882319F00E940D6E03C060E070E081
:1072F000CB016D837E838F8398878AE50E948B6E96
:10730000882379F08AE50E948B6E882319F00E9409
:107310000D6E03C060E070E0CB0169877A878B87D0
:107320009C8718A219A21AA21BA280918B0E811110
:1073300093C620E0AE01405E5F4FBE016F5F7F4F9E
:10734000CE018C960F94021187C60E9447890E9435
:10735000865F1092740D1092730D1092760D10923C
:10736000750D68EE73E080E090E00E948F9B60E016
:1073700086E295E00E945F6F6FC61092A2036CC612
:1073800083E50E948B6E882399F00E940D6E20E0A9
:1073900030E04AE754E40F9477310F94C536609398
:1073A000590270935A0280935B0290935C0254C618
:1073B00088E50E94446E81110C94C14489E50E94C5
:1073C000446E81110C94C1448AE50E94446E81117F
:1073D0000C94C14485E40E94446E81110C94C14414
:1073E0000E94865F39C683E50E94446E882309F4B3
:1073F00033C60E940D6E20E030E04AE754E40F945B
:1074000077310F94C53660939D1570939E158093C8
:107410009F159093A01520C6D6018D916D010E94F5
:10742000446E882309F46DC0133009F063C00E94D4
:107430000D6E4B015C0120E030E040EA51E40F9416
:10744000123187FF4EC0A501940160919612709190
:10745000971280919812909199120F9458362B019F
:107460003C019B01AC0160914215709143158091E4
:107470004415909145150F947731609342157093A0
:1074800043158093441590934515A3019201609193
:107490007A1570917B1580917C1590917D150F94D4
:1074A000773160937A1570937B1580937C15909358
:1074B0007D156091FD037091FE038091FF03909113
:1074C00000040F941631A30192010F9477310F94A9
:1074D000C5366093FD037093FE038093FF03909382
:1074E00000048092961290929712A0929812B092F5
:1074F000991207C00E940D6EF70160837183828329
:1075000093831F5FF4E0EF0EF11C143009F084CF79
:107510000E94726CA1C50E94755F0E9463FA9CC5AF
:10752000E8E1F6E084918F010F5F1F4F882321F07F
:107530000F943D27F801F6CF60E088E096E00E94C6
:107540001FFA61E081E096E00E941FFA61E086EF99
:1075500095E00E941FFA61E086EE95E00E941FFA16
:1075600060E08DED95E00E941FFA61E083ED95E00B
:107570000E941FFA61E089EC95E00E941FFA61E029
:1075800081EC95E00E941FFA61E083EB95E00E9498
:107590001FFA61E085EA95E00E941FFA60E086E943
:1075A00095E00E941FFA60E088E895E00E941FFACB
:1075B00060E082E795E00E941FFA61E081E695E0D5
:1075C0000E941FFA60E08CE495E00E941FFA61E0DF
:1075D00089E395E00E941FFA3FC58091460B909188
:1075E000470BDC012C91211103C00F947B1E34C585
:1075F00060E00E940C7230C50091460B1091470B61
:1076000083E0D12C40E08150E1F0F8019081292FF6
:107610002B7F2134C1F721812133A9F7913421F047
:10762000953421F441E002C0DD24D39498012E5F0B
:107630003F4F89012F5F3F4FD8019C919032C9F392
:10764000E2CF442369F0EDE9F2E484917F01BFEFDA
:10765000EB1AFB0A882321F00F943D27F701F5CFA1
:10766000DD2069F0EFE0F7E084917F012FEFE21A6F
:10767000F20A882321F00F943D27F701F5CFD801B6
:107680008D918D01882309F4E8CC0F943D27F7CF25
:1076900081E080937C0B24982C9A0898109AEDE452
:1076A000F7E084918F010F5F1F4F882321F00F9423
:1076B0003D27F801F6CFE5E4F7E084918F010F5FF5
:1076C0001F4F882321F00F943D27F801F6CF1E9914
:1076D00003C009EE12E002C00EEE12E0F801819143
:1076E0008F01882319F00F943D27F8CF8AE00F947B
:1076F0003D27EDE3F7E084918F010F5F1F4F882353
:1077000021F00F943D27F801F6CF029B03C009EE4C
:1077100012E002C00EEE12E0D8018D918D01882397
:1077200019F00F943D27F8CF8AE00F943D27E5E349
:10773000F7E084918F010F5F1F4F882321F00F9492
:107740003D27F801F6CF1D9903C009EE12E002C0F3
:107750000EEE12E0F80181918F01882319F00F9449
:107760003D27F8CF8AE00F943D27EDE2F7E08491C2
:107770008F010F5F1F4F882321F00F943D27F801E1
:10778000F6CF019903C009EE12E002C00EEE12E03E
:10779000D8018D918D01882319F00F943D27F8CFE2
:1077A0008AE00F943D27E5E2F7E084918F010F5FB7
:1077B0001F4F882321F00F943D27F801F6CF1C9B23
:1077C00003C009EE12E002C00EEE12E0F801819152
:1077D0008F01882319F00F943D27F8CF8AE00F948A
:1077E0003D27EDE1F7E084918F010F5F1F4F882364
:1077F00021F00F943D27F801F6CF379903C009EE29
:1078000012E002C00EEE12E0D8018D918D018823A6
:1078100019F00F943D27F8CF8AE00F943D27E3E15C
:10782000F7E084918F010F5F1F4F882321F00F94A1
:107830003D27F801F6CF009B03C009EE12E002C01D
:107840000EEE12E0F80181918F01882319F00F9458
:107850003D27F8CF8AE00F943D2710927C0B249AA5
:107860002C98089A1098F8C310927A0B1092780B03
:10787000F3C383E50E948B6E882319F00E94DD6DAF
:1078800002C060E070E08B01112702301105CCF0DE
:10789000E8EFFAE484918F010F5F1F4F882321F0F6
:1078A0000F943D27F801F6CFE7E6F7E084918F01CA
:1078B0000F5F1F4F882309F4CFC30F943D27F801B2
:1078C000F5CF88E40E948B6E8823A9F00E94DD6DBD
:1078D000683771053CF06332F1E07F072CF062E21B
:1078E00071E002C068E770E0F801EE0FFF1FEF5C87
:1078F000FA4E7183608386E40E948B6E8823A9F020
:107900000E94DD6DF801EE0FFF1FE75DFA4E7183F7
:1079100060836F3F710519F014F06FEF70E077FF2F
:1079200002C060E070E07183608382E40E948B6E2D
:10793000882309F491C30E94DD6D6530710534F030
:10794000683871052CF067E870E002C065E070E00F
:10795000000F111FF801E35DFA4E718360837CC351
:107960000E94D6F979C3D8018D918D010E94446E91
:10797000882349F00E940D6E0F94C536F70160838D
:10798000718382839383F4E0EF0EF11CD012EBCF6E
:107990000E94F66A61C30E94B4F95EC30E943DF979
:1079A0005BC30E9450FB58C30E94727955C30E946A
:1079B000A48152C30E942F814FC380E50E94446E70
:1079C000882309F449C30E94DD6D6B017C0183E5C6
:1079D0000E948B6E882321F00E94DD6D8B0102C016
:1079E0000FEF1FEF98012F5F3F4F2330310508F055
:1079F00033C3D7FC31C30E94755F0F3F2FEF1207CF
:107A000031F00130110571F401E010E00DC08C2D52
:107A10000E947D9331E020E0892B09F030E0032FB4
:107A2000122F02C000E010E08C2D0E947D93801781
:107A3000910709F411C380E00F94FA20F5CF8AE58D
:107A40000E948B6E8111C8C783E50E948B6E8111E5
:107A5000C3C702C383E50E948B6E882319F00E947E
:107A6000DD6D02C064E071E079A368A380E50E9447
:107A70008B6E882339F00E94DD6D693833E173071E
:107A800030F402C068EE73E07A83698304C088E84A
:107A900093E19A838983BE01605E7F4FCE01019698
:107AA0000E94CEF3D9C285E40E948B6E811110C072
:107AB00080E50E94446E882391F00E940D6E6093D1
:107AC000251570932615809327159093281507C0C8
:107AD0000E94ED6D882361F3E8EFFAE46EC089E45B
:107AE0000E94446E882381F00E940D6E2CEA35ECD2
:107AF00047E25EE30F94773160932115709322156E
:107B0000809323159093241584E40E94446E882367
:107B100081F00E940D6E2CEA35EC47E25EE30F9493
:107B2000583660931D1570931E1580931F15909302
:107B30002015EDE9F2E484918F010F5F1F4F882338
:107B400021F00F943D27F801F6CF40912515509173
:107B50002615609127157091281582EA97E00F94F9
:107B6000E40E2CEA35EC47E25EE36091211570915A
:107B7000221580912315909124150F945836AB014E
:107B8000BC018EE997E00F94E40E2CEA35EC47E255
:107B90005EE360911D1570911E1580911F159091E7
:107BA00020150F947731AB01BC018AE997E00F945F
:107BB000E40E8AE00F943D274FC284918F010F5F3E
:107BC0001F4F882321F00F943D27F801F6CFE6EAF6
:107BD000F7E084918F010F5F1F4F882309F43CC2A7
:107BE0000F943D27F801F5CF0E945A8035C20E94BC
:107BF000B27A32C20E9422762FC20E94B8752CC27D
:107C00000E94755F29C280E00E94F3D80E9463FA47
:107C100023C283E50E94446E882349F00E94FE6DD2
:107C2000182F811106C080E00E94AED802C01091CA
:107C300035158091661290916712A0916812B091EB
:107C4000691289839A83AB83BC8380916A12909175
:107C50006B12A0916C12B0916D128D839E83AF83D5
:107C6000B88780916E1290916F12A0917012B091AE
:107C7000711289879A87AB87BC8786E50E94446E1C
:107C8000882321F085EE97E00F94862B812F0E94A8
:107C9000AED8111103C0EDE9F2E41CC08091351596
:107CA0008111F9CFE8EFFAE484918F010F5F1F4F44
:107CB000882321F00F943D27F801F6CFE6ECF7E09A
:107CC00084918F010F5F1F4F882329F30F943D2765
:107CD000F801F6CF84918F010F5F1F4F882321F0A9
:107CE0000F943D27F801F6CF80913515811103C01F
:107CF0006CEF72E002C068EF72E088EB97E00F94DF
:107D00001A0F8AE00F943D274CE050E066E672E1DE
:107D1000CE0101960F947B38892B09F49DC10E94F6
:107D200063FA9AC18AE50E94446E882329F1809102
:107D30009D0390919E03892B19F00E940D6E08C03F
:107D400060917416709175168091761690917716E1
:107D50006093DE037093DF038093E0039093E1036D
:107D600080E090E0A0E8BFE38093E2039093E30318
:107D7000A093E403B093E50386E40E94446E882355
:107D800081F10E940D6E20E030E040E85FE30F9447
:107D9000A23718166CF40E940D6E20E030E040E827
:107DA0005FE30F94A237181684F00E940D6E11C085
:107DB0000E940D6E20E030E0A9010F94123187FF80
:107DC000EACF60E070E0CB0104C060E070E080E8E2
:107DD0009FE36093E2037093E3038093E403909343
:107DE000E50383E50E94446E882351F00E940D6EE6
:107DF0006093020270930302809304029093050241
:107E00008AE50E94446E811127C186E40E94446E77
:107E1000811122C183E50E94446E81111DC156C6A5
:107E20000E94F7C819C10F94551B16C183E50E9423
:107E3000446E882321F00E94FE6D91E089270F9403
:107E400053160AC183E50E94446E882309F404C1D5
:107E50000E94FE6D80938F0BFFC00E94E576FCC0F0
:107E60000E94DC78F9C08BE40E948B6E8823B1F10C
:107E70008BE40E948B6E8823B1F00E940D6E6B0123
:107E80007C0120E030E0A9010F94A23787FD19C0E2
:107E900020E030E040E251E4C701B6010F94123116
:107EA00018167CF003C0C12CD12C76010E94755F9E
:107EB000C0920D15D0920E15E0920F15F09210158C
:107EC000CBC0E4EEF8E084918F010F5F1F4F882351
:107ED00009F4C2C00F943D27F801F5CFEDE9F2E4B3
:107EE00084918F010F5F1F4F882321F00F943D274E
:107EF000F801F6CF40910D1550910E1560910F15B8
:107F00007091101583E099E00F94E40E8AE00F94CD
:107F10003D27A2C01F5F143069F0D7018D917D010C
:107F20000E94446E8823B1F30E94DD6D812F0E9470
:107F3000B961F0CF82E40E94446E882329F00E9448
:107F4000DD6D84E00E94B96183E50E94446E882360
:107F500009F482C010E00E94DD6D812F0E94B9619A
:107F60001F5F1530C1F778C083E50E948B6E8823B0
:107F700021F00E94DD6D8B0102C000E010E080E581
:107F80000E948B6E882321F00E94DD6DCB0102C020
:107F900080E090E0B8010E94AA615EC081E0809319
:107FA00018021092B31283E50E948B6E882339F079
:107FB0000E94FE6D811150C00F943C254DC083E599
:107FC0000E94446EF7CF0F94712C46C0F090480B7E
:107FD0000E94755FFF2029F1EDE9F2E484918F01A1
:107FE0000F5F1F4F882321F00F943D27F801F6CF34
:107FF00084E50F943D276F2D70E080E090E04AE02B
:108000000F94902780E20F943D27E0E2F9E08491FD
:108010008F010F5F1F4F8823F9F00F943D27F80160
:10802000F6CF10926F16EDE9F2E484918F010F5FA5
:108030001F4F882321F00F943D27F801F6CF609160
:108040006F1670E08EE099E00F94010F8AE00F94B4
:108050003D2702C00F94712C1092E314E596BFAD3A
:10806000E597BB2309F4B7C50F94D824B4C50E9483
:1080700037D784EE94E10F9483248091731683FDA7
:10808000A5C0C090F014D090F114E090F214F090DC
:10809000F314209172123091731240917412509126
:1080A0007512C701B6010F941231882309F48EC0EE
:1080B00060916B1670916C1680916D1690916E1692
:1080C00020917016211129C00F94C03620915E02B4
:1080D00030915F026217730704F5C0927212D0925A
:1080E0007312E0927412F0927512EDE9F2E4849149
:1080F0008F010F5F1F4F882321F00F943D27F80158
:10810000F6CFECE8F2E084918F010F5F1F4F8823D8
:1081100021F00F943D27F801F6CF8090F014909055
:10812000F114A090F214B090F314209172123091D7
:1081300073124091741250917512C501B4010F94DD
:108140007B356B017C0120E030E0A9010F94A23760
:1081500087FF04C0F7FAF094F7F8F094E0916F16F7
:1081600054E0E59FF0011124EA5FFD4F2081318149
:1081700042815381C701B6010F94773120E030E08E
:1081800048E453E40F94A237181604F58092721253
:1081900090927312A0927412B0927512EDE9F2E40B
:1081A00084918F010F5F1F4F882321F00F943D278B
:1081B000F801F6CFEDE6F2E084918F010F5F1F4FDB
:1081C000882321F00F943D27F801F6CF609100023B
:1081D00070910102072E000C880B990B0F94183137
:1081E00020916402309165024091660250916702CD
:1081F0000F9477312AE037ED43E25CE30F94773157
:108200006CA77DA78EA79FA7E0906F168091EC14B6
:108210009091ED14A091EE14B091EF144091E814F8
:108220005091E9146091EA147091EB140091E414F8
:108230001091E5142091E6143091E71409831A8314
:108240002B833C8348A359A36AA37BA38CAB9DAB30
:10825000AEABBFAB18AE19AE1AAE1BAEAE014C5CE6
:108260005F4FBE01605E7F4FCE0101960E94818408
:10827000CE01C8966C018E01045D1F4F20EF34E1E2
:10828000AE014C5C5F4FBE01605E7F4FC7970E949E
:10829000C54D0E94A76EE0CE0E9478FBDDCE812FF7
:1082A0000E942DB46E2D812F0E94A593F12CB70151
:1082B000812F0E947294163029F4F092760DE0928C
:1082C000750DCACE183009F0C7CEF092740DE09249
:1082D000730DC2CE0E94ED6D853620F084E680934A
:1082E0009C03BACE80939C03B7CE0E940D6E0F9470
:1082F000C036709372166093711680E00E94FC88FD
:108300006091711670917216072E000C880B990BF4
:108310000F94183120916B1630916C1640916D16A8
:1083200050916E160F94A237181634F05CAD5111AF
:1083300008C08CED94E002C080EF94E060E00E9401
:108340005F6F81E080935D022C961CAE1DAE1EAE69
:108350001FAE2C97A8961CAE1DAE1EAE1FAEA897E2
:1083600021961FAE219769961FAE69978CE36D9693
:108370008FAF6D979CE1A9969FAFA997A6E4A196B0
:10838000AFAFA197C12CD12C50E8E52E6FEBF62EA4
:10839000412C512C32016091711670917216072E8A
:1083A000000C880B990B0F9418311B01182F092F03
:1083B0009B01482F592FB601C7010F941231882312
:1083C000C9F020916B1630916C1640916D1650914A
:1083D0006E16B101812F902F0F941231881F8827BC
:1083E000881F21968FAF2197BCADBB2331F0882326
:1083F00021F0A0C116011E2D0F2D0E9471956B0159
:108400007C01DC01CB01A8962CAD3DAD4EAD5FAD3E
:10841000A897821B930BA40BB50BB7FD3DC0D701EA
:10842000C60188519C4FAF4FBF4FA8968CAF9DAFF0
:10843000AEAFBFAFA8970E94F787E8EDF4E0849154
:108440005F019FEFA91AB90A882321F00F943D27F5
:10845000F501F5CF4114510461047104B9F0D30161
:10846000C20188519C4FAF4FBF4FBC01CD016C1969
:108470007D098E099F0928EE33E040E050E00F941B
:108480001E35CA01B9010F94F62703C08FE30F947C
:108490003D278AE00F943D2780E00F94FA200E9448
:1084A00071956093991570939A1580939B1590938D
:1084B0009C15A0916B162596AFAF2597B0916C16C1
:1084C0002D96BFAF2D97E0916D166196EFAF619736
:1084D000F0916E166596FFAF65979D01AF01B101F2
:1084E000812F902F0F947B354B015C0120E030E011
:1084F000A9010F94A23787FF04C0B7FAB094B7F868
:10850000B09420E030E040E251E4C501B4014114F0
:1085100051046104710429F40F94123187FF07C0DC
:1085200004C00F94A237181614F4260137012196BF
:108530002FAD2197222309F45EC02C968CAD9DAD02
:10854000AEADBFAD2C97892B8A2B8B2B71F0D70149
:10855000C6012C962CAD3DAD4EAD5FAD2C97821B68
:10856000930BA40BB50BB7FD46C025962FAD2597F1
:108570002D963FAD2D9761964FAD619765965FAD96
:10858000659769966FAD69976D967FAD6D97A99662
:108590008FADA997A1969FADA1970F947B3520E051
:1085A00030E040EC5FE30F94123187FDC3C0D70188
:1085B000C601805A9541AF4FBF4F2C968CAF9DAFEF
:1085C000AEAFBFAF2C9725969FAD259769969FAF0D
:1085D00069972D96AFAD2D976D96AFAF6D9761965C
:1085E000BFAD6197A996BFAFA9976596EFAD6597A7
:1085F000A196EFAFA19780915D02882309F49AC0FC
:10860000411451046104710421F46101E12EF02E42
:10861000C2CEF8EECF1AF3E0DF0AE108F108C41881
:10862000D508E608F708F7FE85C0EFCF0E940D6E6B
:108630000F94C036663971050CF0A0C17093130B0E
:108640006093120B0E94B1886091120B7091130B12
:10865000072E000C880B990B0F94183120910E0BEC
:1086600030910F0B4091100B5091110B0F94A237CA
:1086700018160CF466C088E095E060E00E945F6F19
:1086800081E080935D0280916F1680930D0B24969C
:108690001CAE1DAE1EAE1FAE2497A8961CAE1DAE1E
:1086A0001EAE1FAEA8971CAE69961FAE69972CE34D
:1086B0006D962FAF6D973CE1A9963FAFA99746E421
:1086C000A1964FAFA197C12CD12C30E8E32E4FEBF0
:1086D000F42E412C512C32016091120B7091130B2E
:1086E000072E000C880B990B0F9418311B01182FC3
:1086F000092F9B01482F592FB601C7010F94123142
:10870000882311F120910E0B30910F0B4091100B2B
:108710005091110BB101812F902F0F941231881FAE
:108720008827881F8CAF65965FAD6597552379F0D4
:10873000882369F080915D02882309F48DCC0C9424
:10874000F53A87E195E099CF16011E2D0F2D0E9475
:1087500071956B017C01DC01CB01A8962CAD3DAD80
:108760004EAD5FADA897821B930BA40BB50BB7FD65
:108770003DC0D701C60188519C4FAF4FBF4FA8964F
:108780008CAF9DAFAEAFBFAFA8970E94F787E4E074
:10879000F5E084915F019FEFA91AB90A882321F0BF
:1087A0000F943D27F501F5CF411451046104710484
:1087B000B9F0D301C20188519C4FAF4FBF4FBC01EC
:1087C000CD016C197D098E099F0928EE33E040E048
:1087D00050E00F941E35CA01B9010F94F62703C06B
:1087E0008FE30F943D278AE00F943D2780E00F949C
:1087F000FA200E9471956093991570939A15809351
:108800009B1590939C15A0910E0B2996AFAF2997BD
:10881000B0910F0B2596BFAF2597E091100B2D96C9
:10882000EFAF2D97F091110B6196FFAF61979D010E
:10883000AF01B101812F902F0F947B354B015C016B
:1088400020E030E0A9010F94A23787FF04C0B7FAF7
:10885000B094B7F8B09420E030E040EA50E4C501AD
:10886000B401411451046104710429F40F941231CC
:1088700087FF07C004C00F94A237181614F426010E
:1088800037012CAD222309F45EC024968CAD9DAD3A
:10889000AEADBFAD2497892B8A2B8B2B71F0D701FE
:1088A000C60124962CAD3DAD4EAD5FAD2497821B25
:1088B000930BA40BB50BB7FD46C029962FAD299796
:1088C00025963FAD25972D964FAD2D9761965FADBF
:1088D000619769966FAD69976D967FAD6D97A99613
:1088E0008FADA997A1969FADA1970F947B3520E0FE
:1088F00030E040EC5FE30F94123187FD1BCFD701CE
:10890000C601805A9541AF4FBF4F24968CAF9DAFA3
:10891000AEAFBFAF249729969FAD299769969FAFB9
:1089200069972596AFAD25976D96AFAF6D972D964C
:10893000BFAD2D97A996BFAFA9976196EFAD61978F
:10894000A196EFAFA19780915D02882309F4F2CE42
:10895000411451046104710421F46101E12EF02EEF
:10896000BBCEF8EECF1AF3E0DF0AE108F108C41835
:10897000D508E608F708F7FEDDCEEFCF66E970E030
:108980005DCE0E94755F88E50E94446E882331F0B9
:10899000179A80917B0B8E7F80937B0B89E50E94D9
:1089A000446E882331F0169A80917B0B8D7F8093E3
:1089B0007B0B8AE50E94446E882331F0159A8091E2
:1089C0007B0B8B7F80937B0B85E40E94446E882316
:1089D00009F442CB149A40CB0E940D6E20E030E0A7
:1089E00040E050EC0F94123187FD15C00E940D6ECF
:1089F00020E030E040E050E40F94A23718162CF04D
:108A00000E940D6E6B017C010BC0C12CD12CE12C9E
:108A100020E4F22E05C0C12CD12CE12C90ECF92ED3
:108A2000209192123091931240919412509195128C
:108A300080917B0B82FF10C00091F90A1091FA0A15
:108A4000C701B6010F9477310F94C036600F711FC4
:108A50007093FA0A6093F90A80E50E94446E8823B5
:108A600029F00E94FE6D882309F4F6CAA701960139
:108A700060917612709177128091781290917912AC
:108A80000F947C35609376127093771280937812EE
:108A900090937912EDE9F2E484918F010F5F1F4FFB
:108AA000882321F00F943D27F801F6CF40917612EC
:108AB00050917712609178127091791289E897E05D
:108AC0000F94E40E8AE00F943D27C6CA40917416B5
:108AD00050917516609176167091771687EC98E034
:108AE0000F94E40E8AE00F943D278AE00F943D270F
:108AF00020E030E0A9016091DE037091DF038091F6
:108B0000E0039091E1030F94A23718160CF056C0C1
:108B100020E030E0A9016091E2037091E3038091CD
:108B2000E4039091E5030F94A23718160CF046C0A9
:108B3000E5E8F8E084918F010F5F1F4F882321F053
:108B40000F943D27F801F6CF4091DE035091DF03EB
:108B50006091E0037091E1038BE698E00F94E40EDE
:108B60008AE00F943D2740910202509103026091E8
:108B700004027091050281E598E00F94E40E8AE00A
:108B80000F943D274091E2035091E3036091E40389
:108B90007091E50387E398E00F94E40E8AE00F9468
:108BA0003D27E2E0F8E084918F010F5F1F4F88239B
:108BB00009F452CA0F943D27F801F5CFE5EAF8E031
:108BC00084918F010F5F1F4F882309F4BDCF0F944D
:108BD0003D27F801F5CFCA58DF4F0FB6F894DEBF36
:108BE0000FBECDBFDF91CF911F910F91FF90EF90FE
:108BF000DF90CF90BF90AF909F908F907F906F90BD
:108C00005F904F903F902F9008954F925F926F9298
:108C10007F92BF92CF92DF92EF92FF920F931F93BA
:108C2000CF93DF93CDB7DEB72A970FB6F894DEBFA8
:108C30000FBECDBF10922C0A8091640F882351F192
:108C400020915611222321F180910012909101125E
:108C5000A0910212B09103120097A105B105B9F0DD
:108C6000BC01CD016D597F4F8F4F9F4F24E630E0FF
:108C700040E050E00F941E3560910412709105128F
:108C800080910612909107120F941E3501C020E0CA
:108C900020939C038091320A1092320A882339F083
:108CA0000E9440AF84E091E00E94EDB503C52091A1
:108CB00000023091010240919C0E50919D0E6091F6
:108CC0009E0E70919F0EC901840F951F24363105A9
:108CD00024F4853691053CF416C02436310531F074
:108CE0008436910584F484E690E00DC04730510548
:108CF0006105710514F0069706C04A3F5F4F6F4F3C
:108D00007F4F6CF4069690930102809300021092BC
:108D10009C0E10929D0E10929E0E10929F0E8091AE
:108D20000002909101028A3091053CF0883E43E0B8
:108D300094072CF087EE93E002C08AE090E09093D5
:108D40000102809300020E947275B82E0E94006F8B
:108D500080914712853198F4BB2049F08091730DC2
:108D60009091740D892B19F00BE91FE002C00EE7FA
:108D70001EE023E14FE061E088E00E9486B480912C
:108D800047128D3108F008C18830A0F58091970E08
:108D9000B11002C081112EC06091711670917216CF
:108DA000072E000C880B990B0F94183120E030E04F
:108DB00040E05FE30F947C350F94C036CB010E94F6
:108DC000599BFC012081203229F42181203221F499
:108DD00036E003C030E001C033E025E0231B2093E0
:108DE0004A1227E020934B120E94E9AF8BE79EE0E6
:108DF0000E94DCAF809147128D31A0F5809149121D
:108E0000853180F120E030E040E05FE360916B1657
:108E100070916C1680916D1690916E160F947C3542
:108E20000F94C036CB010E94599BFC018081803297
:108E300009F0B7C28181803209F0ACC296E085E0CA
:108E4000891B80934A128CE180934B12CF010E94C0
:108E5000E9AF8BE79EE00E94DCAF8091471285313D
:108E600008F49AC2809147128830A0F58091960E3E
:108E7000B11002C081112EC06091120B7091130BC2
:108E8000072E000C880B990B0F94183120E030E06E
:108E900040E05FE30F947C350F94C036CB010E9415
:108EA000599BFC012081203229F42181203221F4B8
:108EB00036E003C030E001C033E021E5231B2093FE
:108EC0004A1227E020934B120E94E9AF8BE79EE005
:108ED0000E94DCAF809147128D31A0F5809149123C
:108EE000853180F120E030E040E05FE360910E0BDF
:108EF00070910F0B8091100B9091110B0F947C359A
:108F00000F94C036CB010E94599BFC0180818032B6
:108F100009F07DC28181803209F072C296E081E55C
:108F2000891B80934A128CE180934B12CF010E94DF
:108F3000E9AF8BE79EE00E94DCAF8091471285315C
:108F400008F460C2809147128C3130F5809149124B
:108F5000843110F18091730D9091740D019644E667
:108F6000489F9001499F300D112437FF02C02150C6
:108F70003F4F832F932F990F990B009769F028E6A5
:108F800020934A122BE120934B120E94599B0E947E
:108F9000E9AF85E20E9488B580915611882349F097
:108FA00080914712843328F4809149128A3208F064
:108FB0005DC280914712853328F480914912813334
:108FC00008F07AC260919C03623048F080914712A9
:108FD000843328F480914912823308F072C2809160
:108FE0004712813308F060C080914912893208F439
:108FF0005BC00E941DB12B013C018CE3C82ED12C1B
:10900000E12CF12CC301B201A70196010F941E358A
:10901000CA01B901A70196010F941E35CA01F62EA7
:10902000E72E69018E010F5F1F4F40E8441641E5AE
:10903000540641E06406710408F45EC2B90128E1F7
:1090400030E040E050E00F941E3529013A01EF92E4
:10905000FF92C60168E170E00F9444389F938F93AC
:109060005F924F9284E499E09F938F931F930F93A5
:109070000F94AB300FB6F894DEBF0FBECDBF9AE0B1
:10908000491651046104710408F060C298E0892F08
:10909000880F980F9195955A90934A1280E3809388
:1090A0004B12C8010E94E9AFE0910D12F0910E122F
:1090B000848181112FC120917816309179164091C9
:1090C0007A1650917B1660916612709167128091AA
:1090D0006812909169120F947C356B017C0120E03D
:1090E00030E0A9010F94123187FD05C020E030E087
:1090F00040E05FE304C020E030E040E05FEBC70108
:10910000B6010F947C350F94C036CB010E94C69AED
:10911000BC0184ED93E00F94BA3820917C16309115
:109120007D1640917E1650917F1660916A12709163
:109130006B1280916C1290916D120F947C356B01C3
:109140007C0120E030E0A9010F94123187FD05C0B9
:1091500020E030E040E05FE304C020E030E040E0A9
:109160005FEBC701B6010F947C350F94C036CB017D
:109170000E94C69ABC018FEC93E00F94BA382091FC
:10918000801630918116409182165091831660911D
:109190006E1270916F1280917012909171120F94F3
:1091A0007C356B017C0120E030E04AE754E40F9409
:1091B00077312B013C0120E030E0A901C701B60165
:1091C0000F94123187FD05C020E030E040EA50E402
:1091D00004C020E030E040EA50ECC301B2010F943B
:1091E0007C3520E030E040E251E40F9458360F9493
:1091F000C0366B017C0197FD16C06031F7E27F0736
:1092000081059105D4F020E137E240E050E00F9471
:109210004035CA01B9012AE030E040E050E00F9447
:109220004035605D0BC0F094E094D094C094C11CB4
:10923000D11CE11CF11C6DE201C060E260934C0B9B
:1092400028EEC21623E0D206E104F10494F0C7012F
:10925000B60128EE33E040E050E00F944035CA01FB
:10926000B9012AE030E040E050E00F944035605D05
:1092700001C060E260934D0BC701B60124E630E007
:1092800040E050E00F9440359AE0492E512C612C7B
:10929000712CCA01B901A30192010F944035605DA0
:1092A00060934E0BC701B601A30192010F944035A4
:1092B0006B017C01672B682B692B79F08EE2809320
:1092C0004F0BCA01B901A30192010F944035605DB3
:1092D0006093500B80E38C0D15C0CA01B901A30146
:1092E00092010F944035662339F08EE280934F0B44
:1092F000605D6093500B05C080E28093500B8093BB
:109300004F0B80E28093510B6CE47BE088EC93E0A0
:109310000F94BA38809147128632A8F4809149128E
:109320008E3188F008E020E84EE160E083E192E1D0
:109330000E94A59180914712863228F480914912AB
:109340008F3108F005C180914712823328F4809153
:1093500049128C3208F08FC1809147128F3308F088
:10936000A9C180914912883308F4A4C110924A120D
:109370008EE380934B1280EA9EE00E94BDD5182FA9
:109380000E94A9B5163108F095C180E20E9488B507
:109390001F5FF8CF93E053CD80914912813118F4CB
:1093A00061CD90E04CCD6091711670917216072ED0
:1093B000000C880B990B0F94183120916B1630918B
:1093C0006C1640916D1650916E160F94A2371816B8
:1093D00074F41092331202E022E041E16DE083E187
:1093E00092E10E94A59181E0809333123BCD02E08F
:1093F00022E041E16DE083E192E10E94A59132CD4E
:1094000093E08DCD80914912813118F49BCD90E08D
:1094100086CD6091120B7091130B072E000C880BF8
:10942000990B0F94183120910E0B30910F0B409136
:10943000100B5091110B0F94A237181674F4109260
:10944000331202E022E042E168E583E192E10E940A
:10945000A59181E08093331275CD02E022E042E1D4
:1094600068E583E192E10E94A5916CCD07E028E0D8
:109470004AE26AE283E192E10E94A59105E022E0DE
:109480004CE262E383E192E10E94A5916AE08AE204
:109490000E94DCB4609115127091161282E38093E1
:1094A0002F128BE2809330122FE232E142E383E10C
:1094B00092E10E94E38F7DCD6AE486E30E94DCB4F2
:1094C00081CDF8E46F9FB0011124072E000C880BAA
:1094D000990B0F9418312AE037ED43E25CE30F94C7
:1094E00077310F94C536262F02E042E367E383E12C
:1094F00092E10E94A59173CDE4E6CE16D10498F4D2
:10950000EF92FF923F932F938AE399E09F938F937B
:109510001F930F930F94AB300FB6F894DEBF0FBEBE
:10952000CDBF95E0B4CDEF92FF923F932F9382E3AE
:1095300099E09F938F931F930F930F94AB300FB6C7
:10954000F894DEBF0FBECDBF96E0A1CD99E09FCDD0
:109550001092331283E080934A1215E210934B125B
:1095600089E79EE00E94DCAF8BE080934A12109363
:109570004B12BB2029F084ED93E00E94E9AF19C0A3
:109580008091E21480FD0DC004ED13E0F80181919B
:109590008F01882371F08F3208F08FE30E94CBAFE8
:1095A000F5CF80917B0B80FDE6CF84E79EE00E94A3
:1095B000DCAF8BE280934A1215E210934B1282E7E4
:1095C0009EE00E94DCAF83E380934A1210934B121B
:1095D000BB2029F08FEC93E00E94E9AF19C0809185
:1095E000E21481FD0DC00FEC13E0F80181918F01B1
:1095F000882371F08F3208F08FE30E94CBAFF5CF54
:1096000080917B0B81FDE6CF84E79EE00E94DCAF7A
:1096100083E580934A1215E210934B1280E79EE097
:109620000E94DCAF8BE580934A1210934B12BB2053
:1096300029F088EC93E00E94E9AF19C08091E21410
:1096400082FD0DC008EC13E0F80181918F018823A1
:1096500071F08F3208F08FE30E94CBAFF5CF80918D
:109660007B0B82FDE6CF89E69EE00E94DCAF81E0C5
:109670008093331268CE84E00E949EAF83E0809393
:109680004A1212E310934B1286E00E94CBAF0E9465
:10969000006F8CE080934A1210934B12809100026D
:1096A000909101020E94599B0E94E9AF85E20E94BD
:1096B00088B552CE2A960FB6F894DEBF0FBECDBF46
:1096C000DF91CF911F910F91FF90EF90DF90CF909E
:1096D000BF907F906F905F904F900895282F1092C9
:1096E0002C0A80919C0E90919D0EA0919E0EB0919F
:1096F0009F0E81309048A105B10540F010929C0E5C
:1097000010929D0E10929E0E10929F0E8091210A33
:10971000882331F080919C0E80934E121092990E06
:1097200080914F121816FCF4082E000C990B821B26
:10973000910920914E12022E000C330B2817390785
:1097400094F097FF02C080E090E080934E12092EC3
:10975000000CAA0BBB0B80939C0E90939D0EA093C4
:109760009E0EB0939F0E80914E126623A9F09091A9
:109770005012891714F48093501220915012022E27
:10978000000C330B2C5F3F4F482F082E000C550B5D
:10979000241735071CF4845080935012089580914B
:1097A0009A0E8630D8F496E0899FF0011124EC558A
:1097B000FC4F209146023091470231832083409133
:1097C0009C0E50919D0E60919E0E70919F0E428353
:1097D0005383648375838F5F80939A0E089585E029
:1097E00096E40C94EDB5E0919A0EEE2369F0E15009
:1097F000E0939A0E86E0E89FF0011124EC55FC4FAF
:10980000808191810C94EDB5EACFAF92BF92CF9257
:10981000DF92EF92FF920F931F93CF93DF935C0140
:109820006B010E94AA75EC01C6010E94BDD504E13E
:1098300010E0081B1109DD270C171D071CF0FF2481
:10984000F39402C082E0F82E8091141290E06F2D04
:1098500070E06F5F7F4F0F945838E62EC6E0C60F5A
:1098600080914712C81750F04091491250E02C2FB8
:1098700030E02B503109421753079CF5D0E0C1145A
:10988000D104C1F18AE30E9488B582E0F8120FC0CA
:10989000CE0D80914712C81768F12091491230E02F
:1098A0008C2F90E00B97281739071CF423C0DD2379
:1098B00009F1902F990F090F000F00934A12C093DE
:1098C0004B1280E20E9488B5C601DF91CF911F91B3
:1098D0000F91FF90EF90DF90CF90BF90AF900C94DE
:1098E000E9AF10924A12C0934B12C5010E9493B582
:1098F000D1E0C5CFDF91CF911F910F91FF90EF90F5
:10990000DF90CF90BF90AF9008950F934CE0849F6D
:10991000402D112421E0240F20939F128CE0840F0E
:109920008093A012E0914712F0E090E002968E172B
:109930009F070CF1822F90E02091491230E08217AE
:109940009307CCF4662371F081E0809333124D5F6E
:109950000BE020E860E083E192E10E94A591109283
:10996000331203C081E0809333128091A0121092D1
:109970004A1280934B120F910895CF92DF92EF928B
:10998000FF920F93CF93DF93982F862F6A0179016F
:10999000692FBBDF909147128091A012891708F4BC
:1099A00048C09091491280919F12981708F441C0C5
:1099B000002321F0C7010E94AA7503C0C7010E94BD
:1099C000BDD5D82FC4E1C81BF6018491882339F096
:1099D0000E94B7AFC81BFFEFCF1ADF0AF5CF8AE3AB
:1099E0000E9488B5CC2329F080E20E9488B5C1503E
:1099F000F9CF8091A0129AEFD99FD02D1124D05881
:109A0000D0934A1280934B12C701002349F0DF9193
:109A1000CF910F91FF90EF90DF90CF900C94DCAF3F
:109A2000DF91CF910F91FF90EF90DF90CF900C944A
:109A3000E9AFDF91CF910F91FF90EF90DF90CF9042
:109A40000895CF92DF92EF92FF920F93CF93DF931F
:109A5000CDB7DEB7E989FA89C080D180E280F38092
:109A600020E030E0A901C701B6010F94123187FD53
:109A700005C020E030E040E05FE304C020E030E0DB
:109A800040E05FEBC701B6010F947C350F94C03600
:109A9000CB010E94599B00E09C014D855E856C8541
:109AA0008B856BDFDF91CF910F91FF90EF90DF906F
:109AB000CF900895DF92EF92FF920F931F93CF9371
:109AC000DF931F92CDB7DEB77B01622F49831DDF85
:109AD000909147128091A0124981891708F44CC0D7
:109AE0009091491280919F12981708F445C0442321
:109AF00059F10115110541F5C7010E94AA7526E12A
:109B000030E0281B390B37FF02C02F5F3F4F3595E0
:109B1000279536E1D32E2751822F8D0D87FD11C059
:109B200080E229830E9488B5DA942981F5CFF70174
:109B30008491882361F00E94B7AFD81A8FEFE81A9A
:109B4000F80A1D14A4F303C086E1D82EFACF01153C
:109B5000110559F01D144CF4F80181918F018823EF
:109B600021F00E94B7AFD81AF5CF1D142CF480E273
:109B70000E9488B5DA94F9CF0F90DF91CF911F91B1
:109B80000F91FF90EF90DF9008952F923F924F92A8
:109B90005F926F927F928F929F92AF92BF92CF927D
:109BA000DF92EF92FF920F931F93CF93DF93CDB786
:109BB000DEB7CC57D1090FB6F894DEBF0FBECDBFCC
:109BC000E091EB03F091EC03EF2B11F00C94635751
:109BD0006C96DFAECEAE6C972996EFAE29977901E1
:109BE0006A015B01FC012081318142815381A6968B
:109BF0002CAF3DAF4EAF5FAFA69720918A12309148
:109C00008B1240918C1250918D12A6966CAD7DAD49
:109C10008EAD9FADA6970F9477310F94AD37E29636
:109C20006CAF7DAF8EAF9FAFE297D5018D919D91C7
:109C30000D90BC91A02DAA968CAF9DAFAEAFBFAFDB
:109C4000AA9720918E1230918F12409190125091CC
:109C50009112BC01CD010F9477310F94AD37E69688
:109C60006CAF7DAF8EAF9FAFE697D6012D913D9142
:109C70004D915C91AE962CAF3DAF4EAF5FAFAE97BE
:109C8000209192123091931240919412509195121A
:109C9000AE966CAD7DAD8EAD9FADAE970F94773126
:109CA0000F94AD37EA966CAF7DAF8EAF9FAFEA975A
:109CB000D7012D913D914D915C916A962CAF3DAFAE
:109CC0004EAF5FAF6A9720919612309197124091F4
:109CD0009812509199126A966CAD7DAD8EAD9FAD84
:109CE0006A970F9477310F94AD37A0966CAF7DAF24
:109CF0008EAF9FAFA0978091731683FF1CC0A09674
:109D00002CAD3DAD4EAD5FADA0972093100F3093BD
:109D1000110F4093120F5093130F6A968CAD9DADA7
:109D2000AEADBFAD6A978093000F9093010FA093E3
:109D3000020FB093030FD801BC91BBABF801F181C6
:109D4000F8AFD8011296BC91BCAFF801F3812D9603
:109D5000FFAF2D978091BA0E9091BB0E891B8F702B
:109D60008F3021F480E00F94FA20F4CF0091BA0EE6
:109D7000EB960FAFEB978091BA0E282E312C809185
:109D8000040F9091050FA091060FB091070FE29676
:109D90008CAC9DACAEACBFACE297881A990AAA0A0B
:109DA000BB0A8091080F9091090FA0910A0FB09102
:109DB0000B0FE6964CAC5DAC6EAC7FACE697481AE8
:109DC000590A6A0A7B0A80910C0F90910D0FA0919D
:109DD0000E0FB0910F0FEA962CAD3DAD4EAD5FADBD
:109DE000EA97281B390B4A0B5B0B2BA33CA34DA313
:109DF0005EA38091100F9091110FA091120FB0915E
:109E0000130FA0960CAD1DAD2EAD3FADA097081B56
:109E1000190B2A0B3B0B0FA318A729A73AA7012B55
:109E2000022B032B09F4BDC060916B1670916C1668
:109E300080916D1690916E1620917016211141C07F
:109E40000F94C03620915E0230915F026217730753
:109E5000C4F5A0962CAD3DAD4EAD5FADA09720935F
:109E6000100F3093110F4093120F5093130F6A96F7
:109E70008CAD9DADAEADBFAD6A978093000F909352
:109E8000010FA093020FB093030FEDE9F2E4849168
:109E90008F010F5F1F4F882321F00F943D27F8019A
:109EA000F6CFE7EDF0E184918F010F5F1F4F88231C
:109EB00021F00F943D27F801F6CF1FA218A619A68E
:109EC0001AA66FA178A589A59AA50F94183129968D
:109ED0000FAD2997A4E00A9FF0011124EA5FFD4F1E
:109EE00020813181428153810F9477316B017C0154
:109EF00020E030E0A9010F94A23787FF04C0F7FAF1
:109F0000F094F7F8F0946091961270919712809106
:109F10009812909199120F94C0369B01AC01A8EC55
:109F2000B0E00F945C350F9418319B01AC01C70170
:109F3000B6010F94A2371816C4F5A0962CAD3DAD0E
:109F40004EAD5FADA0972093100F3093110F40934B
:109F5000120F5093130F6A968CAD9DADAEADBFAD91
:109F60006A978093000F9093010FA093020FB09314
:109F7000030FEDE9F2E484918F010F5F1F4F8823F7
:109F800021F00F943D27F801F6CFE8EBF0E1849142
:109F90008F010F5F1F4F882321F00F943D27F80199
:109FA000F6CF1FA218A619A61AA6D501C4018827A4
:109FB000B7FD83959927AA27BB27182F77FC126036
:109FC0002BA13CA14DA15EA157FD14608FA198A5C6
:109FD000A9A5BAA5B7FD18606FA178A589A59AA50E
:109FE0000F94183129960FAD2997A4E00A9FF0012C
:109FF0001124EA5FFD4F20813181428153810F940A
:10A0000077316B017C0120E030E0A9010F94A23789
:10A0100087FF04C0C701B601905802C0C701B6014E
:10A0200020E030E040E05FE30F947C350F94C536CC
:10A030006CAB7DAB8EAB9FAB8AE5829DF001839DBF
:10A04000F00D1124EB5EFB4F108216AB24968CAE04
:10A050009DAEAEAEBFAE2497B7FE0DC0222733270C
:10A06000A901281939094A095B0924962CAF3DAF8B
:10A070004EAF5FAF24978AE5829DF001839DF00D7E
:10A080001124EB5EFB4F24968CAD9DADAEADBFAD04
:10A090002497858B968BA78BB08F62964CAE5DAE66
:10A0A0006EAE7FAE629777FE0DC022273327A901DF
:10A0B000241935094609570962962CAF3DAF4EAFBA
:10A0C0005FAF62978AE5829DF001839DF00D1124B8
:10A0D000EB5EFB4F62968CAD9DADAEADBFAD6297B2
:10A0E000818F928FA38FB48F2BA13CA14DA15EA134
:10A0F00028962CAF3DAF4EAF5FAF289757FF0DC0EE
:10A1000050954095309521953F4F4F4F5F4F289682
:10A110002CAF3DAF4EAF5FAF28978AE5829DF0012F
:10A12000839DF00D1124EB5EFB4F28968CAD9DAD09
:10A13000AEADBFAD2897858F968FA78FB0A3C50111
:10A14000B4010F9418312091010430910204409120
:10A150000304509104040F9477316BA77CA78DA75B
:10A160009EA7698B7A8B8B8B9C8BC301B2010F945A
:10A170001831209105043091060440910704509154
:10A1800008040F9477316FA778AB89AB9AAB6D8BCE
:10A190007E8B8F8B988F2091090430910A04409117
:10A1A0000B0450910C0466962CAF3DAF4EAF5FAFE1
:10A1B00066976BA17CA18DA19EA10F941831669624
:10A1C0002CAD3DAD4EAD5FAD66970F9477314B0131
:10A1D0005C01698F7A8F8B8F9C8F20910D04309159
:10A1E0000E0440910F0450911004C701B6010F9462
:10A1F00077316B017C016D8F7E8F8F8F98A32496B2
:10A200008CAD9DADAEADBFAD24970697A105B10550
:10A210007CF562962CAD3DAD4EAD5FAD62972630BC
:10A2200031054105510524F528968CAD9DADAEADA7
:10A23000BFAD28970697A105B105D4F420E030E022
:10A24000A901C701B6010F94A23787FF04C0F7FA2E
:10A25000F094F7F8F0948AE5829DF001839DF00D6B
:10A260001124EB5EFB4FC586D686E786F08AA1C136
:10A270006C96AEADBFAD6C97CD90DD90ED90FC903F
:10A2800020E030E0A901C701B6010F941231882304
:10A2900069F08AE5829DF001839DF00D1124EB5E4B
:10A2A000FB4FC586D686E786F08A34C02BA53CA531
:10A2B0004DA55EA5CA01B9010F9477316B017C01F0
:10A2C0002FA538A949A95AA9CA01B9010F94773114
:10A2D0009B01AC01C701B6010F947C356B017C0179
:10A2E000A5019401C501B4010F9477319B01AC0124
:10A2F000C701B6010F947C350F94E7372AE5229DFC
:10A30000F001239DF00D1124EB5EFB4F65877687EE
:10A310008787908B80913515882309F44AC1C090B6
:10A32000E203D090E303E090E403F090E50320E043
:10A3300030E0A901C701B6010F941231882309F456
:10A3400038C18090DE039090DF03A090E003B090CE
:10A35000E10320E030E0A901C501B4010F941231FE
:10A36000882309F426C12BA13CA14DA15EA1211592
:10A3700031054105510509F41CC157FD0BC080E0B2
:10A3800090E0A0E8BFE324968CAF9DAFAEAFBFAF27
:10A3900024970AC020E030E040E85FEB24962CAF21
:10A3A0003DAF4EAF5FAF249712FB112710F980919C
:10A3B000DD038117B1F11093DD036091D903709132
:10A3C000DA038091DB039091DC030F9418312B01A9
:10A3D0003C01A501940124966CAD7DAD8EAD9FAD81
:10A3E00024970F947731A70196010F94773120912C
:10A3F00092123091931240919412509195120F94B1
:10A4000077319B01AC01C301B2010F947C350F94ED
:10A41000C0366093D9037093DA038093DB03909383
:10A42000DC034090D9035090DA036090DB03709016
:10A43000DC038BA19CA1ADA1BEA1181619061A06BA
:10A440001B0634F414141504160417041CF0B1C0D0
:10A4500077FEAFC0C301B2010F9418314B015C010C
:10A460008AE5829DF001839DF00D1124EB5EFB4F88
:10A4700020910202309103024091040250910502A2
:10A4800065857685878590890F9458366B017C01A8
:10A4900020E030E040E85FE30F94A237181634F470
:10A4A000C12CD12C30E8E32E3FE3F32EA701960117
:10A4B000C501B4010F9477310F94C0366B017C0154
:10A4C000DC01CB01F7FE07C088279927DC018C1936
:10A4D0009D09AE09BF0928960CAD1DAD2EAD3FAD4F
:10A4E0002897080F191F2A1F3B1FC901B8012AE529
:10A4F000229D8001239D100D11240B5E1B4FD8015E
:10A500005D966D937D938D939C9390974C185D0809
:10A510006E087F084092D9035092DA036092DB0301
:10A520007092DC030F9416319B01AC0124966CAD44
:10A530007DAD8EAD9FAD24970F94773166962CAD8F
:10A540003DAD4EAD5FAD66970F9477316B017C01E9
:10A55000698F7A8F8B8F9C8F2BA53CA54DA55EA50F
:10A56000CA01B9010F9477314B015C012FA538A9BD
:10A5700049A95AA9CA01B9010F9477319B01AC01CD
:10A58000C501B4010F947C354B015C01A701960114
:10A59000C701B6010F9477319B01AC01C501B4012D
:10A5A0000F947C350F94E737F801658776878787A6
:10A5B000908B8AE5829DF001839DF00D1124EB5E66
:10A5C000FB4F0CA91DA92EA93FA901A312A323A3E8
:10A5D00034A3458956896789708D058D168D278D21
:10A5E00030A1818D928DA38DB48D80179107A20724
:10A5F000B30710F4D901C80184179507A607B70758
:10A6000010F4DB01CA010CA91DA92EA93FA98017CE
:10A610009107A207B30710F4D901C8012AE5229DCA
:10A62000F001239DF00D1124EB5EFB4F85A396A353
:10A63000A7A3B0A70697A105B10508F43DC4DF01A3
:10A64000AE5ABF4F8091730D9091740D11969C93EB
:10A650008E9312968091750D9091760D8D939C93AB
:10A6600029961FAD299711A7452B462B472B09F09B
:10A6700017988AE5829DF001839DF00D1124EB5E11
:10A68000FB4F818D928DA38DB48D892B8A2B8B2BC3
:10A6900009F016988AE5829DF001839DF00D112442
:10A6A000EB5EFB4F858D968DA78DB0A1892B8A2BF4
:10A6B0008B2B09F015982CA93DA94EA95FA9232B36
:10A6C000242B252B09F401C48091EA03882319F077
:10A6D00081508093EA0329960FAD2997011104C098
:10A6E000149880E28093EA03E0904A15F0904B15AD
:10A6F00000914C1510914D159701A8016BA978ADEB
:10A700008CAD2D969FAD2D970F94123187FF06C00B
:10A71000EBAAF8AE0CAF2D961FAF2D978AE5829D60
:10A72000F001839DF00D1124EB5EFB4F25853685EE
:10A730004785508960E070E080E89FE30F945836C9
:10A7400024966CAF7DAF8EAF9FAF24979B01AC0179
:10A750006BA978AD8CAD2D969FAD2D970F94773169
:10A760004B015C018091BA0E9091B80E891B8F70DD
:10A7700025968FAF2597A501940160E074E284E7E8
:10A7800099E40F9458360F94AD376B017C012596F0
:10A790008FAD25978250863008F4A0C380916F005A
:10A7A00081FB222720F981FF05C080916F008D7FFA
:10A7B00080936F008091110490911204A091130472
:10A7C000B0911404C80ED91EEA1EFB1EC0921104DB
:10A7D000D0921204E0921304F0921404222329F080
:10A7E00080916F00826080936F008AE5829D800176
:10A7F000839D100D11240B5E1B4FD8011D962D91CA
:10A800003D914D915C915097C501B4010F94773102
:10A810009B01AC010F94773162966CAF7DAF8EAF28
:10A820009FAF6297F801618372838383948325A12C
:10A8300036A147A150A528AF39AF4AAF5BAFCA01D7
:10A84000B9010F9416316CAF7DAF8EAF9FAFA501EC
:10A8500094010F9477310F9442360F94C536669663
:10A860006CAF7DAF8EAF9FAF6697F801EE5BFF4F89
:10A8700060837183828393838E010F5E1F4F2A96BC
:10A880001FAF0EAF2A97005111092E961FAF0EAFC2
:10A890002E970EE615E1A2961FAF0EAFA2978E017E
:10A8A0000F5D1F4F1AA309A32E960EAD1FAD2E9755
:10A8B0006C961FAF0EAF6C971BA21BA610E81FA7CC
:10A8C0000FE30BAB2A96AEADBFAD2A976D917D918C
:10A8D0008D919D912A96BFAFAEAF2A97A5019401A5
:10A8E0000F9477316B017C016C96EEADFFAD6C97E8
:10A8F00061937193819391936C96FFAFEEAF6C97D8
:10A9000020E030E0A9010F94A23787FF04C0F7FAD6
:10A91000F094F7F8F094A296AEADBFADA2974D902B
:10A920005D906D907D90A296BFAFAEAFA297A30150
:10A930009201C701B6010F94A23718160CF40AC38E
:10A940002A960EAD1FAD2A9729A13AA10217130727
:10A9500009F0B8CF20E030E040E85FE36BA17BA5D1
:10A960008FA59BA90F94123187FF57C07E0131E15B
:10A97000E30EF11C2E960EAD1FAD2E972BA13BA51D
:10A980004FA55BA9D8016D917D918D919C910F94FC
:10A990007731F80161937193819391938F01EE1553
:10A9A000FF0561F72AE5229DC001239D900D11242A
:10A9B0008C010B5E1B4F78010E5B1F4F66966CADD2
:10A9C0007DAD8EAD9FAD66970F9416312BA13BA543
:10A9D0004FA55BA90F9477310F94C536D8016D93BD
:10A9E0007D938D939C9313972BA13BA54FA55BA9BA
:10A9F0006BA17BA58FA59BA90F9477319B01AC011F
:10AA000062966CAD7DAD8EAD9FAD62970F94773140
:10AA1000F701618372838383948324962CAD3DADCB
:10AA20004EAD5FAD24976CAD7DAD8EAD9FAD0F94F7
:10AA300077316BA37CA38DA39EA38AE5829D8001C1
:10AA4000839D100D11240B5E1B4FD80155968D90E0
:10AA50009D90AD90BC90589781149104A104B104CD
:10AA600009F090C259968D919D910D90BC91A02DA9
:10AA7000892B8A2B8B2B09F085C2F801858D968D49
:10AA8000A78DB0A1892B8A2B8B2B09F07BC220913B
:10AA900056153091571540915815509159156BA185
:10AAA0007CA18DA19EA10F9477310F9442360F9413
:10AAB000C5362B013C01D801D7961C928AE5829DB0
:10AAC0008001839D100D11240B5E1B4FF801E25B8A
:10AAD000FF4F4082518262827382C301B2010F94A0
:10AAE00016316B017C012BA13CA14DA15EA10F94FD
:10AAF00058362C966CAF7DAF8EAF9FAF2C97D80198
:10AB000051966D937D938D939C9354972DEB37E3E2
:10AB100046E051E4C701B6010F9477310F94C53672
:10AB2000F80162AB73AB84AB95AB87A9882381F145
:10AB3000FE96208131814281538160910D15709183
:10AB40000E1580910F15909110150F9477312C965A
:10AB50002CAD3DAD4EAD5FAD2C970F94773120916C
:10AB600096123091971240919812509199120F9429
:10AB700077319B01AC0160E074E284EF99E40F94BB
:10AB800058360F94C536D801D9967C936E93D897D2
:10AB90008AE5829DF001839DF00D1124EB5EFB4F51
:10ABA000018112812381348124960CAF1DAF2EAF19
:10ABB0003FAF2497C901B8010F94E737162F072F2D
:10ABC0008BA39FA326E335E160963FAF2EAF60973E
:10ABD0003E0131E1630E711C46E355E15DAF4CAFC0
:10ABE0002E964EAC5FAC2E976BA77FA78BAB9CAB22
:10ABF00018AED201CD90DD90ED90FD902D0120E0BA
:10AC000030E0A901C701B6010F94A23787FF04C045
:10AC1000F7FAF094F7F8F094ECADFDAD81909190D7
:10AC2000A190B190FDAFECAFA5019401C701B601B1
:10AC30000F94A23718160CF4B2C446145704C9F680
:10AC40005BA56B965FAF6B978FA5A1968FAFA19712
:10AC50009BA9EC969FAFEC97ACA9ED96AFAFED97A3
:10AC60002596BFAD2597B111DAC46B968FAD6B9762
:10AC7000A1969FADA197EC96AFADEC97ED96BFADC9
:10AC8000ED978093E6039093E703A093E803B093D6
:10AC9000E9038AE5829D8001839D100D11240B5EDE
:10ACA0001B4F2BA53FA54BA95CA96BA57FA58BA925
:10ACB0009CA90F947731D80119966D937D938D934C
:10ACC0009C931C972C966CAD7DAD8EAD9FAD2C9753
:10ACD00090589B01AC010F947C35F8012585368591
:10ACE000478550890F9477319B01AC016BE077ED7C
:10ACF00083E29BE30F947B359B01AC018BE097EDE6
:10AD0000A3E2BBE3F80185839683A783B087108114
:10AD100024966CAD7DAD8EAD9FAD24970F9412310E
:10AD200018160CF0BCC581E0182B8AE5829DF00155
:10AD3000839DF00D1124EB5EFB4F108380E1FE013B
:10AD40003196A4EEBEE001900D928A95E1F724962B
:10AD50000CAD1DAD2EAD3FAD24970093E00E1093CA
:10AD6000E10E2093E20E3093E30EE2962CAD3DAD62
:10AD70004EAD5FADE2972093040F3093050F4093E3
:10AD8000060F5093070FE6968CAD9DADAEADBFADEF
:10AD9000E6978093080F9093090FA0930A0FB09342
:10ADA0000B0FEA960CAD1DAD2EAD3FADEA970093AB
:10ADB0000C0F10930D0F20930E0F30930F0FA096D2
:10ADC0002CAD3DAD4EAD5FADA0972093100F3093ED
:10ADD000110F4093120F5093130FA6968CAD9DAD9B
:10ADE000AEADBFADA6978093F40E9093F50EA093F1
:10ADF000F60EB093F70EAA960CAD1DAD2EAD3FAD7D
:10AE0000AA970093F80E1093F90E2093FA0E309340
:10AE1000FB0EAE962CAD3DAD4EAD5FADAE97209323
:10AE2000FC0E3093FD0E4093FE0E5093FF0E6A967B
:10AE30008CAD9DADAEADBFAD6A978093000F909382
:10AE4000010FA093020FB093030F9091BA0E80915F
:10AE5000BB0E981303C084E68093B70EEB968FADBC
:10AE6000EB978F5F8F708093BA0E8091BA0E90919E
:10AE7000B90E81508F70891314C50091BB0E0BA3BE
:10AE80001091BA0E1FA39AE50FA11BA1011391C542
:10AE9000812C912CA12CB12C1BA61FA61BAA1CAA8D
:10AEA000212C312C00E010E0FBA12FA1F2138EC564
:10AEB0002114310409F03EC680916F0082608093B6
:10AEC0006F0081E099C780E097C7E0904615F09049
:10AED000471500914815109149150ECC80914E15DB
:10AEE00090914F15A0915015B0915115C816D906E3
:10AEF000EA06FB0608F052CC8C199D09AE09BF0981
:10AF0000BC01CD01660F771F881F991F25964FAD95
:10AF10002597042F10E020E030E0A90198010F945C
:10AF20001E35CA01B9010F9416310F94AD37C60E04
:10AF3000D71EE81EF91EC701B6010F9416319B01FA
:10AF4000AC0160E074E284E799E40F9458364B0159
:10AF50005C0124CCA7019601C301B2010F945836BD
:10AF60007B018C019B01AC016BA17BA58FA59BA9EB
:10AF70000F94A23718160CF0E3CCEBA2FBA60FA798
:10AF80001BABDECC0CA91DA92EA93FA9012B022BBE
:10AF9000032B49F060915A1570915B1580915C15F7
:10AFA00090915D1508C06091521570915315809174
:10AFB0005415909155152BA13CA14DA15EA10F9464
:10AFC00077310F9442360F94C5362B013C012CA9E2
:10AFD0003DA94EA95FA9232B242B252BC9F020E0E6
:10AFE00030E0A90160910D1570910E1580910F153B
:10AFF000909110150F941231882351F081E00FA128
:10B0000018A529A53AA510161106120613060CF06C
:10B0100080E09AE5929D8001939D100D11240B5EB6
:10B020001B4FD801D7968C93882309F4BAC020917E
:10B03000F40E3091F50E4091F60E5091F70EA69653
:10B040006CAD7DAD8EAD9FADA6970F947B356FA394
:10B0500078A789A79AA72091F80E3091F90E409110
:10B06000FA0E5091FB0EAA966CAD7DAD8EAD9FADE4
:10B07000AA970F947B356BA77CA78DA79EA72091DD
:10B08000FC0E3091FD0E4091FE0E5091FF0EAE96DB
:10B090006CAD7DAD8EAD9FADAE970F947B356B01E2
:10B0A0007C012FA138A549A55AA5CA01B9010F9461
:10B0B00077316FA378A789A79AA72BA53CA54DA5A3
:10B0C0005EA5CA01B9010F9477319B01AC016FA154
:10B0D00078A589A59AA50F947C356FA378A789A731
:10B0E0009AA7A7019601C701B6010F9477319B017A
:10B0F000AC016FA178A589A59AA50F947C350F9412
:10B10000E7376B017C012091000F3091010F4091D6
:10B11000020F5091030F6A966CAD7DAD8EAD9FAD61
:10B120006A970F947B35A70196010F9458366B01EF
:10B130007C01F801FE96608371838283938320E013
:10B1400030E040E450E40F94A23718161CF4F801E4
:10B1500017AA27C020910D1530910E1540910F159B
:10B1600050911015C701B6010F9477319B01AC01C6
:10B170006091421570914315809144159091451549
:10B180000F9458362BA13CA14DA15EA10F947731AD
:10B190000F94C536641575058605970510F42B01C7
:10B1A0003C018091ED039091EE03A091EF03B091EB
:10B1B000F00308AD19AD2AAD3BAD80179107A2078A
:10B1C000B30708F4DCC081149104A104B10441F177
:10B1D0002091F1033091F2034091F3035091F40375
:10B1E0002415350546055705D8F468AD79AD8AAD07
:10B1F0009BAD0F940F356B017C01A3019201C5013A
:10B20000B4010F940F35C616D706E806F90640F4C8
:10B21000C701B601A50194010F941E3529013A0119
:10B220008AE5829DF001839DF00D1124EB5EFB4FBA
:10B23000C18CD28CE38CF48CC114D104E104F104F0
:10B2400041F12091F5033091F6034091F7035091BD
:10B25000F8032415350546055705D8F468AD79ADD2
:10B260008AAD9BAD0F940F354B015C01A301920198
:10B27000C701B6010F940F3586169706A806B906C2
:10B2800040F4C501B401A70196010F941E352901B0
:10B290003A018AE5829DF001839DF00D1124EB5E59
:10B2A000FB4FC58CD68CE78CF0A0C114D104E1040F
:10B2B000F10441F12091F9033091FA034091FB032D
:10B2C0005091FC032415350546055705D8F468ADA3
:10B2D00079AD8AAD9BAD0F940F354B015C01A30195
:10B2E0009201C701B6010F940F3586169706A8067E
:10B2F000B90640F4C501B401A70196010F941E35AB
:10B3000029013A018AE5829DF001839DF00D112407
:10B31000EB5EFB4FC1A0D2A0E3A0F4A0C114D10406
:10B32000E104F10409F4CACB2091FD033091FE033E
:10B330004091FF035091000424153505460557053B
:10B3400008F0BCCB68AD79AD8AAD9BAD0F940F35DD
:10B350004B015C01A3019201C701B6010F940F35A7
:10B3600086169706A806B90608F0A8CBC501B40151
:10B37000A70196010F941E3529013A019FCB811434
:10B380009104A104B104A9F16091F1037091F20359
:10B390008091F3039091F403641575058605970574
:10B3A00040F50F9416312CAD3DAD4EAD5FAD0F9411
:10B3B00077316B017C01C501B4010F9416314B014B
:10B3C0005C01C301B2010F941631A50194010F94E1
:10B3D0007731A70196010F94A237181654F4A501EE
:10B3E0009401C701B6010F9458360F94C5362B014E
:10B3F0003C018AE5829DF001839DF00D1124EB5EF6
:10B40000FB4F818C928CA38CB48C81149104A10489
:10B41000B104A9F16091F5037091F6038091F703EF
:10B420009091F803641575058605970540F50F940E
:10B4300016312CAD3DAD4EAD5FAD0F9477316B0144
:10B440007C01C501B4010F9416314B015C01C301AD
:10B45000B2010F941631A50194010F947731A70121
:10B4600096010F94A237181654F4A5019401C70150
:10B47000B6010F9458360F94C5362B013C018AE56E
:10B48000829DF001839DF00D1124EB5EFB4F858CB6
:10B49000968CA78CB0A081149104A104B104A9F1E9
:10B4A0006091F9037091FA038091FB039091FC0382
:10B4B000641575058605970540F50F9416312CAD7A
:10B4C0003DAD4EAD5FAD0F9477316B017C01C50191
:10B4D000B4010F9416314B015C01C301B2010F940A
:10B4E0001631A50194010F947731A70196010F94AD
:10B4F000A237181654F4A5019401C701B6010F94A0
:10B5000058360F94C5362B013C018AE5829DF00127
:10B51000839DF00D1124EB5EFB4FC1A0D2A0E3A0F0
:10B52000F4A0C114D104E104F10409F4C7CA609184
:10B53000FD037091FE038091FF0390910004641558
:10B5400075058605970508F0B9CA0F9416312CAD1C
:10B550003DAD4EAD5FAD0F9477314B015C01C7013E
:10B56000B6010F9416316B017C01C301B2010F9437
:10B570001631A70196010F947731A50194010F941C
:10B58000A23718160CF09ACAA7019601C501B4019A
:10B590000F9458360F94C5362B013C018FCAF8AD75
:10B5A000FF2329F1A5019401612F702F8BA19FA189
:10B5B0000F9477314B015C012BA53FA54BA95CA9EA
:10B5C000C701B6010F947731A50194010F94A237FA
:10B5D000181614F5A7019601C501B4010F94583649
:10B5E0006BA77FA78BAB9CAB21E028AF26CBA70135
:10B5F0009601C501B4010F9458369B01AC016BA5AF
:10B600007FA58BA99CA90F9477316BA77FA78BABE4
:10B610009CAB31E038AF11CB41E048AF0ECBC090CE
:10B62000E00ED090E10EE090E20EF090E30E2DEBF4
:10B6300037E346E855E3C701B6010F94123187FDA1
:10B6400014CBC701B6010F94E7376B017C019B0156
:10B65000AC01612F702F8BA19FA10F94123187FD38
:10B6600004C01C2D0D2DEBA2FFA29601A701612F96
:10B67000702F8BA19FA10F94583666966CAF7DAF4B
:10B680008EAF9FAF6697E4EEFEE02696FFAFEEAF7B
:10B69000269720E030E040E85FE328AF39AF4AAFBB
:10B6A0005BAF1CAE2696AEADBFAD26976D917D917A
:10B6B0008D919D912696BFAFAEAF269766962CAD25
:10B6C0003DAD4EAD5FAD66970F9477316B017C0158
:10B6D0002E96EEADFFAD2E9781909190A190B190F6
:10B6E0002E96FFAFEEAF2E97FCADFF2391F028AD65
:10B6F00039AD4AAD5BAD0F9477316B017C0128AD5C
:10B7000039AD4AAD5BADC501B4010F9477314B0142
:10B710005C01A5019401C701B6010F94A23720E096
:10B7200030E0A90118162CF5C501B4010F94A23719
:10B7300018164CF020E030E0A901C701B6010F94C3
:10B74000123187FF05C0A5019401C701B60124C0CD
:10B750002401350177FA709477F87094A30192016F
:10B76000C701B6010F94A23718165CF52601370100
:10B7700028C0C501B4010F94123187FD09C020E033
:10B7800030E0A901C701B6010F94A23718164CF496
:10B79000A7019601C501B4010F947B352B013C0133
:10B7A00010C02601370177FA709477F87094A501DC
:10B7B0009401C301B2010F94A237181614F02401AA
:10B7C00035016096AEADBFAD6097CD90DD90ED9048
:10B7D000FD906096BFAFAEAF6097A7019601C30121
:10B7E000B2010F94A2371816ACF4A3019201C7015D
:10B7F000B6010F9458369B01AC0168AD79AD8AADA6
:10B800009BAD0F94773168AF79AF8AAF9BAFBCAD7A
:10B81000BF5FBCAF2696EEADFFAD2697E45FFE405E
:10B8200009F040CF3CAD332371F028AD39AD4AADBE
:10B830005BAD612F702F8BA19FA10F947731162FD5
:10B84000072F8BA39FA324EA30E74DE75FE3612F27
:10B85000702F8BA19FA10F9477316B017C019B010D
:10B86000AC016091E6037091E7038091E803909149
:10B87000E9030F94A23718165CF4A70196016BA593
:10B880007FA58BA99CA90F94A23718160CF4EDC9BB
:10B890001BA70FA70BA10BAB1FA11CABE6C983E035
:10B8A00043CAF090BA0E8FEF8F0D8F708BA3B090BC
:10B8B000B90E8091BA0EB81206C00091B90E0BA352
:10B8C000C12CD12C69C0C12CD12C1BA11B15A9F3F3
:10B8D0001BA1812E912C2AE5289D8001299D100D08
:10B8E00011240B5E1B4FD8018C9183FD27C00BAB3D
:10B8F0001CAB0115110521F11996BC91BFA3F801EC
:10B90000F285FBA7D8011B96BC91BFA7F801A484C0
:10B9100045805680678070842FA13BA54B2F5A2D00
:10B92000C301B2010F94123181117CC1C114D10441
:10B9300039F0D6018C9180FD75C102C0CBAADCAA7A
:10B940008BA181508F708BA38091B90EB81649F0EE
:10B950000BA10B1509F4B1CF81E08B0D8F70B82EC0
:10B96000F3CFCBA8DCA8B1CF0BA1802E912C2AE578
:10B97000289D8001299D100D11240B5E1B4FD801BD
:10B980008C9183FD14C05801C114D10459F48BA1CA
:10B990008F5F8F708BA365018091BA0E1BA1181366
:10B9A000E3CF6BCAC6014CD58111F1CFB0C15601AE
:10B9B000EECF8FA181508F70989FF0011124EB5E24
:10B9C000FB4F208123FF64CA8FA35ECA2AE53BA1F7
:10B9D000239FC0011124AC014B5E5B4F1A01DA01B9
:10B9E0008C9183FD19C015966D917D918D919C91DF
:10B9F00018970F94E737F62EE72ED82EC92E01158B
:10BA0000110509F489C0F801808180FD0AC0D101C7
:10BA10008C9180FD06C080C0FBA4EFA4DBA8CCA85D
:10BA200080C0F801808181608083C80109D58111BF
:10BA30006FC0F80161817281838194810F94E7372F
:10BA40002B013C019B01AC0160E070E080E89FE3CA
:10BA50000F9458364B015C019B01AC016F2D7E2D7C
:10BA60008D2D9C2D0F94773169837A838B839C83F2
:10BA7000A50194016BA57FA58BA99CA90F94773193
:10BA8000698B7A8B8B8B9C8BAE014F5F5F4FBE01B6
:10BA90006F5E7F4FC8010E946C85D801D7968C914C
:10BAA0008823B1F120910D1530910E1540910F159D
:10BAB00050911015F801FE96608171818281938109
:10BAC0000F947731209196123091971240919812ED
:10BAD000509199120F9477314B015C019B01AC019D
:10BAE000C301B2010F9477310F94C536F80173AFDB
:10BAF00062AFA50194016F2D7E2D8D2D9C2D0F948D
:10BB000077310F94C536D801DD967C936E93DC9720
:10BB1000F80180818E7F80838F2C9E2CAD2CBC2CD5
:10BB200081018BA18F5F8F708BA3FBA6EFA6DBAA91
:10BB3000CCAABAC9D1018C9181608C93C80180D400
:10BB400081116BC0F10161817281838194810F94B5
:10BB5000E7376B017C019B01AC0160E070E080E89D
:10BB60009FE30F9458362B013C012DEC3CEC4CE448
:10BB70005DE30F94773169837A838B839C83A30180
:10BB80009201B401C5010F947731698B7A8B8B8B4D
:10BB90009C8BAE014F5F5F4FBE016F5E7F4FC10157
:10BBA0000E946C85D101D7968C918823B1F12091A8
:10BBB0000D1530910E1540910F1550911015F10192
:10BBC000FE9660817181828193810F9477312091FB
:10BBD00096123091971240919812509199120F94A9
:10BBE00077314B015C019B01AC01C701B6010F9499
:10BBF00077310F94C536F10173AF62AF2DEC3CEC99
:10BC00004CE45DE3C501B4010F9477310F94C53660
:10BC1000D101DD967C936E93DC97F10180818E7F5C
:10BC200080834AC92AE5289DF001299DF00D112441
:10BC3000EB5EFB4F808181FD3FC0C114D10431F028
:10BC4000F601C580D680E780F08408C08BE0C82E5E
:10BC500087EDD82E83E2E82E8BE3F82E2AE5289D87
:10BC6000F001299DF00D1124EB5EFB4F8189928933
:10BC7000A389B489BC01CD0190589B01AC010F94FC
:10BC80007C35D8011D962D913D914D915C91509739
:10BC90000F9477319B01AC01C701B6010F947B353E
:10BCA0001B016C019B01AC016FA17BA58FA59A2D97
:10BCB0000F94123187FF04C02FA03BA4CFA4DA2C2D
:10BCC0009101A601C301B2010F941231882309F436
:10BCD00037CEBAE5B89DC001B99D900D1124FC0185
:10BCE000EB5EFB4F4F01808181608083C801A8D348
:10BCF000882329F0D4018C918E7F8C9321CEC101B1
:10BD0000D601F40185839683A783B08719CED60127
:10BD10008C9181FD4FC0D60115962D913D914D918D
:10BD20005C9118972FA338A749A75AA71501B5E02A
:10BD30002B0E311CF8014580568067807084A3016A
:10BD400092016FA178A589A59AA50F94123187FF5A
:10BD500031C0F60181899289A389B489BC01CD01E2
:10BD600090589B01AC010F947C35D6011D962D9106
:10BD70003D914D915C9150970F9477319B01AC01AF
:10BD80006FA178A589A59AA50F947B356B017C01DD
:10BD9000A30192010F94123187FF0CC0D8018C913E
:10BDA00081608C93C5014CD38823E1F0F801808138
:10BDB0008E7F80831AE5189DF001199DF00D1124E6
:10BDC000EB5EFB4F21853285438554856581768105
:10BDD000878190850F9412318111D9CD0BA10093E9
:10BDE000B90ED5CDD101CD92DD92ED92FC92139793
:10BDF0000BA10093B90EDECFC458DF4F0FB6F894F5
:10BE0000DEBF0FBECDBFDF91CF911F910F91FF908D
:10BE1000EF90DF90CF90BF90AF909F908F907F90EA
:10BE20006F905F904F903F902F9008958091BA0E41
:10BE30009091BB0E891B8F708F3021F480E00F949E
:10BE4000FA20F4CF8091BA0E8F5F8F70E091BA0E16
:10BE50009AE59E9FF0011124EB5EFB4FDF011D92DE
:10BE60009A95E9F798E090834091040F5091050F5F
:10BE70006091060F7091070F458B568B678B708F03
:10BE80004091080F5091090F60910A0F70910B0FAC
:10BE9000418F528F638F748F40910C0F50910D0F13
:10BEA00060910E0F70910F0F458F568F678F70A3A3
:10BEB0004091100F5091110F6091120F7091130F5C
:10BEC00041A352A363A374A32091BA0E9091BB0E19
:10BED000291303C094E69093B70E8093BA0E809115
:10BEE0006F00826080936F0008959091BA0E8091E8
:10BEF000BB0E981721F080E00F94FA20F6CF8091C6
:10BF0000EB039091EC03892BB1F708959091BA0E51
:10BF10008091BB0E981721F080E00F94FA20F6CFA5
:10BF20008091EB039091EC03892BB1F70D943224AF
:10BF3000CF93DF9390916F0091FB222720F991FF1F
:10BF400005C090916F009D7F90936F0094E0899F52
:10BF5000E0011124FE01E45FF54F6081718182816F
:10BF60009381222329F020916F00226020936F009B
:10BF70000F941831CF5FDB4F288139814A815B8173
:10BF80000F947731DF91CF9108952F923F924F9286
:10BF90005F926F927F928F929F92AF92BF92CF9259
:10BFA000DF92EF92FF920F931F93CF93DF93CDB762
:10BFB000DEB7E8970FB6F894DEBF0FBECDBF209175
:10BFC0003515222309F4E6C01C010091C00E109122
:10BFD000C10E2091C20E3091C30E4090C40E5090FD
:10BFE000C50E6090C60E7090C70E4DA65EA66FA6D9
:10BFF00078AA8090C80E9090C90EA090CA0EB090FA
:10C00000CB0E4091CC0E5091CD0E6091CE0E709122
:10C01000CF0E8091D00E9091D10EA091D20EB09102
:10C02000D30E89AB9AABABABBCABC090D40ED09067
:10C03000D50EE090D60EF090D70E8091D80E90914C
:10C04000D90EA091DA0EB091DB0E4090DC0E50902C
:10C05000DD0E6090DE0E7090DF0E4DAA5EAA6FAA14
:10C0600078AE4090BC0E5090BD0E6090BE0E7090A9
:10C07000BF0E49825A826B827C828D829E82AF8201
:10C08000B886C986DA86EB86FC860D871E872F87E1
:10C09000388B498B5A8B6B8B7C8B8D8B9E8BAF8BAC
:10C0A000B88F8DA59EA5AFA5B8A9898F9A8FAB8FA4
:10C0B000BC8F49A85AA86BA87CA84D8E5E8E6F8E47
:10C0C00078A28DA99EA9AFA9B8AD89A39AA3ABA365
:10C0D000BCA320E030E048E951E4D1016D917D91AD
:10C0E0008D919C910F947C3569A77AA78BA79CA70B
:10C0F00020E030E041E853E4F101648175818681FC
:10C1000097810F947B356DA37EA38FA398A7C10160
:10C1100008969F938F93CE0185969F938F93049655
:10C120009F938F938DB79EB784970FB6F8949EBF59
:10C130000FBE8DBFADB7BEB7119684E2FE0131963A
:10C1400001900D928A95E1F70F94420F20E030E0C4
:10C1500048E951E469A57AA58BA59CA50F947B3588
:10C16000D1016D937D938D939C93139720E030E0E4
:10C1700041E853E46DA17EA18FA198A50F947C3571
:10C18000F10164837583868397830FB6F894DEBFCD
:10C190000FBECDBFE8960FB6F894DEBF0FBECDBF81
:10C1A000DF91CF911F910F91FF90EF90DF90CF9093
:10C1B000BF90AF909F908F907F906F905F904F90C7
:10C1C0003F902F900895CF93DF938091BA0E909176
:10C1D000BB0E891B8F7009F445C09091B70E99234F
:10C1E00051F0833030F48FEF890F19F08093B70E40
:10C1F0003BC01092B70EE091BB0E8AE5E89FF001BC
:10C200001124EB5EFB4F808180FD2EC080911104D4
:10C2100090911204A0911304B0911404EF01CA5A32
:10C22000DF4F488159816A817B81841B950BA60B66
:10C23000B70B8093110490931204A0931304B0934E
:10C2400014048091BB0E8F5F8F708093B80E909115
:10C25000BB0E8091B90E98130AC08091B80E8093DE
:10C26000B90E05C00E943F8780E090E001C0CF0179
:10C27000DF91CF91089567FD3BC08230D9F028F45B
:10C28000882341F0813061F033C08330E9F084309D
:10C2900029F12EC0662311F0A19A39C0A19837C0A8
:10C2A000809108016111809580788093060147FF95
:10C2B00036C0089580910801611180958074809343
:10C2C000060147FF32C008958091080161118095F1
:10C2D00088708093060147FF2EC008958091080161
:10C2E0006111809582708093060147FF2AC00895EE
:10C2F00047FD2FC08230C9F028F4882351F08130E7
:10C3000071F008958330B9F08430D9F0089547FD75
:10C3100020C0442311F0A09A0895A09808954423C2
:10C3200011F0A29A0895A2980895809108014111F0
:10C33000809580720BC080910801411180958071B9
:10C3400005C0809108014111809584708093060199
:10C35000089508955F988EBD00000DB407FEFDCFCF
:10C360008EB56EBD00000DB407FEFDCF8EB55F9A91
:10C370000895CF93DF9300D01F921F92CDB7DEB701
:10C3800095E0E8E6F2E0DE01119601900D929A95B3
:10C39000E1F7E1E0F0E0EC0FFD1FE80FF11D808117
:10C3A00090E00F900F900F900F900F90DF91CF9132
:10C3B000D1CF90916F0091FB222720F991FF05C00A
:10C3C00090916F009D7F90936F0034E0839FC00138
:10C3D0001124FC01E658FD4E408151816281738138
:10C3E000FC01E45FF54F408351836283738381E0F6
:10C3F00080930B0A222329F080916F008260809342
:10C400006F00089590916F0091FB222720F991FF12
:10C4100005C090916F009D7F90936F0094E0899F7D
:10C42000F0011124E658FD4E608171818281938173
:10C43000222329F020916F00226020936F0008953D
:10C44000BC012091090A30910A0A4091090A5091D1
:10C450000A0A2417350711F09A01F7CF81E0621715
:10C46000730709F080E008950F930FB70F930091C1
:10C470006E000F930B7F00936E0000916F000D7F95
:10C4800000936F000F930BB70F930CB70F921F928F
:10C490002F933F934F935F936F937F938F939F93CC
:10C4A000AF93BF93EF93FF9311245DD0FF91EF9172
:10C4B000BF91AF919F918F917F916F915F914F91BC
:10C4C0003F912F911F900F900CBF0F910BBF0F91B9
:10C4D0000260F89400936F000F9100936E000F912B
:10C4E0000FBF0F9118958091BB0980FF07C0809105
:10C4F0000B018270809309018FEF07C080910B01BF
:10C50000809582708093090181E08093B5098091C4
:10C51000BB0981FF08C080910B01809581708093D9
:10C5200009018FEF06C080910B0181708093090192
:10C5300081E08093B6098091BB0982FF07C080919A
:10C540000B018470809309018FEF07C080910B016C
:10C55000809584708093090181E08093B709000081
:10C560000000000008952F923F924F925F926F92C9
:10C570007F928F929F92AF92BF92CF92DF92EF9273
:10C58000FF920F931F93CF93DF9300D000D0CDB7CE
:10C59000DEB7F8948FEF9FEF909389008093880027
:10C5A0002AE02D83212C312C78948091050A9091DA
:10C5B000060AA091070AB091080A892B8A2B8B2BB7
:10C5C00009F0CDC180910B0A8823D1F010920B0A9B
:10C5D0008091090A90910A0A892B91F01092FC0926
:10C5E00010920A0A1092090A9091BA0E8091BB0E1D
:10C5F000981731F08091BB0E8F5F8F708093BB0EC8
:10C600008091090A90910A0A892B09F4A8C14091E6
:10C61000010A5091020A6091030A7091040A9091F4
:10C62000EF090091FD091091FE092091FF09309159
:10C63000000A041B150B260B370B892F90E0A0E096
:10C64000B0E0081719072A073B0710F4D901C80101
:10C65000E82F840F951FA61FB71F8093010A9093A0
:10C66000020AA093030AB093040A20918400309137
:10C670008500225E3F4F4091D5095091D6096091C7
:10C68000D7097091D8098091C5099091C609A091E8
:10C69000C709B091C809840F951FA61FB71F8093C3
:10C6A000D5099093D609A093D709B093D809B7FDBF
:10C6B0001CC0409A40917A1250917B1260917C127A
:10C6C00070917D128091B509082E000C990BAA0B70
:10C6D000BB0B840F951FA61FB71F80937A129093F0
:10C6E0007B12A0937C12B0937D124091D909509196
:10C6F000DA096091DB097091DC098091C909909198
:10C70000CA09A091CB09B091CC09840F951FA61F2F
:10C71000B71F8093D9099093DA09A093DB09B093EE
:10C72000DC09B7FD1CC0419A40917E1250917F12E6
:10C7300060918012709181128091B609082E000CD0
:10C74000990BAA0BBB0B840F951FA61FB71F8093D5
:10C750007E1290937F12A0938012B0938112409129
:10C76000DD095091DE096091DF097091E009809147
:10C77000CD099091CE09A091CF09B091D009840F35
:10C78000951FA61FB71F8093DD099093DE09A09324
:10C79000DF09B093E009B7FD1CC0429A40918212B4
:10C7A0005091831260918412709185128091B70923
:10C7B000082E000C990BAA0BBB0B840F951FA61F0C
:10C7C000B71F8093821290938312A0938412B09328
:10C7D00085124091E1095091E2096091E30970915D
:10C7E000E4098091D1099091D209A091D309B09127
:10C7F000D409840F951FA61FB71F8093E10990935A
:10C80000E209A093E309B093E409B7FD3AC0C090F0
:10C810008612D0908712E0908812F0908912409191
:10C82000B809042E000C550B660B770B4C0D5D1DE3
:10C830006E1D7F1D4093861250938712609388125D
:10C84000709389124091C1095091C2096091C30946
:10C850007091C409841B950BA60BB70B8093E1095B
:10C860009093E209A093E309B093E4099091BB0986
:10C870008091ED0993FF02C0815001C08F5F8093CA
:10C88000ED09809184009091850082179307C8F389
:10C890008091D5099091D609A091D709B091D80976
:10C8A000B7FD15C04091C1095091C2096091C309FB
:10C8B0007091C409841B950BA60BB70B8093D50907
:10C8C0009093D609A093D709B093D8094098809146
:10C8D000D9099091DA09A091DB09B091DC09B7FD83
:10C8E00015C04091C1095091C2096091C30970916E
:10C8F000C409841B950BA60BB70B8093D9099093A1
:10C90000DA09A093DB09B093DC0941988091DD0935
:10C910009091DE09A091DF09B091E009B7FD15C043
:10C920004091C1095091C2096091C3097091C40935
:10C93000841B950BA60BB70B8093DD099093DE0942
:10C94000A093DF09B093E0094298E15041F0809153
:10C9500084009091850082179307C8F38ACE809156
:10C96000130290911402A0911502B0911602892B26
:10C970008A2B8B2B09F09AC08091EE09882309F449
:10C9800055C0C090010AD090020AE090030AF090CE
:10C99000040A4091E9095091EA096091EB0970910C
:10C9A000EC098091ED094C155D056E057F0588F455
:10C9B0002091B9093091BA09E091BE09F091BF09FF
:10C9C000E217F30730F481508093ED0921503109CB
:10C9D00015C0C416D506E606F706E8F42091B90995
:10C9E0003091BA094091BC095091BD09241735070F
:10C9F00090F48F5F8093ED092F5F3F4F3093BA091A
:10CA00002093B90940910F025091100260911102D8
:10CA1000709112020EC08FEF9FEFDC0180930F0226
:10CA200090931002A0931102B09312024FEF5FEFA8
:10CA3000BA018091ED0987FD03C080910B0103C00D
:10CA400080910B018095807480930901209184006E
:10CA500030918500225E3F4F8091ED098823F1F0EF
:10CA6000439A809184009091850082179307C8F3C0
:10CA70008091ED0987FF02C08F5F01C081508093D4
:10CA8000ED0943988091ED09882331F3809184006A
:10CA90009091850082179307C8F3DCCF409313026F
:10CAA0005093140260931502709316028091050A48
:10CAB0009091060AA091070AB091080A892B8A2B47
:10CAC0008B2B09F06BC3A091090AB0910A0A109749
:10CAD00039F1C090010AD090020AE090030AF09068
:10CAE000040A4091FD095091FE096091FF0970917F
:10CAF000000AC416D506E606F706C8F01092FC092F
:10CB000010920A0A1092090A9091BA0E8091BB0EF7
:10CB1000981731F08091BB0E8F5F8F708093BB0EA2
:10CB2000A0ED8A2EA7E09A2EA12CB12C81C14091B4
:10CB3000F8095091F9096091FA097091FB094C15B7
:10CB40005D056E057F0508F46EC04091F4095091B3
:10CB5000F5096091F6097091F709D2960D911D9132
:10CB60002D913C91D597EE27419FF12D529FC00109
:10CB7000629F900D619F800D911D429FF00D811D60
:10CB80009E1F519FF00D811D9E1F609FF00D811D06
:10CB90009E1F509FF10D8E1F9E1FF6958E1F9E1F8C
:10CBA000349F800D911D359F900D1124FD01EA5B8E
:10CBB000FF4F0081118122813381080F191F211D30
:10CBC000311D0093F0091093F1092093F20930937D
:10CBD000F309349780809180A280B38080169106FB
:10CBE000A206B30640F48092F0099092F109A09257
:10CBF000F209B092F3098090F0099090F109A090A9
:10CC0000F209B090F30982EF98E177247394FC0164
:10CC10000591159125913491081519052A053B05B3
:10CC200008F433C33DC32091E9093091EA094091EA
:10CC3000EB095091EC0929833A834B835C832C15D3
:10CC40003D054E055F0508F068C04091E50950912B
:10CC5000E6096091E7097091E809D2960D911D915E
:10CC60002D913C91D597EE27419FF12D529FC00108
:10CC7000629F900D619F800D911D429FF00D811D5F
:10CC80009E1F519FF00D811D9E1F609FF00D811D05
:10CC90009E1F509FF10D8E1F9E1FF6958E1F9E1F8B
:10CCA000349F800D911D359F900D11248C0120E043
:10CCB00030E04090F0095090F1096090F2097090D6
:10CCC000F309FD01E65BFF4F041515052605370541
:10CCD00080F480809180A280B380401A510A620A59
:10CCE000730A481459046A047B0438F4240135019A
:10CCF00004C0408051806280738082EF98E131E00F
:10CD00003E83FC010591159125913491041515057B
:10CD10002605370508F441C34DC38091ED098823EA
:10CD2000D9F0D8964D915C91D99760E070E0009170
:10CD30000F0210911002209111023091120204177B
:10CD400015072607370741F01092130210921402BC
:10CD5000109215021092160240910B0250910C0293
:10CD600060910D0270910E0277FF5AC0AE5BBF4F0B
:10CD70008D919D910D90BC91A02D22EF38E141E065
:10CD8000F901C590D590E590F490C816D906EA0649
:10CD9000FB0658F4B695A79597958795440F2C5F99
:10CDA0003F4F59E12E30350759F74093EF09803254
:10CDB0009105A105B10508F4ECC38097A109B1095B
:10CDC0008115E8E09E07A105B10508F4BDC324E084
:10CDD000929FF00111249F012E503B4EF901329693
:10CDE00045915491EE27859FB001849F610D7E1F70
:10CDF00006946E1F7E1F1124AB0160E070E0F90104
:10CE000085919491A0E0B0E0841B950BA60BB70B25
:10CE100080930B0290930C02A0930D02B0930E022C
:10CE200080900B0290900C02A0900D02B0900E0228
:10CE30008091090A90910A0A892B09F0A7C1C3D9E8
:10CE400090930A0A8093090A892B09F49FC1609084
:10CE5000090A70900A0AD3018C9183FF3FC0F30145
:10CE600085899689A789B08D80937A1290937B12D9
:10CE7000A0937C12B0937D12818D928DA38DB48D81
:10CE800080937E1290937F12A0938012B0938112B0
:10CE9000858D968DA78DB0A1809382129093831279
:10CEA000A0938412B093851281A192A1A3A1B4A1F1
:10CEB0008093861290938712A0938812B093891260
:10CEC0009091BA0E8091BB0E981709F4B8CF80915B
:10CED000BB0E8F5F8F708093BB0EB1CF5596CD90F8
:10CEE000DD90ED90FC90589781E0C114D104E104ED
:10CEF000F10409F480E0F301018D128D238D348D4E
:10CF0000011511052105310509F08260D3015D96F7
:10CF10004D915D916D917C91909741155105610501
:10CF2000710509F084608093FC091092E509109264
:10CF3000E6091092E7091092E8091092F40910929C
:10CF4000F5091092F6091092F709F30185A196A14F
:10CF5000A7A1B0A58093FD099093FE09A093FF09B6
:10CF6000B093000A882499245401881A990AAA0ABD
:10CF7000BB0A8092E1099092E209A092E309B09283
:10CF8000E4098092DD099092DE09A092DF09B09257
:10CF9000E0098092D9099092DA09A092DB09B09257
:10CFA000DC098092D5099092D609A092D709B09257
:10CFB000D809CC0CDD1CEE1CFF1CC092C509D09218
:10CFC000C609E092C709F092C809000F111F221F7D
:10CFD000331F0093C9091093CA092093CB093093DA
:10CFE000CC09440F551F661F771F4093CD095093FE
:10CFF000CE096093CF097093D00941A152A163A1DA
:10D0000074A1440F551F661F771F4093D109509399
:10D01000D2096093D3097093D409880F991FAA1F6E
:10D02000BB1F8093C1099093C209A093C309B09319
:10D03000C4091092010A1092020A1092030A109277
:10D04000040A82A593A5A4A5B5A58093F809909399
:10D05000F909A093FA09B093FB0986A597A5A0A9A1
:10D06000B1A98093E9099093EA09A093EB09B093E1
:10D07000EC0981A58093C00997A99093EE099923A3
:10D0800061F024AD35AD3093BF092093BE0922ADC8
:10D0900033AD3093BD092093BC09D301D6969C9142
:10D0A0002091BB0992130AC020910A0230E0482F58
:10D0B000082E000C550B4217530729F09093BB091B
:10D0C00080930A0210DA0E944DB02FEF3FEFA901C2
:10D0D00020930B0230930C0240930D0250930E02EA
:10D0E000F301EA5BFF4F80819181A281B38180933C
:10D0F000F0099093F109A093F209B093F30922EF9C
:10D1000038E141E0F901C590D590E590F490C8165A
:10D11000D906EA06FB0658F4B695A7959795879524
:10D12000440F2C5F3F4FE9E12E303E0759F7409303
:10D13000EF0980329105A105B10508F452C280972C
:10D14000A109B109811538E09307A105B10508F4DB
:10D1500025C244E0949F900111242E503B4EF901CA
:10D16000329645915491EE27859FB001849F610DC1
:10D170007E1F06946E1F7E1F1124F90185909490E6
:10D18000A12CB12C861A970AA108B1088092050A31
:10D190009092060AA092070AB092080A0091050A26
:10D1A0001091060A2091070A3091080A4091130253
:10D1B0005091140260911502709116027801F22FBD
:10D1C000E32F401751076207730718F47A01F62F0F
:10D1D000E72FC701AF2FBE2F0097E1E0AE07B105E3
:10D1E00020F08FEF9FEFA0E0B0E0081B190B2A0B97
:10D1F0003B0B0093050A1093060A2093070A30930D
:10D20000080A4F3FFFEF5F076F077F0761F0481B7A
:10D21000590B6A0B7B0B40931302509314026093DB
:10D22000150270931602F8942091840030918500C5
:10D23000205F3F4F4D8141504D83442339F0280EEC
:10D24000391E2216330608F4AFC901C01901309205
:10D25000890020928800789426960FB6F894DEBF55
:10D260000FBECDBFDF91CF911F910F91FF90EF9037
:10D27000DF90CF90BF90AF909F908F907F906F90F6
:10D280005F904F903F902F900895B694A7949794F5
:10D290008794770C0496E9E18E309E0709F0B7CCAD
:10D2A0007092EF0980E288169104A104B10408F499
:10D2B0001CC190E2891A9108A108B1088114E8E024
:10D2C0009E06A104B104F8F0F4E09F9EC001112471
:10D2D0008E509B4EFC01329625913491F82DEE270D
:10D2E000F39F8001F29F010D1E1F06940E1F1E1F4B
:10D2F0001124FC0185909490A12CB12C801A910AE4
:10D30000A108B10823C0950184013695279517958A
:10D310000795F801EC7F9F012E503F4EF901859152
:10D320009491F901329605911491E82DE770E09FF0
:10D330009001E19F300D1124F3E036952795FA9581
:10D34000E1F74C01821A930AA12CB12C480D591D0A
:10D350006A1D7B1D4093F4095093F5096093F6090B
:10D360007093F7098091EE09882359F0472D50E01A
:10D3700060E070E0C416D506E606F70609F06CC05A
:10D3800084C02FEF3FEFA90120930F0230931002CA
:10D3900040931102509312029AC076946794579466
:10D3A00047942E81220F2E83049639E18E30930705
:10D3B00009F0A7CC2E812093EF0930E243165104E7
:10D3C0006104710408F4BAC080E2481A5108610887
:10D3D0007108411498E059066104710408F48BC087
:10D3E000E4E05E9EC00111248E509B4EFC013296FB
:10D3F00005911491F42DEE27F19F9001F09F210DDE
:10D400003E1F06942E1F3E1F1124FC018590949010
:10D41000A12CB12C821A930AA108B108480D591DFC
:10D420006A1D7B1D4093E5095093E6096093E70967
:10D430007093E8098091EE098823F1F149815A81BE
:10D440006B817C812E81420F511D611D711D4C1518
:10D450005D056E057F05C8F48091ED09882309F408
:10D46000E7CCD8964D915C91D99760E070E000913F
:10D470000F02109110022091110230911202041734
:10D4800015072607370709F4D3CC10921302109220
:10D4900014021092150210921602D8968D919C914A
:10D4A000D997A0E0B0E080930F0290931002A09370
:10D4B0001102B0931202BCCC8FEF9FEFDC0180937E
:10D4C0000F0290931002A0931102B0931202809168
:10D4D000ED09882309F4ACCC1092130210921402C7
:10D4E0001092150210921602A3CC00E2802E912C0D
:10D4F000A12CB12CDECE930182013695279517958C
:10D500000795F801EC7FCF018E509F4EFC0185906E
:10D510009490FC01329625913491E42DE770E29FBE
:10D52000C001E39F900D112423E0969587952A95DD
:10D53000E1F7881A990AA12CB12C70CFF0E24F2E96
:10D54000512C612C712C40CFAC01BD0176956795B3
:10D5500057954795FA01EC7FAF014E505F4EFA01A7
:10D5600025913491FA013296459154918770849FA8
:10D57000B001859F700D1124CB01F3E0969587953E
:10D58000FA95E1F7A901481B590BCA01A0E0B0E0E8
:10D590003FCC80E290E0A0E0B0E00FCCAC01BD0158
:10D5A0007695679557954795FA01EC7F9F012E5028
:10D5B0003F4EF90185909490F9013296259134916E
:10D5C0008770829FA001839F500D1124CA0123E020
:10D5D000969587952A95E1F7881A990AA12CB12C7E
:10D5E000D5CD80E290E0A0E0B0E0A9CD8F929F92EF
:10D5F000AF92BF92CF92DF92EF92FF920F931F9361
:10D60000CF93DF9300D01F92CDB7DEB78EE5882E83
:10D6100085E1982E9AE8A92E92E1B92E01EF13E048
:10D62000C12CD12C7601C394F40161917191819147
:10D6300091914F01F50121913191419151915F01FA
:10D6400029833A834B835C830F94163129813A8175
:10D650004B815C810F9477310F94C536F80161934B
:10D660007193819391938F01C616D706E806F90648
:10D6700010F46B017C01FEE68F16F5E19F06A1F622
:10D680006FEF7FEFCB01A70196010F941E3520931A
:10D69000ED033093EE034093EF035093F0030F90AC
:10D6A0000F900F900F90DF91CF911F910F91FF90EE
:10D6B000EF90DF90CF90BF90AF909F908F900895A4
:10D6C0008F929F92AF92BF92EF92FF920F931F9310
:10D6D000CF93DF937B018A01E901FC018080918077
:10D6E000A280B38020918A1230918B1240918C12CB
:10D6F00050918D12C501B4010F9477310F94AD375D
:10D700006093040F7093050F8093060F9093070F9B
:10D7100020918E1230918F1240919012509191125F
:10D72000F70160817181828193810F9477310F9429
:10D73000AD376093080F7093090F80930A0F909391
:10D740000B0F2091921230919312409194125091AC
:10D750009512F80160817181828193810F947731F4
:10D760000F94AD3760930C0F70930D0F80930E0FD5
:10D7700090930F0F2091961230919712409198122A
:10D7800050919912688179818A819B810F947731B8
:10D790000F94AD376093100F7093110F8093120F99
:10D7A0009093130F8092F40E9092F50EA092F60EC5
:10D7B000B092F70EF70180819181A281B3818093AD
:10D7C000F80E9093F90EA093FA0EB093FB0EF801A9
:10D7D00080819181A281B3818093FC0E9093FD0E94
:10D7E000A093FE0EB093FF0E88819981AA81BB8120
:10D7F0008093000F9093010FA093020FB093030F3B
:10D800009091BA0E8091BB0E981761F0DF91CF9185
:10D810001F910F91FF90EF90BF90AF909F908F90CE
:10D820000C94165F0E94755F80916F0081FB9927B1
:10D8300090F981FF05C080916F008D7F80936F000C
:10D840004091040F5091050F6091060F7091070FE2
:10D8500040937A1250937B1260937C1270937D12E6
:10D860004091080F5091090F60910A0F70910B0FB2
:10D8700040937E1250937F126093801270938112B6
:10D8800040910C0F50910D0F60910E0F70910F0F82
:10D890004093821250938312609384127093851286
:10D8A0004091100F5091110F6091120F7091130F52
:10D8B0004093861250938712609388127093891256
:10D8C000992329F080916F00826080936F00DF912F
:10D8D000CF911F910F91FF90EF90BF90AF909F90CD
:10D8E0008F900895EF92FF920F931F93CF93DF9342
:10D8F000CDB7DEB72C970FB6F894DEBF0FBECDBF05
:10D900000AE812E181E0E82E84E0F82EF801219186
:10D910003191419151918F0160E070E080E89FE387
:10D920000F945836F70161937193819391937F011E
:10D93000F2E10A391F0751F7809166129091671240
:10D94000A0916812B091691289839A83AB83BC83DA
:10D9500080916A1290916B12A0916C12B0916D122D
:10D960008D839E83AF83B88780916E1290916F12E2
:10D97000A0917012B091711289879A87AB87BC878A
:10D98000AE01475F5F4FBE016B5F7F4FCE010196D7
:10D990000E94818422E732E1AE01475F5F4FBE0102
:10D9A0006B5F7F4FCE0101968BDE20DE2C960FB68B
:10D9B000F894DEBF0FBECDBFDF91CF911F910F91C5
:10D9C000FF90EF90089590918E0BE92FF0E0E757CC
:10D9D000F44F80839F5F953018F490938E0B02C0B4
:10D9E00010928E0B8091720D8F5F8093720D08954F
:10D9F000CF93FC0180818B33A1F08091720D853033
:10DA000080F4C62FBF0180918E0B20E6829FC0015B
:10DA100011248F56944F0F94BA388C2FD4DF81E0A5
:10DA200001C080E0CF910895CF93DF93EC0160E0D7
:10DA3000CE01DEDF811104C080E00F94FA20F7CF21
:10DA4000CE010F94DF148823B9F3DF91CF910895AD
:10DA5000DF92EF92FF920F931F93CF93DF93CDB797
:10DA6000DEB76E970FB6F894DEBF0FBECDBF6091E4
:10DA70009A1270919B126115710501F14DE150E010
:10DA8000CE0101967C010F9482301E8EF7018F012A
:10DA90000E191F09D190DD2019F09AE0D912F7CFA5
:10DAA000F701E00FF11F108260E0C701A1DF8823BA
:10DAB00029F0C7010F94DF14811109C081E0209182
:10DAC0009A1230919B12232BA1F480E012C0DD202A
:10DAD00049F00F5F1F4F80919A1290919B12080F8F
:10DAE000191F02C000E010E010939B1200939A12DD
:10DAF000E5CF6E960FB6F894DEBF0FBECDBFDF91B7
:10DB0000CF911F910F91FF90EF90DF9008950F93A9
:10DB10001F93CF93DF93CDB7DEB72C970FB6F89452
:10DB2000DEBF0FBECDBFE6E6F2E180859185A2851E
:10DB3000B38544815581668177810081118122817D
:10DB4000338109831A832B833C834D835E836F83E8
:10DB5000788789879A87AB87BC87AE01475F5F4F1D
:10DB6000BE016B5F7F4FCE0101960E94818422E748
:10DB700032E1AE01475F5F4FBE016B5F7F4FCE0169
:10DB800001969EDD2C960FB6F894DEBF0FBECDBF7A
:10DB9000DF91CF911F910F91089580919D039091F6
:10DBA0009E03009731F04AE050E060E070E00D9491
:10DBB0001A2F60E070E0CB01089580919D03909151
:10DBC0009E03009731F04AE050E060E070E00D9471
:10DBD000F22D60E070E0CB010895EFDF97FD0AC001
:10DBE000ECDF6F3F71058105910509F02CF4E5DF4D
:10DBF000862F089580E008958FEF089580919D030A
:10DC000090919E03892B31F0E8DF91E0811103C0F0
:10DC100090E001C091E0892F08950F931F93CF9357
:10DC200080919D0390919E03009711F1FC018F015B
:10DC3000C1912C2F2F7DA9F0C53411F0C536B9F74D
:10DC4000F801108260E070E080919D0390919E0346
:10DC50000F948B2CF801C083562F472F382F292F74
:10DC60000BC060E070E0CF911F910F910D948B2C51
:10DC700050E040E030E020E0652F742F832F922F9A
:10DC8000CF911F910F91089581548A3108F041C0BE
:10DC9000A82FB0E04091420B5091430B6091440B90
:10DCA0007091450B04C076956795579547958A9571
:10DCB000D2F740FF2EC0E0916916F0916A16A85D78
:10DCC000B44F8C918823E9F0E80FF11D808190ED2D
:10DCD000980F9A3098F08E3211F481810CC08D32F9
:10DCE00011F08B3271F4818190ED980F9A3030F001
:10DCF0008E3239F4828180538A3018F49E2F8F2F10
:10DD000002C090E080E090939D0380939E0381E0A9
:10DD1000089580E00895B8DF882341F081E02091E4
:10DD20009D0330919E03232B09F480E00895FC01AC
:10DD3000238121110C9450E7089580E1E6E6F2E199
:10DD4000A4EEB4E101900D928A95E1F7089580E187
:10DD5000E4EEF4E1A6E6B2E101900D928A95E1F7D6
:10DD6000089543E952E064E670E080E090E00F94AB
:10DD70007E1D4AEB52E064E670E080E090E00D9496
:10DD80007E1D0F931F93CF93DF93982F862F8A01C9
:10DD9000D22F692F0E94854C909147128091A0123A
:10DDA000891748F19091491280919F12981718F1A4
:10DDB000C4E1F8018491882331F00E94B7AFC81BF9
:10DDC0000F5F1F4FF6CFCC2329F080E20E9488B569
:10DDD000C150F9CF8091A0129AE790934A12809394
:10DDE0004B128D2F0E94CBAF80E2DF91CF911F911C
:10DDF0000F910C9488B5DF91CF911F910F910895E9
:10DE00008DE299E10E943BB581E080933C0A089540
:10DE10000F931F930E9471950091380A1091390A4F
:10DE200020913A0A30913B0ADC01CB01801B910B17
:10DE3000A20BB30BB7FD0FC08091030185FB99279F
:10DE400090F981E089279091030196FF8260629B9F
:10DE500084608093370A8091370A81709091370AE5
:10DE600091FD82609091360A891731F18130A9F0D5
:10DE700028F0823041F0833059F01CC0913089F095
:10DE8000923099F017C0992361F0933071F012C06D
:10DE9000913059F0923071F404C0992331F09330ED
:10DEA00049F49091350A9F5F03C09091350A9150D3
:10DEB0009093350A8093360A1F910F9108950F931E
:10DEC0001F93CF93DF938C0167FF03C01092B312AF
:10DED00060E08091B31290E0262F062E000C330BE9
:10DEE000281739070CF16093B312C8010F94613001
:10DEF000F801E80FF91FEF01C01BD10BC731D105A5
:10DF000034F031978491807C8038D9F3F4CFDD27C9
:10DF1000AE01B80180EA9EE00F948230C056D14F26
:10DF2000188283E080934502DF91CF911F910F917A
:10DF300008954F925F926F927F929F92AF92BF929D
:10DF4000CF92DF92EF92FF920F931F93CF93DF93C5
:10DF50001F92CDB7DEB77CDD81114DC28091720D6D
:10DF6000853028F40F948128AC0197FF3BC1809144
:10DF7000640F882309F43FC28091720D811102C0A1
:10DF80001092A30AEE24E3944091041250910512DA
:10DF90006091061270910712809100129091011207
:10DFA000A0910212B0910312481759076A077B0724
:10DFB00008F4E12C00E010E0BB24B39480E6A82E26
:10DFC00095E5C92E93E2D92E2DE8922E8091720DFF
:10DFD000853008F010C2E1100EC28091A30A8111B1
:10DFE0000AC280915B1190915C11A0915D11B0917A
:10DFF0005E118093041290930512A0930612B093C1
:10E00000071241E050E0BE016F5F7F4F83E591E171
:10E010000E9426E3019719F4898190E002C08FEFF6
:10E020009FEFF82EEE24E3944090041250900512D6
:10E0300060900612709007124091001250910112E8
:10E040006091021270910312441655066606770617
:10E05000C8F4E12C8F3FFFEF9F0709F46DC02AE061
:10E06000821709F48EC08DE0F81609F48AC093E295
:10E07000F91619F0EAE3FE129BC08091A20A811101
:10E0800097C074C00E94755F83E591E10E9450E7DC
:10E0900080916E11882359F1815080936E11989E62
:10E0A000C001112441E061E08D589E4E0E949CF019
:10E0B000E0916E1124E0E29FF0011124E159FE4E3F
:10E0C0004081518162817381409304125093051203
:10E0D000609306127093071283E591E10E9411E1AB
:10E0E0008091650F8823B9F0B092640F14C010922C
:10E0F000640F0E94865F0E94C3B10E941DB16D3300
:10E1000071058105910528F0D0929B12C0929A1258
:10E110009FDC10929C038091640F81112BC0E8E674
:10E12000F3E284913F019FEF691A790A8823F1F0A5
:10E130000F943D27F301F5CFE8EFFAE484913F0116
:10E140002FEF621A720A882321F00F943D27F30102
:10E15000F5CFE9E5F3E284913F019FEF691A790A6F
:10E16000882321F00F943D27F301F5CFE3E2FE125F
:10E1700008C005C023E2F2123BC100E010E0B092FB
:10E18000A30A1092A20A0115110519F40E94338CFA
:10E190000CC080918E0BA89E000D111D1124F8015A
:10E1A000EF56F44F108280E00EDC00E010E00ECF5E
:10E1B0000F35110508F00ACFFBE3FF1202C0B09241
:10E1C000A20A8091A20A811101CF80918E0BF801E1
:10E1D000A89EE00DF11D1124EF56F44FF0820F5F61
:10E1E0001F4FF4CE982F2091BF143091C0148A3065
:10E1F00019F09D3009F0CAC01092A10A211531050D
:10E2000019F40E94338CAACEF901EF5BF54F10820E
:10E210001092C0141092BF1421E43AE08901F90170
:10E2200080812F5F3F4F8032C9F378018E3409F02F
:10E230007CC00115110509F478C060E573E2C801DE
:10E240000F949130DD24D394892B11F4D12C09C083
:10E250006EE470E0C80104960F94AF38009709F09F
:10E260008C014AE050E060E070E0C80101960F9434
:10E27000F22D60933D0A70933E0A80933F0A90937B
:10E28000400A0091C1141091C2142091C31430911E
:10E29000C4140F5F1F4F2F4F3F4F60177107820746
:10E2A000930729F0D11003C08DE193E22AC06AE2FE
:10E2B00070E0C7010F94DE389C01009701F1982FA0
:10E2C0009E1910E0992339F09150F701E90FF11DE3
:10E2D00080811827F7CF4AE050E060E070E0C90184
:10E2E00001960F94F22D012F10E020E030E060172E
:10E2F00071078207930741F08EEF92E202C084ED2E
:10E3000092E20E944EF233CE80913D0A90913E0AF5
:10E31000A0913F0AB091400A8093C1149093C21417
:10E32000A093C314B093C41407C08091620F8823D4
:10E3300019F089E292E2E5CF80911802811121C0A3
:10E3400067E470E0C7010F94AF380097D1F04AE05E
:10E3500050E060E070E001960F94F22D643071059A
:10E3600080F4EDE5F2E284918F010F5F1F4F882367
:10E3700021F00F943D27F801F6CF60E083E592E2AB
:10E380009EDD61E081E49AE033DBE8CD2F35310595
:10E390000CF0E4CD9C35C1F40F94812897FDDECDBF
:10E3A0002091A10A2111DACD2091BF143091C0141F
:10E3B000A9014F5F5F4F5093C0144093BF14F90100
:10E3C000EF5BF54F8083CACD9B3319F481E08093D6
:10E3D000A10A8091A10A8111C1CDC9010196909332
:10E3E000C0148093BF14F901EF5BF54F4083B6CDA5
:10E3F0001092A20ACBCE0F90DF91CF911F910F9177
:10E40000FF90EF90DF90CF90BF90AF909F907F9064
:10E410006F905F904F900895CF93DF932091B31248
:10E4200021111EC0FC0101900020E9F73197EF0196
:10E43000C81BD90BC731D10534F031972081207C1E
:10E440002038D9F3F4CFBC01DD27AE0180EA9EE08D
:10E450000F94CF38C056D14F188283E08093450285
:10E46000DF91CF9108954F925F926F927F928F923A
:10E470009F92AF92BF92CF92DF92EF92FF920F9353
:10E480001F93CF93DF93CDB7DEB764970FB6F894A1
:10E49000DEBF0FBECDBF109117021F3F09F47BC036
:10E4A0000E947195C0901D0AD0901E0AE0901F0A2C
:10E4B000F090200ADC01CB018C199D09AE09BF093F
:10E4C000B7FD69C09091BB0E8091BA0E8F5F8F70BF
:10E4D000981709F460C0133009F493C2E0906F16E6
:10E4E00024E01202F0011124EC5FFC4F20E030E048
:10E4F00040E752E460817181828193810F945836A4
:10E500006D877E878F87988B198A1A8A1B8A1C8A47
:10E510008091661290916712A0916812B091691271
:10E5200089839A83AB83BC8380916A1290916B122A
:10E53000A0916C12B0916D128D839E83AF83B887CA
:10E5400080916E1290916F12A0917012B091711221
:10E5500089879A87AB87BC87AE01475F5F4FBE0153
:10E560006B5F7F4FCE0101960E948184AE014F5EAA
:10E570005F4F6A018E01035F1F4F22E732E148506F
:10E580005109BE016B5F7F4FCE0101960E94C54DC0
:10E590008FEF809317023CDC8091370A82FF3DC0E9
:10E5A0008091340A81113BC091E09093340A20910C
:10E5B000C315211103C08091330A89278093320A41
:10E5C0001092C31583E0809345021092370A0E948F
:10E5D0007195DC01CB018C509E4FAF4FBF4F8093A4
:10E5E000380A9093390AA0933A0AB0933B0A48E854
:10E5F00053E162E070E080E090E00F947E1D16E051
:10E60000115069F084E19FE00E94F3AE62E070E097
:10E6100080E090E00E943995F3CF1092340A89B1DE
:10E6200084FB992790F981E089271091310A81179D
:10E6300041F18093310A882309F4E9C164EF71E064
:10E6400080E090E00E948F9B0E948DF2123009F0D2
:10E65000DAC11092B60F8BE1EBEBFFE0AAEDBFE061
:10E6600001900D928A95E1F78091B90F9091BA0FC0
:10E670009093D90F8093D80F83E0809345020E9436
:10E6800040AF0E9471956B017C0180912D0A9091A1
:10E690002E0AA0912F0AB091300AA7019601281BDB
:10E6A000390B4A0B5B0B57FF05C08091980E8823EE
:10E6B00009F401C2D701C6018C599F4FAF4FBF4F1C
:10E6C00080932D0A90932E0AA0932F0AB093300ABC
:10E6D0008091350A082E000C990B97FF03C0919585
:10E6E0008195910982302CF48091320A811193C076
:10E6F000A3C080912C0A882309F466C08091350A52
:10E700008090280A9090290AA0902A0AB0902B0A9B
:10E7100081149104A104B10409F449C0082E000C2D
:10E72000990B97FF03C0919581959109682F87FFF9
:10E7300002C061E0680F6595062E000C770B880B10
:10E74000990B0F9418312B013C01C701B6016819D0
:10E7500079098A099B090F9416319B01AC01C30109
:10E76000B2010F94583620E030E04AE754E40F94A9
:10E7700077314B015C0120E030E040E253E40F943C
:10E78000A23787FF0FC020E030E046E952E4C50120
:10E79000B4010F94A23787FD0AC02AE030E040E0C0
:10E7A00050E009C024E630E040E050E004C021E041
:10E7B00030E040E050E0C092280AD092290AE0926E
:10E7C0002A0AF0922B0A04C021E030E040E050E039
:10E7D000A091350A0A2E000CBB0B0F94663522E07F
:10E7E00030E040E050E00F94403580919C0E9091D5
:10E7F0009D0EA0919E0EB0919F0E820F931FA41F9D
:10E80000B51F80939C0E90939D0EA0939E0EB09387
:10E810009F0E1092350AD701C6018856954CAF4F0E
:10E82000BF4F8093240A9093250AA093260AB093A1
:10E83000270A81E0809345022091460230914702E9
:10E8400046E42530340741F480914A02882309F4D4
:10E85000EAC0815080934A022C503C4E71F4809162
:10E860009C1290919D12891740F490914A0299232D
:10E8700009F4E9C0915090934A0280916F0081FBA6
:10E88000222720F981FF05C080916F008D7F809342
:10E890006F008091110490911204A0911304B09123
:10E8A0001404222329F020916F00226020936F002E
:10E8B0003AE0B695A795979587953A95D1F7009741
:10E8C00021E0A207B10520F08FEF9FEFA0E0B0E0BC
:10E8D0009695879520914502211105C03091980E9B
:10E8E0003111E5C059C0009741F04091220A509182
:10E8F000230A4817590708F04FC08091980E8111DC
:10E9000013C0223050F0243028F0243031F410921B
:10E91000450203C081E0809345020E94B8B581E0C2
:10E920008093210A8093980E84E00E949EAF81E03C
:10E9300080933312E0914602F091470219951092AC
:10E94000210A8091980E882351F00E944CB491E0E6
:10E95000811101C090E09093980E91118CC010929B
:10E96000320A8090220A9090230AA12CB12C0E9496
:10E970007195DC01CB018C199D09AE09BF09881680
:10E980009906AA06BB0640F40E9471956C197D0990
:10E990007093230A6093220A809146029091470265
:10E9A0008550964421F080919B0E882379F048E9A8
:10E9B000C40E4AE3D41EE11CF11CC092240AD0927A
:10E9C000250AE092260AF092270A0FC08091240AB5
:10E9D0009091250AA091260AB091270AC81AD90A4F
:10E9E000EA0AFB0AF7FE0E94EF4B8091980E811114
:10E9F00062C080914502813009F05DC010924502ED
:10EA00005AC0E12C6DCD60E08FE199E10AC010920F
:10EA1000640F1092650F123009F42ECE60E082E18F
:10EA200099E14DDA29CE8CE080934A028091220A46
:10EA30009091230A01979093230A8093220A81E000
:10EA40008093450209CF96E090934A0291E090931B
:10EA500045028F5F80939C12D701C6018856954C62
:10EA6000AF4FBF4F8093240A9093250AA093260AA4
:10EA7000B093270A02CF8090220A9090230AA12CFB
:10EA8000B12C0E947195DC01CB018C199D09AE0956
:10EA9000BF0988169906AA06BB0668F40E947195FC
:10EAA0006C197D097093230A6093220A04C00097B1
:10EAB00009F43ACF1ACF64960FB6F894DEBF0FBEB2
:10EAC000CDBFDF91CF911F910F91FF90EF90DF901D
:10EAD000CF90BF90AF909F908F907F906F905F90FE
:10EAE0004F900895CF92DF92EF92FF920F931F9372
:10EAF0000E9471950091190A10911A0A20911B0A1F
:10EB000030911C0A6B017C01C01AD10AE20AF30A97
:10EB1000F7FC13C02091180A20952093180ADC01F5
:10EB2000CB018A549C4FAF4FBF4F8093190A9093EB
:10EB30001A0AA0931B0AB0931C0A81E09091180A4C
:10EB4000911101C080E01F910F91FF90EF90DF9035
:10EB5000CF900895FC0180E090E02491222339F0C9
:10EB60002491207C203809F001963196F6CF089543
:10EB7000CF93DF93E8EFFAE48491EF0121968823A5
:10EB800021F00F943D27FE01F7CFE2E8F6E28491F1
:10EB9000EF012196882321F00F943D27FE01F7CF46
:10EBA000DF91CF9108950F931F93CF9383E5B3D84F
:10EBB000882309F442C011D8813039F0823009F03D
:10EBC0003CC000E013E0C0E01FC000E013E0C0E084
:10EBD000F80181918F019FD8882339F00E94ED6D53
:10EBE0004FEF682F8C2F0E943B61CF5FC43081F7BD
:10EBF00082E491D8882309F10E94ED6D4FEF682FD0
:10EC000019C0CF5FC43071F0F80181918F0183D8B2
:10EC10008823B9F30E94ED6D482F6FEF8C2F0E946F
:10EC20003B61EFCF82E477D8882339F00E94ED6D05
:10EC3000482F6FEF84E00E943B61CF911F910F91AD
:10EC40000C94249D0F931F93CF9383E51DD88111BE
:10EC500004C000E013E0C0E00EC0C0E00E94ED6D13
:10EC6000682F8C2F0E94DC9DCF5FC530B9F7F1CFA4
:10EC7000CF5FC43069F0F80181918F0105D88823F6
:10EC8000B9F30E94ED6D682F8C2F0E94DC9DF0CFB0
:10EC900082E40E94446E882331F00E94ED6D682F5B
:10ECA00084E00E94DC9DCF911F910F910C94249DD4
:10ECB000CF92DF92EF92FF92CF93DF938BE592E0BA
:10ECC0000E949FDE81117AC085E50E94446E8823F0
:10ECD000C1F1C0910D0BD0E00E940D6E6B017C0163
:10ECE00020E030E0A9010F94A23787FF04C0F7FAB3
:10ECF000F094F7F8F094CC0FDD1FCC0FDD1FCB5F45
:10ED0000DA4EC882D982EA82FB82C0910D0B84E080
:10ED1000C89FE0011124CB5FDA4E20E030E048E4E8
:10ED200053E4688179818A819B810F94A2371816F8
:10ED300044F480E090E0A8E4B3E488839983AA8354
:10ED4000BB838CE40E94446E8823C1F1C0910D0BFB
:10ED5000D0E00E940D6E6B017C0120E030E0A90143
:10ED60000F94A23787FF04C0F7FAF094F7F8F094F5
:10ED7000CC0FDD1FCC0FDD1FC75FDA4EC882D982F2
:10ED8000EA82FB82C0910D0B84E0C89FE001112450
:10ED9000C75FDA4E20E030E048E453E468817981CF
:10EDA0008A819B810F94A237181644F480E090E08A
:10EDB000A8E4B3E488839983AA83BB83DF91CF91CE
:10EDC000FF90EF90DF90CF900895CF92DF92EF9277
:10EDD000FF920F931F93CF93DF93CDB7DEB7A0972A
:10EDE0000FB6F894DEBF0FBECDBF80E090E0A8EC78
:10EDF000B2E489839A83AB83BC8380E090E0A6E988
:10EE0000B3E48D839E83AF83B88780E090E0A0EA6F
:10EE1000B1E489879A87AB87BC8788E592E00E9436
:10EE20009FDE8111BAC160910D0B0E941BF441E07D
:10EE300061E081E00E9439D9882319F081E00E94C5
:10EE4000ACDB85E40E94446E882381F00E940D6E45
:10EE50006B017C0120E030E0A9010F94A23787FF0D
:10EE60000AC0F7FAF094F7F8F09405C0C12CD12C41
:10EE7000E12C80E4F82EF7FAF094F7F8F094C98EBC
:10EE8000DA8EEB8EFC8E8AE50E948B6E882379F0F9
:10EE90008AE50E948B6E882319F00E940D6E03C0D4
:10EEA00060E070E0CB0169877A878B879C8788E573
:10EEB0000E948B6E882379F088E50E948B6E8823F0
:10EEC00019F00E940D6E03C060E070E0CB01698311
:10EED0007A838B839C8389E50E948B6E882379F0EB
:10EEE00089E50E948B6E882319F00E940D6E03C085
:10EEF00060E070E0CB016D837E838F83988785E52A
:10EF00000E94446E882329F00E940D6E6B017C01E3
:10EF10000CC0E0916F1684E0E89FF0011124EB5FD4
:10EF2000FA4EC080D180E280F38020E030E0A90179
:10EF3000C701B6010F94A23787FF04C0F7FAF09417
:10EF4000F7F8F094F7FAF094F7F8F094CD8ADE8AA7
:10EF5000EF8AF88E198A1A8A1B8A1C8A8CE40E940E
:10EF6000446E882329F00E940D6E6B017C010CC059
:10EF7000E0916F1694E0E99FF0011124E75FFA4EEB
:10EF8000C080D180E280F38020E030E0A901C70199
:10EF9000B6010F94A23787FF04C0F7FAF094F7F890
:10EFA000F094CD86DE86EF86F88A82E40E948B6E2E
:10EFB000882321F00E94DD6D162F01C01AE0009118
:10EFC000660B80918B0E8111E4C021E0AE014B5E97
:10EFD0005F4FBE016F5F7F4FCE0149960F940211C4
:10EFE000882309F4D6C060916F1682E00E941BF45A
:10EFF000EDE9F2E484917F019FEFE91AF90A882391
:10F0000021F00F943D27F701F5CFE6E5F6E2849174
:10F010007F019FEFE91AF90A882321F00F943D2719
:10F02000F701F5CF61E0812F0E9468FD0E94719584
:10F03000DC01CB0180529C46AB4FBF4F8093E00A6E
:10F040009093E10AA093E20AB093E30A1092970E1C
:10F0500083E08093E31481E08093C315DD24D3948F
:10F060008091C315882309F47AC060E0812F0E9443
:10F0700068FD8091970E882309F46DC060916F162A
:10F0800088E00E941BF4EDE9F2E484917F019FEF98
:10F09000E91AF90A882321F00F943D27F701F5CFEB
:10F0A000EFE2F6E284917F019FEFE91AF90A8823E3
:10F0B00021F00F943D27F701F5CF8091C3158823E8
:10F0C00021F081E00F94FA20F8CF1092E00A10921C
:10F0D000E10A1092E20A1092E30A1092970E0E943F
:10F0E000FC880F94F42B60916F1682E00E941BF451
:10F0F000EDE9F2E484917F019FEFE91AF90A882390
:10F1000021F00F943D27F701F5CFE3E0F6E284917B
:10F110007F019FEFE91AF90A811119C00E947195C8
:10F12000DC01CB0180529C46AB4FBF4F8093E00A7D
:10F130009093E10AA093E20AB093E30A1092970E2B
:10F14000D092C31561E0812F0E9468FD04C00F9426
:10F150003D27F701DCCF81E00F94FA2081CF81E0D9
:10F160008093E31480E090E0A0EAB1E48D8F9E8F5D
:10F17000AF8FB8A380918B0E882359F0212FAE0159
:10F18000435E5F4FBE01635F7F4FCE0141960F9498
:10F190004712013011F40E9466B1A0960FB6F894A0
:10F1A000DEBF0FBECDBFDF91CF911F910F91FF90BA
:10F1B000EF90DF90CF900895CF92DF92EF92FF9281
:10F1C000CF93DF938AE50E948B6E8823A9F10E947A
:10F1D0000D6E6B017C0120E030E040E050EC0F94BC
:10F1E000A23787FD13C020E030E040EA50E4C701B9
:10F1F000B6010F94123118164CF0C0927612D092CC
:10F200007712E0927812F092791241C0E8EFFAE4B6
:10F210008491EF01219681110BC0E8EEF5E2849113
:10F22000EF012196882399F10F943D27FE01F7CF36
:10F230000F943D27FE01ECCFEDE9F2E48491EF015C
:10F240002196882321F00F943D27FE01F7CFE9EDA9
:10F25000F5E28491EF012196882321F00F943D2758
:10F26000FE01F7CF4091761250917712609178129B
:10F270007091791286ED95E20F94E40E8AE0DF91A9
:10F28000CF91FF90EF90DF90CF900D943D27DF91CD
:10F29000CF91FF90EF90DF90CF900895CF93DF93C1
:10F2A00081E0809304150E9433C3109204158823D3
:10F2B000B1F0EDE9F2E48491EF012196882321F089
:10F2C0000F943D27FE01F7CFEBECF5E28491EF01BF
:10F2D0002196882321F00F943D27FE01F7CFDF917F
:10F2E000CF9108952F923F924F925F926F927F92AB
:10F2F0008F929F92AF92BF92CF92DF92EF92FF9246
:10F300000F931F93CF93DF93CDB7DEB763970FB6FD
:10F31000F894DEBF0FBECDBF41E061E081E00E9406
:10F3200039D98111CFC092E7892E9EE4992E86E6C5
:10F3300092E19A8B898BFE0131965F010BEC1EE402
:10F340001F01F3E0F00FFB8BF4016591759185913E
:10F350009491E989FA89C190D190E190F190FA8B6A
:10F36000E98BA70196010F947B352B013C0120E02E
:10F3700030E040EA51EC0F94A23787FD10C020E046
:10F3800030E040EA51E4C301B2010F941231181683
:10F3900034F0F10140825182628273820DC0F80123
:10F3A00084911816B4F7F7FAF094F7F8F094F10195
:10F3B000C082D182E282F382F101C190D190E190CA
:10F3C000F1901F0120E030E040EA51ECC701B601A6
:10F3D0000F94A23787FF03C0E8EFFAE40BC020E0E8
:10F3E00030E040EA51E4C701B6010F94123118161B
:10F3F0003CF5F2CF84918F010F5F1F4F882321F0DE
:10F400000F943D27F801F6CFEDEAF5E284918F01E4
:10F410000F5F1F4F882321F00F943D27F801F6CF8F
:10F4200061E08FE995E20E945F6F0E94EF4B88E2F6
:10F4300090E0988B8F8788EC90E09E878D873BC00B
:10F44000F4E08F0E911C0F5F1F4F8B8980137CCFD0
:10F450008DE7E82E8BE0F82E10E0F5018191919177
:10F46000A191B1915F01F70181939193A193B19320
:10F470007F01812F0E945FDE1F5F133071F70E94B2
:10F4800063FA60E08FE895E20E945F6F83E992E0A3
:10F49000988B8F8704E610E01E870D87BE01615FA1
:10F4A0007F4FCE010D960E94CEF38AEB92E0988BAF
:10F4B0008F871E870D87BE01615F7F4FCE010D963E
:10F4C0000E94CEF363960FB6F894DEBF0FBECDBF99
:10F4D000DF91CF911F910F91FF90EF90DF90CF9030
:10F4E000BF90AF909F908F907F906F905F904F9064
:10F4F0003F902F900895CF9380916F0081FBCC2790
:10F50000C0F981FF05C080916F008D7F80936F00EF
:10F510008091BB0E8093BA0E8093B90E8093B80E83
:10F5200084E68093B70E0E943F8788EE93E0909325
:10F53000EC038093EB03CC2329F080916F00826071
:10F5400080936F0081E080930B0A0E94755F0F9497
:10F55000462489E592E10E94C55F0F94F313CF9191
:10F560000C94876D2F923F924F925F926F927F9291
:10F570008F929F92AF92BF92CF92DF92EF92FF92C3
:10F580000F931F93CF93DF93CDB7DEB7CA55D10941
:10F590000FB6F894DEBF0FBECDBF85E40E948B6E20
:10F5A000882321F00E94DD6D7B0102C0E12CF12C4B
:10F5B00083E40E948B6E882321F00E94DD6D68A396
:10F5C00002C005E008A385E50E948B6E882319F030
:10F5D0000E94FE6D03C085E50E94446E8CA7F7FC77
:10F5E00007C0812C912C26E1A22E23E4B22E06C066
:10F5F000812C912C9CE8A92E92E4B92E83E50E94DF
:10F600008B6E882321F00E940D6E4B015C01E1148A
:10F61000F10411F410920D0B3E2C0E9471952B01F8
:10F620003C01E7FE07C00CE310E082E0D82E45E085
:10F6300050E006C008E210E0BAE0DB2E4AE050E0FD
:10F640005A83498361E06E0D623068F0E1E5F5E2CE
:10F6500084918F010F5F1F4F882309F411C50F9408
:10F660003D27F801F5CFEBE7F5E284917F015FEFED
:10F67000E51AF50A882321F00F943D27F701F5CF0D
:10F680000E94478937FE0CC087E680930C0B87E603
:10F6900090E0A0E0B0E08D839E83AF83B88710C078
:10F6A000E32D032C000CFF0BE55FF44F8FE7808305
:10F6B0002FE730E040E050E02D833E834F835887B2
:10F6C000C501B4010F94C036072E000C880B990BAE
:10F6D0000F94183169877A878B879C874D2D50E06E
:10F6E0009801A8EEB3E00F946C356DA77EA78FA7A5
:10F6F00098ABDC01CB01840D951DA61DB71D89AF0C
:10F700009AAFABAFBCAF81E080935D0237FE05C01E
:10F710008EEC90E0A0E0B0E004C08FEF90E0A0E0BD
:10F72000B0E08C019D010351110921093109239693
:10F730000CAF1DAF2EAF3FAF23978C019D0104513D
:10F7400011092109310927960CAF1DAF2EAF3FAF2C
:10F7500027978C019D0135952795179507952B9631
:10F760000CAF1DAF2EAF3FAF2B978C019D01015009
:10F770001109210931092F960CAF1DAF2EAF3FAFF4
:10F780002F978D809E80AF80B8844CA25DA26EA220
:10F790007FA249AA5AAA6BAA7CAA1BA21DAA1EAACA
:10F7A0001FAA18AE10E000E40F8B0CE1088F06E4EE
:10F7B000098F1A8E1B8E1C8E1D8E1B8A1C8A1D8A19
:10F7C0001E8A1F86188A198A1A8AC12CD12C7601A2
:10F7D00018A619A61AA61BA601E00AA31E861D8656
:10F7E0006A961FAE6A97212C00E06B961FAE6B974E
:10F7F000832D032C000C990B9C01255F344F3EAFE9
:10F800002DAF880F991F880F991FDC01A559B94E9C
:10F81000BF8FAE8FCA01052E000CAA0BBB0B6396DF
:10F820008CAF9DAFAEAFBFAF6397A981BA814A0FCE
:10F830005B1F4F5F5F4FCA01550FAA0BBB0B67964B
:10F840008CAF9DAFAEAFBFAF6797A8A10A2E000CDB
:10F85000BB0BB9A3A8A380915D02882309F4EFC074
:10F860000E94719569837A838B839C838091F40ACB
:10F87000882309F4C4C00E94058A37FE0FC0009196
:10F880000E0B6A960FAF6A9720900F0B0091100B2A
:10F890002091110B6B962FAF6B970EC0AE8DBF8D65
:10F8A000BC916A96BFAF6A97EE8DFF8D2180028171
:10F8B000F3816B96FFAF6B976A962FAD6A97322DE7
:10F8C000402F6B965FAD6B976A8D7B8D8C8D9D8D78
:10F8D0000F94123187FF0AC06A962FAD6A972A8F5C
:10F8E0002B8E0C8F6B963FAD6B973D8F6A962FAD2D
:10F8F0006A97322D402F6B965FAD6B97612F7F8992
:10F90000888D998D0F94A23718164CF46A961FAD06
:10F910006A972F8A088F6B964FAD6B97498F5AA1C4
:10F9200029853A854B85552309F448C05C856A963C
:10F930006FAD6A97722D802F6B969FAD6B970F946A
:10F94000A23718160CF05BC049815A816B817C810B
:10F950004419550966097709DB01CA0188589341A2
:10F96000A109B109B7FD4BC08D819E81AF81B885DA
:10F9700088199909AA09BB09B595A79597958795FF
:10F9800037FE03C080930C0B03C0EDADFEAD80834A
:10F9900048A759A76AA77BA7F985FA8F2A852B8FD5
:10F9A0003B853C8F4C854D8F89819A81AB81BC8191
:10F9B0008CA39DA3AEA3BFA31AA221C05C856A96A7
:10F9C0006FAD6A97722D802F6B969FAD6B970F94DA
:10F9D000123187FF14C089819A81AB81BC812CA12F
:10F9E0003DA14EA15FA1821B930BA40BB50BAC01F3
:10F9F000BD01485853416109710977FFCDC120E02D
:10FA000030E040EA51E469857A858B859C850F94C6
:10FA10007C359B01AC016A966FAD6A97722D802F81
:10FA20006B969FAD6B970F94A23718163CF5EDEDD2
:10FA3000F4E284918F010F5F1F4F81111BC0C65AE2
:10FA4000DF4F0FB6F894DEBF0FBECDBFDF91CF9171
:10FA50001F910F91FF90EF90DF90CF90BF90AF90EC
:10FA60009F908F907F906F905F904F903F902F90DE
:10FA70000C9447890F943D27F801DBCF89819A8147
:10FA8000AB81BC8129A93AA94BA95CA9821B930B24
:10FA9000A40BB50BB7FDAEC00E94F7878AE00F94A8
:10FAA0003D2789819A81AB81BC818053984FAF4FAC
:10FAB000BF4F89AB9AABABABBCAB9BA1911175C0EF
:10FAC0002DA93EA94FA958AD6A966FAD6A97722DC0
:10FAD000802F6B969FAD6B970F94A23718160CF082
:10FAE0004BC063966CAD7DAD8EAD9FAD63970F94AB
:10FAF00018319B01AC016A966FAD6A97722D802F09
:10FB00006B969FAD6B970F947C356DAB7EAB8FABD7
:10FB100098AF29813A814B815C818DA59EA5AFA5C7
:10FB2000B8A9280F391F4A1F5B1F29AF3AAF4BAF47
:10FB30005CAF67966CAD7DAD8EAD9FAD67970F9452
:10FB400018319B01AC0169857A858B859C850F9462
:10FB50007B359B01AC0191E09BA36A966FAD6A97E0
:10FB6000722D802F6B969FAD6B970F94A23718164E
:10FB70000CF440C01BA23EC089819A81AB81BC813C
:10FB800029AD3AAD4BAD5CAD821B930BA40BB50B0D
:10FB9000B7FD30C03FEF331619F049EA54E202C016
:10FBA0004BEB54E26EEC74E222C020E030E040EA1D
:10FBB00051E469857A858B859C850F947B359B0103
:10FBC000AC016A966FAD6A97722D802F6B969FADD0
:10FBD0006B970F94123187FF0DC04FEF341619F059
:10FBE00042E754E202C045E854E269E974E2832D39
:10FBF0000E94248A89819A81AB81BC81880F991FD8
:10FC0000AA1FBB1F2CA13DA14EA15FA1821B930B7C
:10FC1000A40BB50B84199509A609B70981389F442F
:10FC2000A241B10568F0E4E5F4E284918F010F5F31
:10FC30001F4F882309F403CF0F943D27F801F5CF18
:10FC40004D855E8588A199A1841795070CF0A1C008
:10FC5000E7EFF3E284918F010F5F1F4F882321F0BC
:10FC60000F943D27F801F6CF37FC03C00BEF12E0ED
:10FC700002C004E113E0B80186EE93E20F941A0F7C
:10FC8000B701A60182EE93E20F94E40E8AE00F948E
:10FC90003D27B80181ED93E20F941A0F4F855889E3
:10FCA00069897A898DEC93E20F94E40E8AE00F94CF
:10FCB0003D27B8018CEB93E20F941A0F4B895C89B6
:10FCC0006D897E8988EB93E20F94E40E8AE00F94AD
:10FCD0003D270CA5002309F4D3C137FE2DC0C092E7
:10FCE0001915D0921A15E0921B15F0921C152CEAEA
:10FCF00035EC47E25EE36F85788989899A890F94AC
:10FD0000773160931515709316158093171590939E
:10FD100018152CEA35EC47E25EE36B897C898D8906
:10FD20009E890F9458366093111570931215809325
:10FD3000131590931415A4C1C0922515D0922615C1
:10FD4000E0922715F09228152CEA35EC47E25EE3A5
:10FD50006F85788989899A890F9477316093211505
:10FD60007093221580932315909324152CEA35EC7B
:10FD700047E25EE36B897C898D899E890F945836B2
:10FD800060931D1570931E1580931F159093201579
:10FD900077C10E9433725FCD4D855E85452B09F496
:10FDA00032C148A459A46AA47BA4480E591E6A1EF5
:10FDB0007B1E28A539A54AA55BA5281B390B4A0B34
:10FDC0005B0BCA01B901A50194010F940F35A30182
:10FDD00092010F9440358D809E80AF80B884820E52
:10FDE000931EA41EB51E34E183169104A104B10430
:10FDF0000CF438C123968CAD9DADAEADBFAD23974D
:10FE000088169906AA06BB060CF025C12B962CADC8
:10FE10003DAD4EAD5FAD2B97281539054A055B0505
:10FE20008CF48D829E82AF82B8862F968CAD9DAD6C
:10FE3000AEADBFAD2F9788199909AA09BB094C012E
:10FE40005D0104C08D829E82AF82B886E9E4F5E24E
:10FE500084919F012F5F3F4F882381F068962FAFD9
:10FE6000689769963FAF69970F943D2768962FADC5
:10FE7000689769963FAD6997F901EACF6D817E81F8
:10FE80008F8198850F94F627E4E4F5E284919F0131
:10FE90002F5F3F4F882381F068962FAF6897699650
:10FEA0003FAF69970F943D2768962FAD6897699685
:10FEB0003FAD6997F901EACFC501B4010F94F62768
:10FEC000412F5F89688D798D8DE395E20F94E40E63
:10FED0004A8D5B8D6C8D7D8D86E395E20F94E40EEB
:10FEE000AD85BE8513970CF48EC0C501B4010F9487
:10FEF000183120E030E040E850E40F9477316B0196
:10FF00007C01212F3F89488D598D6A8D7B8D8C8D89
:10FF10009D8D0F947B352BED3FE049E450E40F9429
:10FF2000773120E030E040E05FE30F9477319B01D0
:10FF3000AC01C701B6010F9458366B017C01C301B7
:10FF4000B2010F9418312FE632E143E85AE30F94DF
:10FF500077312B013C01B701A60180E395E20F94B4
:10FF6000E40EB301A2018AE295E20F94E40E2AE9BD
:10FF700039E949E15FE3C701B6010F9477316B01BD
:10FF80007C019B01AC010F947C35A30192010F947D
:10FF900058366F87788B898B9A8BA3019201C701A2
:10FFA000B6010F94773120E030E040E05EE30F943B
:10FFB00077316B8B7C8B8D8B9E8BEAE1F5E28491A4
:10FFC0003F01BFEF6B1A7B0A882321F00F943D2776
:10FFD000F301F5CFB701A60184E195E20F94E40E99
:10FFE0004F85588969897A898EE095E20F94E40EED
:10FFF0004B895C896D897E8988E095E20F94E40ED7
:020000021000EC
:100000008AE00F943D278D819E81AF81B885880D50
:10001000991DAA1DBB1DB595A7959795879537FE88
:1000200003C080930C0B03C0EDADFEAD80832D8526
:100030003E852F5F3F4F3E872D8719853A853F8B41
:100040004B85488F5C85598F49805A806B807C80B6
:1000500081E08AA3D4CC27968CAC9DACAEACBFAC6F
:100060002797DFCE84E1882E912CA12CB12C24E19E
:1000700030E040E050E02D833E834F835887E6CE4A
:10008000C65ADF4F0FB6F894DEBF0FBECDBFDF916B
:10009000CF911F910F91FF90EF90DF90CF90BF9085
:1000A000AF909F908F907F906F905F904F903F9018
:1000B0002F900895CF93DF9383E50E94446EC82F5D
:1000C000882371F00E940D6E0F94C03670935F020A
:1000D00060935E0221E0672B09F020E02093701608
:1000E00080E50E94446E882359F020915E02309191
:1000F0005F02232B11F00E94FE6D809370162DC0BD
:10010000C1112BC0EDE9F2E48491EF01219688231F
:1001100021F00F943D27FE01F7CF809170168111D9
:1001200003C068E173E002C06BEE72E085EA93E21F
:100130000F941A0F60915E0270915F0284E993E25E
:100140000F94010FE0E9F3E28491EF0121968823F7
:1001500021F00F943D27FE01F7CFDF91CF91089555
:10016000CF93DF9380E50E94446E882351F00E9474
:100170000D6E6093191570931A1580931B1590934B
:100180001C1589E40E94446E882381F00E940D6E44
:100190002CEA35EC47E25EE30F9477316093151556
:1001A00070931615809317159093181584E40E9488
:1001B000446E882381F00E940D6E2CEA35EC47E2F4
:1001C0005EE30F9458366093111570931215809367
:1001D000131590931415EDE9F2E48491EF01219643
:1001E000882321F00F943D27FE01F7CF4091191588
:1001F00050911A1560911B1570911C158CE893E2B3
:100200000F94E40E2CEA35EC47E25EE3609115159D
:100210007091161580911715909118150F945836F6
:10022000AB01BC0188E893E20F94E40E2CEA35ECB4
:1002300047E25EE3609111157091121580911315DC
:10024000909114150F947731AB01BC0184E893E2CF
:100250000F94E40E8AE0DF91CF910D943D270F9328
:100260001F93CF93DF938DED90E00E949FDE81116D
:1002700066C083E50E948B6E8823B9F1C0910D0B97
:10028000D0E00E94DD6DCC0FDD1FC25EDD4F7983B3
:10029000688380910D0B90E0EC01CC0FDD1FCC0F3B
:1002A000DD1F8E010A5F1D4F880F991FFC01E25E62
:1002B000FD4F60817181072E000C880B990B0F9404
:1002C00018312AE037ED43E25CE30F947731CC5EDE
:1002D000D44F288139814A815B810F947731F801AD
:1002E00060837183828393832AC0EDE9F2E4849171
:1002F000EF012196882321F00F943D27FE01F7CFCF
:1003000085E40F943D2780910D0B805D0F943D2770
:10031000E0910D0BF0E0EE0FFF1FE25EFD4F6081FC
:1003200071818CE793E20F94010F85E20F943D27D2
:100330008AE0DF91CF911F910F910D943D27DF91BE
:10034000CF911F910F91089583E50E948B6E8823B2
:1003500031F00E94DD6D70930102609300020895F8
:100360004F925F926F927F928F929F92AF92BF92C5
:10037000CF92DF92EF92FF92CF93DF93CDB7DEB7AC
:100380002C970FB6F894DEBF0FBECDBF80910E0B39
:1003900090910F0BA091100BB091110B89839A8350
:1003A000AB83BC836091120B7091130B072E000C72
:1003B000880B990B0F94183129813A814B815C810C
:1003C0000F947B356B017C016093D20A7093D30A42
:1003D0008093D40A9093D50A2091191530911A155B
:1003E00040911B1550911C150F9477316D837E83BE
:1003F0008F8398876093CE0A7093CF0A8093D00A38
:100400009093D10A2091CA0A3091CB0A4091CC0A2C
:100410005091CD0AC701B6010F947C354B015C01A8
:100420006093CA0A7093CB0A8093CC0A9093CD0A4A
:1004300020911515309116154091171550911815EA
:100440000F94773169877A878B879C876093C60A78
:100450007093C70A8093C80A9093C90A20ED3CECB8
:100460004CE45DE3609111157091121580911315A4
:10047000909114150F9477312B013C012091C20A01
:100480003091C30A4091C40A5091C50A69817A81AA
:100490008B819C810F947B359B01AC01C301B20120
:1004A0000F9477312B013C0123E333E343E75FE310
:1004B0006091BE0A7091BF0A8091C00A9091C10AF2
:1004C0000F9477319B01AC01C301B2010F947C35CD
:1004D0002B013C016093BE0A7093BF0A8093C00A4F
:1004E0009093C10A89819A81AB81BC818093C20AB1
:1004F0009093C30AA093C40AB093C50A29853A858C
:100500004B855C856D817E818F8198850F947C35CC
:10051000A30192010F947B352B013C0120E030E0D8
:100520004EE453E40F94A23720E030E0A9011816FE
:10053000ACF4C701B6010F94A23718166CF5A701E9
:100540009601C501B4010F947B356093CA0A70937C
:10055000CB0A8093CC0A9093CD0A1EC0C301B2018E
:100560000F94123187FF22C020E030E0A901C701BB
:10057000B6010F94123187FF16C0A7019601C5017D
:10058000B4010F947B356093CA0A7093CB0A8093B1
:10059000CC0A9093CD0A07C0412C512C8EE4682ED2
:1005A00083E4782E03C0412C512C3201C301B201E7
:1005B0002C960FB6F894DEBF0FBECDBFDF91CF9162
:1005C000FF90EF90DF90CF90BF90AF909F908F9073
:1005D0007F906F905F904F9008952F923F924F922F
:1005E0005F926F927F928F929F92AF92BF92CF92C3
:1005F000DF92EF92FF92CF93DF9300D01F92CDB79F
:10060000DEB7609071167090721680906B169090A5
:100610006C16A0906D16B0906E16B301072C000CEE
:10062000880B990B0F941831A50194010F947B3519
:100630006B017C016093BA0A7093BB0A8093BC0A79
:100640009093BD0A20ED3CEC4CE45DE360911D15F8
:1006500070911E1580911F15909120150F94773180
:100660001B012C012091B60A3091B70A4091B80ABB
:100670005091B90AC501B4010F947B359B01AC01BF
:10068000C201B1010F9477311B012C0123E333E345
:1006900043E75FE36091B20A7091B30A8091B40AB4
:1006A0009091B50A0F9477319B01AC01C201B10161
:1006B0000F947C3569837A838B839C836093B20A21
:1006C0007093B30A8093B40A9093B50A8092B60AE5
:1006D0009092B70AA092B80AB092B90A8091970E88
:1006E000882321F081E08093B10AB9C020E030E096
:1006F00040E251E4C701B6010F94A237181624F462
:1007000081E08093B10AA4C020E030E040E251ECE7
:10071000C701B6010F94123187FDE4CF672811F3AA
:100720008091B10A882351F01092AD0A1092AE0A5E
:100730001092AF0A1092B00A1092B10A20912515BA
:10074000309126154091271550912815C701B60103
:100750000F9477312B013C016093A90A7093AA0A88
:100760008093AB0A9093AC0A2091AD0A3091AE0A07
:100770004091AF0A5091B00AC701B6010F947C3581
:100780004B015C016093AD0A7093AE0A8093AF0A8F
:100790009093B00A20912115309122154091231594
:1007A000509124150F9477319B01AC016093A50AF9
:1007B0007093A60A8093A70A9093A80AC301B20176
:1007C0000F947C3529813A814B815C810F947B3574
:1007D0002B013C0120E030E04FE753E40F94A237B7
:1007E00020E030E0A9011816ACF4C701B6010F945F
:1007F000A23718166CF5A7019601C501B4010F9434
:100800007B356093AD0A7093AE0A8093AF0A9093E4
:10081000B00A1EC0C301B2010F94123187FF22C07B
:1008200020E030E0A901C701B6010F94123187FF23
:1008300016C0A7019601C501B4010F947B356093E2
:10084000AD0A7093AE0A8093AF0A9093B00A07C0C6
:10085000412C512C8FE7682E83E4782E03C0412C65
:10086000512C3201C301B2010F900F900F900F90E5
:10087000DF91CF91FF90EF90DF90CF90BF90AF903E
:100880009F908F907F906F905F904F903F902F90B0
:100890000895EF92FF920F931F93CF93DF931F92D0
:1008A000CDB7DEB78C017B0180E249830F943D27F1
:1008B00049814F3F11F084E501C082E40F943D2748
:1008C0008AE30F943D27F8016081718182819381D1
:1008D00042E00F941028F7014081518162817381B9
:1008E0008AED98E20F94E40E62E070E080E090E020
:1008F0000F90DF91CF911F910F91FF90EF900C948B
:100900003995CF92DF92EF92FF920F931F93CF937F
:10091000DF93CDB7DEB728970FB6F894DEBF0FBED2
:10092000CDBF20913515222309F462C0C52ED42EE7
:100930008B017C0120E030E048E951E4FC0160815A
:100940007181828193810F947C356D837E838F8347
:10095000988720E030E041E853E4F801608171813C
:10096000828193810F947B3569837A838B839C8307
:10097000CF92DF92CE0101969F938F9304969F931F
:100980008F938DB79EB784970FB6F8949EBF0FBE16
:100990008DBFADB7BEB7119684E2ECEBFEE00190DF
:1009A0000D928A95E1F70F94420F20E030E048E97C
:1009B00051E46D817E818F8198850F947B35F7019D
:1009C000608371838283938320E030E041E853E4C5
:1009D00069817A818B819C810F947C35F8016083D9
:1009E0007183828393830FB6F894DEBF0FBECDBFB1
:1009F00028960FB6F894DEBF0FBECDBFDF91CF9122
:100A00001F910F91FF90EF90DF90CF900895CF92BC
:100A1000DF92EF92FF9280918215882371F1C0904E
:100A20007E15D0907F15E0908015F090811520E024
:100A300030E0A901C701B6010F9412318823E9F013
:100A400020E030E040E05FE3C701B6010F9477316A
:100A50009B01AC010F9477312BED3FE049E450E46A
:100A60000F9477319B01AC0160E070E080E89FE378
:100A70000F9458366B017C0106C0C12CD12C80E844
:100A8000E82E8FE3F82EC092140BD092150BE09253
:100A9000160BF092170B60911E0270911F02072E29
:100AA000000C880B990B0F9418312AE037ED43E2C4
:100AB0005CE30F947731A70196010F94773160932F
:100AC0000602709307028093080290930902FF9038
:100AD000EF90DF90CF9008954F925F926F927F9248
:100AE0008F929F92AF92BF92CF92DF92EF92FF923E
:100AF0000F931F93CF93DF93CDB7DEB768970FB6F1
:100B0000F894DEBF0FBECDBF8C015B014A01FC0132
:100B1000EE5BFF4F60817181828193810F9416316A
:100B20006B017C01D5012D913D914D915C910F940C
:100B300077310F9442360F94C53669877A878B8751
:100B40009C87F4012081318142815381C701B60124
:100B50000F9477310F9442360F94C5366D877E8798
:100B60008F87988B29853A854B855C852837310599
:100B70004105510540F488E790E0A0E0B0E08987A6
:100B80009A87AB87BC872D853E854F855889283746
:100B900031054105510540F488E790E0A0E0B0E060
:100BA0008D879E87AF87B88B9801225B3F4FD90115
:100BB0008D919D910D90BC91A02D89839A83AB83DB
:100BC000BC83BC01CD010F9418312B013C01698518
:100BD0007A858B859C850F941631698B7A8B8B8BEC
:100BE0009C8B20E030E0A901C301B2010F941231C7
:100BF000882329F1A7019601C701B6010F94773127
:100C00004B015C0129893A894B895C89CA01B90188
:100C10000F9477319B01AC01C501B4010F947B3572
:100C20004B015C01A3019201C301B2010F947C3519
:100C30009B01AC01C501B4010F94583603C060E0BC
:100C400070E0CB010F9442360F94C5366D837E83DE
:100C50008F83988769817A818B819C81909580951B
:100C6000709561957F4F8F4F9F4F0F9418314B01B7
:100C70005C016D857E858F8598890F941631698317
:100C80007A838B839C8320E030E0A901C501B40105
:100C90000F941231882349F129813A814B815C817B
:100CA000CA01B9010F9477316D8B7E8B8F8B988F32
:100CB000A7019601C701B6010F9477319B01AC01E2
:100CC0006D897E898F89988D0F947B356B017C01AE
:100CD000A5019401C501B4010F947C359B01AC01C1
:100CE000C701B6010F94583603C060E070E0CB0135
:100CF0000F94F136F80185A096A0A7A0B0A47501C5
:100D000064012D813E814F815885C21AD30AE40ABD
:100D1000F50A0F94C536C61AD70AE80AF90AF7FE8B
:100D200073C020E030E0A901C301B2010F94123179
:100D3000882309F443C0A3019201C301B2010F94B7
:100D40007C356B017C01C501B4010F9416319B0108
:100D5000AC01C701B6010F9477316B017C01298981
:100D60003A894B895C89CA01B9010F9477319B019B
:100D7000AC01C701B6010F947B356B017C01298161
:100D80003A814B815C81CA01B9010F9477319B0193
:100D9000AC01C701B6010F947C356B017C0120E0EA
:100DA00030E040E850E4C301B2010F9477319B0179
:100DB000AC01C701B6010F94583603C060E070E083
:100DC000CB010F9442367B016C0120E030E0A90199
:100DD0000F94A237181624F0E12CF12CC12CD12C41
:100DE000B701C6010F94C5366D837E838F839887C4
:100DF00086169706A806B90620F48D829E82AF82D9
:100E0000B886C12CD12C76018D819E81AF81B885A9
:100E1000F80182A793A7A4A7B5A7C80ED91EEA1EFA
:100E2000FB1EC6A6D7A6E0AAF1AAEA5BFF4F29855A
:100E30003A854B855C852083318342835383349686
:100E40008D859E85AF85B88980839183A283B38386
:100E500068960FB6F894DEBF0FBECDBFDF91CF917D
:100E60001F910F91FF90EF90DF90CF90BF90AF90C8
:100E70009F908F907F906F905F904F90089580919A
:100E80006F0081FB992790F981FF05C080916F0069
:100E90008D7F80936F0010921104109212041092B3
:100EA000130410921404992329F080916F0082603A
:100EB00080936F0008954F925F926F927F928F920E
:100EC0009F92AF92BF92CF92DF92EF92FF920F93D9
:100ED0001F93CF93DF933C01B0E2A0E06A2F70E054
:100EE000AB014B0F511D559547954A1711F04B1308
:100EF0000BC0EFE0F7E265917491072E000C880BB0
:100F0000990B0F94183162C0CA010197880F991F7D
:100F1000880F991FFC01EF56F94D059114919A0124
:100F2000220F331F220F331FF901EF56F94DC591E0
:100F3000D4916016710614F4B42FD2CFA42FC61525
:100F4000D7050CF4CBCF8D56994DFC01E590F4906C
:100F5000F901ED56F94DC590D490B7010F2C000C56
:100F6000880B990B0F9418314B015C01B301601B86
:100F7000710B072E000C880B990B0F9418312B0165
:100F80003C01B6016E197F09072E000C880B990BE6
:100F90000F9418319B01AC01C301B2010F9477315A
:100FA0006B017C01C01BD10BBE01DD0F880B990BBF
:100FB0000F9418319B01AC01C701B6010F9458364C
:100FC0009B01AC01C501B4010F947C35DF91CF9139
:100FD0001F910F91FF90EF90DF90CF90BF90AF9057
:100FE0009F908F907F906F905F904F9008950F9398
:100FF0001F93CF93DF93CDB7DEB728970FB6F89442
:10100000DEBF0FBECDBF6091711670917216072EB4
:10101000000C880B990B0F9418316D837E838F839E
:10102000988780916B1690916C16A0916D16B09177
:101030006E1689839A83AB83BC834DEFBE016B5FD1
:101040007F4FCE01019625DC6091120B7091130B3E
:10105000072E000C880B990B0F9418316D837E833B
:101060008F83988780910E0B90910F0BA091100B9E
:10107000B091110B89839A83AB83BC834FEFBE0180
:101080006B5F7F4FCE01019604DCE2EEF8E28491C3
:101090008F010F5F1F4F882321F00F943D27F80128
:1010A000F6CFE0910D0BF0E0E55FF44F608170E06A
:1010B00080E090E00F94F627EDEDF8E284918F0147
:1010C0000F5F1F4F882321F00F943D27F801F6CFC3
:1010D00060910C0B70E080E090E00F94F62728966A
:1010E0000FB6F894DEBF0FBECDBFDF91CF911F9139
:1010F0000F9108950F930FB70F9300916E000B7F20
:1011000000936E0078940F930BB70F930CB70F9268
:101110001F922F933F934F935F936F937F938F9380
:101120009F93AF93BF93EF93FF9311240DD2FF9141
:10113000EF91BF91AF919F918F917F916F915F914F
:101140004F913F912F911F900F900CBF0F910BBFAC
:101150000F910460F89400936E000F910FBF0F91F0
:101160001895CF92DF92EF92FF92C0900E0BD09025
:101170000F0BE090100BF090110B8091120B9091DF
:10118000130B0897BC01990F880B990B0F9418311A
:101190009B01AC01C701B6010F94123187FF1FC03C
:1011A00020E030E040E050E4C701B6010F947C3508
:1011B0000F94C5367093EF0A6093EE0A0E94719502
:1011C000DC01CB01805A9541AF4FBF4F8093EA0AB3
:1011D0009093EB0AA093EC0AB093ED0A08C010922A
:1011E000EA0A1092EB0A1092EC0A1092ED0AFF90B4
:1011F000EF90DF90CF900895CF92DF92EF92FF9221
:10120000C0906B16D0906C16E0906D16F0906E1634
:1012100080917116909172164597BC01990F880BB9
:10122000990B0F9418319B01AC01C701B6010F94C3
:10123000123187FF1FC020E030E040E251E4C701D7
:10124000B6010F947C350F94C5367093E90A60930C
:10125000E80A0E947195DC01CB01805C9346AF4F98
:10126000BF4F8093E40A9093E50AA093E60AB093F7
:10127000E70A08C01092E40A1092E50A1092E60A02
:101280001092E70AFF90EF90DF90CF9008951092B0
:1012900072161092711680E0AFDF1092130B10924D
:1012A000120B5FDF0E94C3B110927216109271167A
:1012B00080E0A2DF10920B0B80910201807480937A
:1012C00000011092130B1092120B10920C0B7598D8
:1012D00008954F925F926F927F928F929F92AF92FA
:1012E000BF92CF92DF92EF92FF920F931F93CF9313
:1012F000DF933C01BAE3A0E06A2F70E0AB014B0F33
:10130000511D559547954A1711F04B130BC0E6E652
:10131000F8E265917491072E000C880B990B0F94DD
:10132000183162C0CA010197880F991F880F991F51
:10133000FC01E058F84D059114919A01220F331FDA
:10134000220F331FF901E058F84DC591D491601672
:10135000710614F4B42FD2CFA42FC615D7050CF400
:10136000CBCF8E57984DFC01E590F490F901EE57E4
:10137000F84DC590D490B7010F2C000C880B990B39
:101380000F9418314B015C01B301601B710B072EE8
:10139000000C880B990B0F9418312B013C01B601FE
:1013A0006E197F09072E000C880B990B0F941831CA
:1013B0009B01AC01C301B2010F9477316B017C0139
:1013C000C01BD10BBE01DD0F880B990B0F94183198
:1013D0009B01AC01C701B6010F9458369B01AC01CB
:1013E000C501B4010F947C35DF91CF911F910F910E
:1013F000FF90EF90DF90CF90BF90AF909F908F9035
:101400007F906F905F904F90089560E08091F20A16
:101410009091F30A50DD60936B1670936C16809375
:101420006D1690936E168091F00A9091F10A51DF3B
:1014300060930E0B70930F0B8093100B9093110B16
:10144000A8951092F40A0895CF92DF92FF920F931D
:101450001F93CF93DF931F921F92CDB7DEB7F82E65
:101460008A0180911802882309F444C0E8EFFAE465
:1014700084916F019FEFC91AD90A882341F06983CB
:101480007A830F943D27F60169817A81F1CFFB01C0
:1014900084916F019FEFC91AD90A882321F00F9414
:1014A0003D27F601F5CFE6E1F7E284916F019FEF6A
:1014B000C91AD90A882321F00F943D27F601F5CFE8
:1014C000F7FC0BC06F2DFF0C770B880B990B0F945B
:1014D000F6278AE00F943D270DC0E1E1F7E2849101
:1014E0006F019FEFC91AD90A882321F00F943D2775
:1014F000F601F5CF8091A40A811108C0109218025C
:1015000081E08093A40AC8010F94F2150F900F9008
:10151000DF91CF911F910F91FF90DF90CF90B7CEC9
:101520008F3F19F04BE958E202C04BEA58E26CEBEE
:1015300078E28ACF8F3F19F048E658E202C048E7C8
:1015400058E269E878E280CF0F931F93CF93DF933F
:1015500080911D028F37A0F08F5720910B0B2093A5
:101560000A0B9091020121119095907490930001C3
:1015700090910C0B9093090B992379F0759A0EC0FA
:1015800090910A0B891728F0909102019074909322
:1015900000019091090B891708F075988F5F80936F
:1015A0001D029091080B81E089278093080B81111F
:1015B0000E94086F80911C02853018F4C1E0C80FAA
:1015C00001C0C0E0823009F4ACC048F48823F9F0CF
:1015D000813009F0DAC010927B0080E4B8C084301A
:1015E00009F4BDC008F4B0C0853009F0CEC09091B8
:1015F000070B911102C08093070B8091070B81505C
:101600008093070B882309F4C0C0C5E0BEC0809159
:101610001B028F5F80311CF480931B02B6C01092B6
:101620001B028091F40A811113C08091FD0A9091F0
:10163000FE0A9093F30A8093F20A8091FB0A90913C
:10164000FC0A9093F10A8093F00A81E08093F40AF7
:101650008AE0EDEFFAE0DF011D928A95E9F710923A
:10166000FC0A1092FB0A0091F20A1091F30A1195FC
:1016700001951109D1E080910B0B811101C0D0E0DF
:101680008091560B9091570B9195819591098017F8
:10169000910744F4DD2331F048E658E269E878E246
:1016A00080E0D2DE80913302909134029195819551
:1016B00091090817190744F4DD2331F04BE958E28A
:1016C0006CEB78E280E0C0DE11E080910C0B8111C0
:1016D00001C010E02091F00A3091F10A8091540B82
:1016E0009091550B8217930744F0112331F048E78E
:1016F00058E269E878E28FEFA7DE2091310230915D
:1017000032028091F00A9091F10A82179307ECF16E
:101710001123D9F14BEA58E26CEB78E28FEF94DEBB
:1017200034C080917A0086FD2DC080917800909120
:1017300079002091FD0A3091FE0A820F931F909349
:10174000FE0A8093FD0A21C010927B0082E4809300
:101750007C0080917A00806480937A0016C080912A
:101760007A0086FD11C080917800909179002091D7
:10177000FB0A3091FC0A820F931F9093FC0A80931E
:10178000FB0A03C0C2E001C0C4E0C0931C0220E019
:1017900030E0A1E0B4E0C901880F991FFC01EB50D3
:1017A000F54F608171816115710509F436C0F894B7
:1017B000223001F5509109015470159840910B01A8
:1017C000161617060CF4409544704093090100006A
:1017D00000004A2F4A950000E9F7429A4B2F4A959C
:1017E0000000E9F7429840910B0151114095447077
:1017F000409309017894FC01EB50F54F161617063B
:101800003CF440815181415051095183408305C0CE
:10181000808191810196918380832F5F3F4F233098
:10182000310509F0B8CF0E944DB08091EB03909143
:10183000EC03009799F001979093EC038093EB03EE
:10184000892B61F48EEC98E290939B1280939A120C
:10185000DF91CF911F910F910C94286DDF91CF9163
:101860001F910F9108958F929F92AF92BF92CF9246
:10187000DF92EF92FF920F93CF93DF9300D01F92EE
:10188000CDB7DEB78091C21581111CC18091F40AD9
:10189000811110C00F900F900F900F90DF91CF919A
:1018A0000F91FF90EF90DF90CF90BF90AF909F90FF
:1018B0008F900895AADD0E9471954B015C01809183
:1018C000190290911A02181619060CF01CC1019702
:1018D00090931A02809319028091970E811117C07C
:1018E0008091E00A9091E10AA091E20AB091E30AA6
:1018F0000097A105B10559F0A5019401281B390BEA
:101900004A0B5B0B57FD03C081E08093970E6091FB
:10191000711670917216072E000C880B990B0F949C
:10192000183169837A838B839C833EE1E32EF12C0B
:1019300000E09E012F5F3F4F4BE656E16CED7AE0F1
:101940008BED9AE00E9410B6C0906B16D0906C168A
:10195000E0906D16F0906E168091580B9091590B97
:10196000BC01990F880B990B0F9418319B01AC01A6
:10197000C701B6010F94A23718160CF4A7C060E097
:1019800060930B0B8091E40A9091E50AA091E60A1E
:10199000B091E70A0097A105B10521F1A5019401D5
:1019A000281B390B4A0B5B0B57FD1CC06091E80AE2
:1019B0007091E90A80E090E00F9416319B01AC0130
:1019C00060916B1670916C1680916D1690916E16E9
:1019D0000F94123187FFBFC046E557E268E677E211
:1019E00080E032DD8091EA0A9091EB0AA091EC0A46
:1019F000B091ED0A0097A105B10511F1881A990A75
:101A0000AA0ABB0AB7FC1CC06091EE0A7091EF0AEB
:101A100080E090E00F9416319B01AC0160910E0BB9
:101A200070910F0B8091100B9091110B0F9412314C
:101A300087FF88C044E357E267E477E28FEF04DD75
:101A40006091120B7091130B072E000C880B990BF1
:101A50000F94183169837A838B839C839AE0E92EF3
:101A6000F12C0FEF9E012F5F3F4F4EE05BE066EDE4
:101A70007AE08AED9AE00E9410B68091960E81116C
:101A80003FC0C0900E0BD0900F0BE090100BF09069
:101A9000110B20E030E040EA50E4C701B6010F949A
:101AA000A23787FD0BC020E030E046E153E4C701D8
:101AB000B6010F94123118160CF046C060E0609326
:101AC0000C0BE8CE87E797E20F94F2156091350290
:101AD00070913602072E000C880B990B0F94183169
:101AE0009B01AC01C701B6010F94123187FF47CFAC
:101AF00080E00E94ED820F94C0367595679540CFC7
:101B000010920C0BC7CEC0906B16D0906C16E09064
:101B10006D16F0906E1620E030E848E953E4C701F6
:101B2000B6010F94A2371816CCF020E030E040EA5E
:101B300050E4C701B6010F94123187FFCDCE80E08B
:101B4000EFDCCACE0EDB7CCF0E94B0810F94C03692
:101B500075956795B4CF80E04FDB44CF80E0EADC39
:101B6000C0906B16D0906C16E0906D16F0906E16CB
:101B7000DCCFCF92DF92EF92FF920F931F93CF9320
:101B8000DF936C017A018B01C0E0D0E0CE15DF0558
:101B900089F0D8016D918D01D601ED91FC910190F4
:101BA000F081E02DC6011995892B11F47E0102C048
:101BB0002196ECCFC701DF91CF911F910F91FF903C
:101BC000EF90DF90CF900895089580E090E0089521
:101BD00080E008950B96FC01849108950A96FC011B
:101BE00084910895FC0184910895FCDF882321F0FD
:101BF000823011F083E0089586E00895FC01E60F3D
:101C0000F11D849190E0982F88273196E4918E0FF2
